:020000040000FA
:10000000F83F002045200000B563000031200000CB
:10001000312000003120000031200000312000009C
:10002000000000000000000000000000E9200000C7
:1000300031200000000000003120000031200000CD
:100040005D2200005D2200005D2200005D220000B4
:100050005D2200005D2200005D2200005D220000A4
:100060005D2200005D2200005D2200005D22000094
:100070005D2200005D2200005D2200005D22000084
:100080005D2200005D2200005D2200005D22000074
:100090005D2200005D2200005D2200005D22000064
:1000A0005D2200005D2200005D2200005D22000054
:1000B0005D2200005D2200005D2200005D22000044
:1000C0005D2200005D2200005D2200005D22000034
:1000D0005D2200005D2200005D2200005D22000024
:1000E0005D2200005D2200005D2200005D22000014
:1000F0005D2200005D2200005D2200005D22000004
:100100005D2200005D2200005D2200005D220000F3
:100110005D2200005D2200005D2200005D220000E3
:100120005D2200005D2200005D2200005D220000D3
:100130005D2200005D2200005D2200005D220000C3
:100140005D22000053B94AB9002908BF00281CBF2E
:100150004FF0FF314FF0FF3000F00CB8ADF1080C5C
:100160006DE904CE00F008F8DDF804E0DDE90223D3
:1001700004B07047704700BF2DE9F04786468C46B3
:100180000846089E154674461946002B40F0C1806B
:100190008542B2FA82F245D94AB1C2F1200300FA8F
:1001A00002FC954094402EFA03F343EA0C0C4FEA0C
:1001B000154EA8B2230CBCFBFEF80EFB18CC08FBB6
:1001C00000F943EA0C43994528D9EB1808F1FF37A9
:1001D00004D2994502D9A8F102072B44A3EB0903E5
:1001E000A4B2B3FBFEFC0EFB1C330CFB00F044EA94
:1001F0000344A04214D92C190CF1FF3304D2A042BD
:1002000002D9ACF102032C44241A43EA07401EB180
:10021000D440002334607360BDE8F0874746DDE7D3
:100220006346F1E792BB431B01214FEA154EAFB283
:10023000200CB3FBFEFC0EFB1C330CFB07F840EA62
:100240000343984561D9EB180CF1FF3004D298456F
:1002500002D9ACF102002B44A3EB0803A4B2B3FB18
:10026000FEFC0EFB1C330CFB07F744EA0344A742D9
:100270004DD92C190CF1FF3304D2A74202D9ACF1AD
:1002800002032C44E41B43EA0040C0E7C2F1200310
:100290009540944020FA03F12EFA03F34FEA154EED
:1002A0009040AFB20343B1FBFEFC0EFB1C10190CD7
:1002B0000CFB07F841EA0041884522D969180CF186
:1002C000FF3004D2884502D9ACF102002944A1EBE9
:1002D00008019BB2B1FBFEFC0EFB1C110CFB07F7E7
:1002E00043EA01439F420ED9EB180CF1FF3104D2CF
:1002F0009F4202D9ACF102012B44DB1B41EA0041D1
:1003000093E76046E3E76146F7E76046A4E76346A4
:10031000B8E7834206D916B9002108467CE7C6E94A
:1003200000E0F9E7B3FA83F78FB9834201D372454E
:1003300008D8BEEB020460EB030301209C461EB903
:10034000002169E73846FAE7C6E9004CF8E7C7F14B
:10035000200CBB400EFA07F522FA0CF42EFA0CF131
:10036000BA401C4320FA0CF3B8404FEA1449014349
:100370001FFA84FEB3FBF9F809FB18300B0C08FBDD
:100380000EFA43EA00439A4540D9E31808F1FF30DA
:1003900004D29A4502D9A8F102002344A3EB0A0330
:1003A00089B2B3FBF9F809FB183308FB0EFE41EAEA
:1003B00003418E452CD9611808F1FF3304D28E45D4
:1003C00002D9A8F10203214443EA0040A1EB0E0147
:1003D000A0FB02984145CE46434602D306D14D4587
:1003E00004D20138B9EB020E68EB0403002EA7D04B
:1003F000B5EB0E0261EB030101FA0CFC22FA07F3E4
:10040000F9404CEA0303C6E9003199E74046C5E7E5
:100410004346D9E7F0B5344B344A4921C3F80026A6
:100420003348C3F8042685B0C3F80826C3F80C2661
:10043000C3F81026C3F81426C3F81826C3F81C26E0
:1004400005F02EFF05F0D4FA00F098FA054601A851
:1004500000F03AFD0446284600F0A0FA254B1B6840
:10046000A34205D04521244805F01AFF05F0C2FB40
:10047000039A4921214805F013FF4921204805F03E
:100480000FFF4FF48031002002F0C2FE044620B17D
:1004900045211C4805F004FFFEE769469DF8080069
:1004A00000F034F8009B039D1D44019B1E8902F05F
:1004B00097FEAF1901F078F801F048F801F062F802
:1004C00084F30B8884F30A88AB5983F3088884F398
:1004D0001488BFF36F8FBFF36F8F7B6898474521F8
:1004E000094805F0DDFEFEE7008001503546526EFA
:1004F0006073000008000020797300009C73000006
:10050000CB730000F073000023740000024608B5AE
:1005100038B105480023452105F0C2FE6FF01500F3
:1005200008BD0860FCE700BF4674000021B1012946
:1005300006D06FF015007047044B53F83000704739
:10054000024B03EBC0035868704700BFB86F000050
:100550002DE9F04FDFF848B2DDB01646DDE96889D5
:100560001C466A9FDBF8005000F0BAFF0122884B5E
:100570003CA8C3F8002504F059F9B8F1000F07D0E2
:10058000B9F1000F04DD4A4641463CA805F085FD5F
:100590004FF0000833897289D6F80CA013449A44AE
:1005A000C24565D80FA93CA804F0B2F90022784BE7
:1005B000C3F80025C3F8002527B1202238460FA92B
:1005C00005F039FF00233146009322464FF6FF73B2
:1005D00009A805F00EFA064600285AD120460E9FBB
:1005E00000F0B6F9874254D84FF0FF37DFF8B4A1D6
:1005F000DFF89C810DF11E0307AA08A909A805F0E0
:1006000046FA002845DB40F0BA80089909A805F0B1
:100610008AFA50B94FF6FF71BDF81E005D4A32F8F4
:10062000023B8B4235D09842F9D1BDF81E90B9F10A
:10063000100F38D1BDF81C90B9F1200F29D14B46CD
:10064000204608993CAA05F039FE10BB00F096F947
:100650004A4606463CA90FA800F028F981463046D4
:1006600000F09CF94C4B1B684B4512D10126C1E7A9
:10067000679BAAEB0809994528BF994641464B4616
:100680002046669A05F01AFE30B10022404BC3F8AE
:100690000025DBF8005074E04A4666993CA805F056
:1006A000FCFCC8447CE7B9F1010F41D1BDF81C3016
:1006B000202BEED8204608993CAA05F0FFFD0746FE
:1006C0000028E6D19DF81C30202B039309D8DAF8D6
:1006D0000020324B0492049A974205DB0023C8F8AD
:1006E00000354FF0FF3785E7059300F0F9FEC8F8B5
:1006F00000951FA804F09AF8059B1FA85A6853F8A4
:10070000081B1268059305F0C8FC17A91FA804F080
:10071000FFF80022C8F80025039A3CA917A805F0A5
:100720007AFE059B10B9C8F8000563E70137D2E7E8
:10073000B9F1220F7FF45EAF7B1C3FF45BAFDAF8B8
:100740000030BB42CDDDBDF81C30802BA1D8204647
:1007500008993CAA05F0B2FD00289AD100F00EF9E4
:10076000FFB281462021BDF81C303CAA00970FA89B
:1007700000F01AF80546484600F010F9B1E7002EDF
:1007800087D000F003F928465DB0BDE8F08F00BFC8
:10079000000084503473000008000020C46F000083
:1007A00004000020C06F00002DE9F04796B0164607
:1007B0001D469DF87820384B074653F8321003EB5E
:1007C000C2035B6801911868DFF8DC8001443023C4
:1007D00002AA01A8D8F8009005F0EDFB002851D13D
:1007E000DDE901431C44214606AB03AA01A805F03C
:1007F0000AFC002846D1049A072A43D127490598C4
:1008000005F009FE00283DD1079A082A3AD124496B
:10081000089805F000FEA8BB214602AA01A805F031
:10082000DEFB78BBDDE901A30AEB0302944229D188
:10083000412B27D135443023294603AA02A802962A
:1008400005F0B9FBE0B9DDE9023213449D4217D34C
:100850002A4602A906A805F074F988B92A4602A911
:100860000EA805F06EF958B99AF80030042B07D19C
:100870002023384606AA0AF1010100F049FE38B1EA
:10088000D8F8009000F082F8484616B0BDE8F0872E
:10089000044BD3F80090F5E7C46F000075740000B6
:1008A0006C740000080000200400002070B5094BA3
:1008B00004461D680023934205D1074B1D6800F0D4
:1008C00065F8284670BDE65CC85C8642F7D1013306
:1008D000F1E700BF0400002008000020094A4000A2
:1008E0000B7852F820108B4209D0013052F82000CA
:1008F000834214BF4FF0FF304FF4C07070474FF485
:10090000C0707047CC6F00001FB50F4B0C4613F83A
:10091000300001F0E1F950B92068102381686A467F
:10092000103905F0CBFC28B1206805F0C6FC4FF06B
:10093000FF3006E010226846044905F06CFD0028EF
:10094000F2D104B010BD00BFCC6F000050730000A6
:1009500013B5044605F026F96A460146204605F01F
:100960002EF830B10448452105F09AFC002002B071
:1009700010BD0098FBE700BF7D740000024B1868B3
:10098000421C1A60704700BFD8010020024A136859
:10099000013B1360704700BFD8010020034B1B6868
:1009A000834201D005F026B9704700BFD80100206E
:1009B0002DE9F04F414B8BB0064600200D461C68D8
:1009C000FFF7B4FD08A9C0B201F086F928B1FFF71E
:1009D000DDFF20460BB0BDE8F08F2946FFF7A6FDEE
:1009E0004FF02C0B09A9C0B20BFB056B01F074F999
:1009F000002844D02C276F4306EB0708D8F8104096
:100A000014F010044CD1FFF7B9FF089B81460793FF
:100A1000FFF7B4FF4FF480720192294A21468246C3
:100A2000CDE90344079B0294009220465A46FFF703
:100A30008FFD04465046FFF7B1FFFFF7A7FF48467A
:100A4000FFF7ACFF1F4BF25908989A420CD1D8F827
:100A50000C20B8F808309B1806D28268934203D263
:100A6000194B1B68A34222D02DB38268002105F0E8
:100A70004FFC164A4521164805F012FC15E009986E
:100A800005F063FC0446099805F017FC0BF1FF33F1
:100A90000BF1030213F8011FA142ABD19342F9D12C
:100AA0001DB13046089905F07AF90A4B1C68089880
:100AB00005F003FC8BE7084ADCE700BF04000020D8
:100AC000EC0E00203DB8F39608000020C074000032
:100AD000CA74000000000020B87400007FB50D4605
:100AE000002104462846CDE9021105F017F928B384
:100AF0002368194EB34203D1204603AA05F0A3F898
:100B0000E36AB34204D10121204602AA05F09BF812
:100B1000DDE90232934288BF0393039BAB60039AE3
:100B20002946204600F0DAFB0C4B1A68002A03DD48
:100B300057210B4805F0B4FB04B070BD01A9FFF7C5
:100B4000E3FE019805F1080105F037F8AB6801985C
:100B5000039305F0B2FBE2E73DB8F3963C0E0020AC
:100B6000F27400002DE9F84F884691469A46002617
:100B7000DFF870B0194C1A4D0B9B9E4201D3002038
:100B80000FE00B9B40469F1BB7F5806F28BF4FF4CB
:100B90008067144A3B4606EB0A0105F08FFB10B153
:100BA0000120BDE8F88F0A993B465A46484671181D
:100BB00005F099FB0028F3D1C4F800563E44C4F870
:100BC0000456C4F80856C4F80C56C4F81056C4F8B5
:100BD0001456C4F81856C4F81C56CDE700800150CE
:100BE0003546526EDC0900202DE9F0410E46002109
:100BF000AB4B04464362AB4B88B003650846FFF736
:100C000095FC04F120010546C0B201F065F848B139
:100C100000232A46452101900093A34805F040FB9C
:100C200004F0E8FF01210020FFF780FC04F14C01F3
:100C30000546C0B201F050F850B101232A464521C3
:100C4000019000939848002305F02AFB04F0D2FF9E
:100C5000204605F039F8054668B9002220461146BD
:100C600004F0DBFF054600B3002257218F4805F052
:100C700017FB01239EE0802257218D4805F010FBD1
:100C800001239D4284F85830E7D194F85830042B62
:100C90008DF8173000F29180012B00F2958000F062
:100CA000A880FF2384F85830A3E0204600F028FAFB
:100CB0000028DED004A805F028F80146204605F0FB
:100CC000C3F818B12A4657217A48D0E704A805F09E
:100CD00025F880F0010104AA2046C9B204F09DFF66
:100CE00002460028C0D104A805F018F8054660BBEC
:100CF000204604A9FFF7F2FE9DF8173084F858301B
:100D0000033B012B06D8284600F00EF910B1FF2353
:100D100084F858309DF81730023B022B0BD8002086
:100D200000F0ECF838B1FF2384F8583045216248D0
:100D300005F0B6FAFEE794F85830FF2BF6D0002104
:100D4000204604AA04F069FF93E79DF81770012F6D
:100D50001ED1104602F0F0FA831E022B054614D86D
:100D6000FFF70CFE394680462046FFF721FE074676
:100D70004046FFF713FE514B1B689F4205D0504B76
:100D80001D68AF4214BF0525012584F858507CE743
:100D9000FFF7F4FD012107462046FFF709FE05464F
:100DA0003846FFF7FBFD454B1B689D4214BF0523EA
:100DB0009DF8173084F8583067E7052B7FF471AF42
:100DC000002000F0B1F811E0204604A9FFF786FEEC
:100DD00094F85830DA1E012A34D8002000F0A4F824
:100DE00000287FF45EAF002000F088F800287FF430
:100DF00058AF94F85830FF2B05D145212E4805F007
:100E00004FFA04F0F7FE002294F858302D4F012BD2
:100E100003921AD01146204604F0FFFEA8B13D68A7
:100E2000102200210DEB020005F010FBE06C05F034
:100E300044FA206A05F041FAFFF7A8FD284608B0F9
:100E4000BDE8F081022BD4D1CDE7FFF797FD00215B
:100E500080462046FFF7ACFD05464046FFF79EFD65
:100E6000DFF85880D8F800309D42D8D13B689D42C9
:100E7000D5D0134B1B689D42D1D0039B0133039304
:100E8000039B012B01D004F0B5FE206A04F095FD10
:100E90003071236A5B683460D8F80050B360BFE7F4
:100EA000DC050020DC01002021750000B075000089
:100EB0006E750000DC75000006760000080000205A
:100EC000000000200400002070B50B4E0446602294
:100ED0000021304605F0BAFAFFF750FD21460546DD
:100EE0003046FFF781FE04462846FFF757FDFFF71F
:100EF0004DFD204670BD00BFDC0D002013B5094B31
:100F000001A913F8300000F0E7FE48B9019805F098
:100F100074FD0446019805F0D0F9204602B010BDDA
:100F20000124FAE7D46F00001FB50F4B01A913F895
:100F3000300000F0D1FEA8B9019802A902F0A6F98C
:100F4000044668B99DF80B30032B03D1019805F0D6
:100F500022FD0446019805F0B0F9204604B010BD0A
:100F60000124F7E70124F8E7D46F00002DE9F341ED
:100F700006460C4617461D460BB9002628E01846C3
:100F800004F0CCFE0028F8D16946FFF7BDFC0098BC
:100F900038B90124009805F090F9204602B0BDE868
:100FA000F08101A904F009FE0028F2D1009805F0B3
:100FB00084F93046019904F095FF736A5E686B7995
:100FC000012B21D1002CD8D12B68834298BF002659
:100FD00021460020FFF7AAFA6946C0B200F07CFE65
:100FE0000028D6D120233A463146009805F066F90C
:100FF00004460028CDD1002DCCD03C680D4BE41A1E
:1010000018BF4FF0FF34C5E7022BB6D12B68012B78
:1010100005D98342B1D8B4FA84F46409ADE7ACD100
:10102000002CD5D0012CA8D12C79023C18BF01246A
:10103000A3E700BF3DB8F3962DE9F04F07460C46F5
:1010400085B0014600201646FFF748FC051E50DB20
:101050003846E46D04F0A6FD5FFA84F94FF0000A0B
:101060004FF0010B4FF0FF346B1E09FB03089DB9D5
:10107000BAF1010F03DD4521204805F011F9631C89
:1010800006D07F2C2ADC40F2011301343460B38097
:10109000284605B0BDE8F08F6B1E00934146012342
:1010A00038460DF10F0205F009F9031E019322DB0A
:1010B000012238460DF10F0105F008FC019B40B1FB
:1010C0005B4501D00AF1010A9B46009DA8EB090887
:1010D000CDE7B4F1FF3F08BF2C46F5E70223803C83
:1010E0007371631004F0010401330134336034710F
:1010F000CEE70725CCE70125CAE700BF127600003E
:1011000070B5866A456D044604F0DBFEAE420AD037
:101110006B1CB34207D0834205D05721134805F01A
:10112000BFF8002070BD802E1CD957211048F6E76B
:10113000626A216D02EBC30201EBC3015268496888
:10114000914202D057210B48E9E701339D42EFD18C
:10115000AE4205D9636A03EBC5035B689342F1D1E4
:101160000120DFE700231A46F0E700BF35760000D4
:101170006D7600009C76000000B589B0032004A9BC
:1011800005F016FC9DF81020012A41D0254B264978
:10119000032A08BF0B469DF81320492102929DF8AF
:1011A0001220224801929DF811200092204A05F059
:1011B00077F8092006A905F0FBFB9DF81820012A05
:1011C00028D0184B1849032A08BF0B469DF81B204E
:1011D000492102929DF81A20144801929DF8192085
:1011E0000092144A05F05CF89DF81030012B13D1E1
:1011F0009DF81230032B0FD19DF81830012B0BD026
:101200000D48492105F04CF8022009B05DF804FBB7
:101210000A4BC0E7094BD9E70948492105F040F8D6
:101220000020F2E7C8760000D1760000E5760000E5
:10123000D77600002677000036770000CC760000D5
:101240005577000070B54B6814461E4A03F0FF2323
:10125000934206460D4686B02FD10B68012B2CD148
:10126000204604A902F012F89DF81020012A26D089
:10127000154B1649032A08BF0B469DF81320492138
:1012800002929DF81220124801929DF811200092BE
:10129000104A05F005F89DF81030032B0DD12146BA
:1012A000304604F07CFD204605F075FB2046A96819
:1012B00004F091FC204601F0C9FF06B070BD064B5A
:1012C000DBE700BF00010004C8760000D176000013
:1012D000E576000026770000CC7600002DE9F04F7F
:1012E0001646054689B00C467448492104F0D8FFDB
:1012F0003146284604F0F6FD6B6A824620465E6859
:1013000004F00CFDE8B1E86D04F047FC0023AF6A7F
:10131000013F3344834201D2013FFAE7BA4510D37B
:101320005721674804F0BCFF07FB06F357210AFB6F
:101330000662644804F0B4FF0123E37109B0BDE81C
:10134000F08F06A9032000F0C7FC07A9092000F0D0
:10135000C3FC21462846079AFFF774FF6379012BE7
:101360004BD15746DFF860B141E02268C2F101037A
:1013700053449F423AD86B6A012A196853F83700E0
:1013800003EBC70353F8083CA0EB0109A3EB0103EF
:10139000049311D1079B0393E368022B08D04146C5
:1013A000284604F0FCFC22464146284604F02DFD68
:1013B0002846039904F0F3FC32464946404604F0BF
:1013C000ECFC049B424641462846CDE90096FFF7D7
:1013D000C9FB2146284604F0AEFC23680133236094
:1013E00020B1DBF800300133CBF80030013FDDF8ED
:1013F0001880002FB9D101232360022301276371D4
:10140000BA45DDF8189006D2484604F056FF079812
:1014100004F053FF92E723689F424DD36A6AFB00B2
:1014200052F83710083B04911168DDF81CB00391A5
:10143000D1582A6DD0581368A0EB03082379012BEB
:1014400038D1039B3246C91A4846059104F0A5FCE1
:10145000059943464A460091284659460196FFF7AA
:1014600081FB2146284604F066FC0223237118B153
:10147000154A13680133136032464146584604F05A
:101480008CFCDDE9032349469B1A28465A46CDE9E0
:101490000086FFF767FB2146284604F04CFC2368D2
:1014A000013323600123237130B1074A13680133EC
:1014B000136001E0022BDFD00137A1E76C77000059
:1014C00095770000C47700003C0E00200A4619B151
:1014D000024B00211B681847704700BF0C0000201A
:1014E00070B5094D2B780BB1002070BD0126074C5B
:1014F000C4F8006503F03CFA18B92E70C4F8000572
:10150000F2E74FF0FF30F0E7EC0F002000008450CE
:101510002DE9F041ACB01F4606460C461546FFF7D4
:10152000DFFF0123DFF820802A46C8F80035214676
:101530003346009703A805F09FFB0023C8F8003549
:101540002CB0BDE8F08100BF00008450BFF36F8F66
:1015500072B600234FF0FF30094A03F12001013336
:10156000102B42F82100F8D100234FF0FF30044A3D
:1015700003F160010133102B42F82100F8D17047CC
:1015800000E100E0002318460649D1F89020C2F39C
:101590000722934200DB7047C1F89830C1F8A000E1
:1015A0000133F6E700ED00E02DE9F8434FF0FF3599
:1015B00001274FF00008204BDFF884905F60C3F8EC
:1015C0004853C3F8085303F580535F60C3F848538A
:1015D000C3F8085359F8044B002644F30730C4F805
:1015E000085300F09FFD80226760C4F84C61D4F876
:1015F0004C31C4F81061D4F81031C4F8446131465C
:10160000D4F84431A018C4F8006504F01FFF80220C
:10161000314604F5C07004F019FFB8F1000F08D08E
:10162000064BC3F808554FF05023C3F80853BDE8E4
:10163000F8834FF00108CDE70040015000700150E1
:10164000E06F0000014B1B68184700BF100000202E
:1016500007B50B46002102460091034800F00CF844
:1016600003B05DF804FB00BF45160000014B186095
:10167000704700BF100000202DE9F04F82464FF068
:1016800000098DB01D46531E01910393039B5878AA
:101690005C1C252819D100204FF0FF381E46444617
:1016A00003460236029031780396392955D81F290E
:1016B00014D8002900F0EF8101992520D047019925
:1016C0003078D04709F10209E0E7002800F0E38113
:1016D0000199D04709F101090394D7E7A1F120024C
:1016E000192AE9D801A757F822F000BF55170000C2
:1016F000B9160000B916000055170000B916000011
:10170000D5170000B9160000B9160000B916000080
:10171000B91600002118000055170000B916000086
:1017200035180000E1170000B9160000EF1700009F
:101730000F1800000F1800000F1800000F1800000D
:101740000F1800000F1800000F1800000F180000FD
:101750000F18000008460136A5E7582900F0EB8075
:10176000A1F16302D7B2172FA6D8172AA4D801A7D0
:1017700057F822F0DD1900005B180000B9160000D0
:10178000B9160000B91600003B1800005B180000F5
:10179000B9160000B91600003B180000B916000089
:1017A000B9160000B916000011190000B9160000A2
:1017B000B9160000B1190000B91600005B1800004E
:1017C000B9160000B916000011190000B916000082
:1017D0003B18000025200199D04709F1010955E780
:1017E000029A4FF0000802F0FE020292B3E7002CCA
:1017F0000DDAB8F1000F0DDA029A002A00F04381E9
:101800000A2224EAE47402FB0414303CA3E7B8F192
:10181000000FF5DB0A2202FB0812A2F130089AE75A
:10182000B8F1000F55F8042B80F22F81002A80F2C6
:101830002E815442022202928DE7682903D1682B3F
:1018400006D1482387E76C2902D16C2B00F0218157
:10185000002B7FF431AF0B467DE77A2B06D175293B
:1018600055F8046B14D14FF0000B0CE06C2BF6D044
:101870004C2BF4D1073525F00703752903F1080532
:10188000D3E9006B06D120283BD1854F013C09E00C
:101890004FEAE67BBBF1000FF5DA7642814F6BEB46
:1018A0004B0B013C0DF12D030593002304933046AF
:1018B00059460A220023FEF745FC059BB446303208
:1018C00003F8012D5A460593049BBCF10A0F8B4681
:1018D00072F1000203F1FF3106460491E7D2C3F131
:1018E000010B30330DEB0306B8F1000FA6F104062F
:1018F0006DDA029BD9077DD4A8EB0B03A4EB0B0494
:1019000013E02B280ABF684F684F04F1FF34C9E782
:1019100070290FD155F8042B0023FAB96FF0040396
:101920004FF0050B614F624E053C029A920770D44E
:10193000A04666E078216C2B03D1002355F8042BD8
:1019400008E04C2BF9D1073525F007031D465B68ED
:1019500055F8082B232825D1880621D5554F023C60
:10196000002601F06001A1F1390B0DF12D0E02F0FE
:101970000F01092988BF594430310EF8011D102A82
:101980004FEA121141EA03714FEA131C73F100038D
:1019900006F1FF3008D2C6F1010B06F13003A1E7D2
:1019A000454FDCE7414FDBE706460A466346DEE784
:1019B00055F8046B304604F027FDB8F1000F83465C
:1019C00002DB4045A8BFC3464FF00008374FA8EBE5
:1019D0000B03002B92DDA4EB0804A6E755F8043BAB
:1019E0004FF0010B8DF81830304F4FF0FF33013CB2
:1019F00006AE9AE7A046EAE7029320200199D04775
:101A0000029BB8F10108F7D524EAE472013C914445
:101A1000A41AB84606E0049302920199D047029AAC
:101A2000049B9046424612F8010B0028F3D11A4657
:101A3000013A15D5002BACBFC7EB03077F425B46CD
:101A4000013B15D5BBF1000FA8BF5F4426464F44AC
:101A5000013E14D5002CA8BF3F1907EB080915E675
:101A60000493029230200199D047049B029ADFE749
:101A70000293019916F8010BD047029BE0E7019908
:101A80002020D047E4E70122D5E6904663E61446DD
:101A900061E64C235FE648460DB0BDE8F08F00BF1D
:101AA0005278000050780000547800001176000051
:101AB0005C78000056780000597800002DE9F04766
:101AC000058B04462807904611D4022905F0070526
:101AD00040F0CC80204604F00AFB78B10138218B1D
:101AE000042811D8DFE800F0C2106D8595000129A7
:101AF0000CBF45F0100545F02005258388F31188BB
:101B0000BFF36F8FBDE8F08701F0070AAA4500F028
:101B1000A5800027B9463E46A368002B00F0BC8094
:101B200041F00801218388F31188BFF36F8FA1680A
:101B3000002900F0BA800D68002900F0B680334615
:101B400052462046D1F80480C047002D76D02B683D
:101B500029461D46F0E701F007035A1F012A1BD84A
:101B6000002221F00701062B276889B2C4E9002270
:101B700009D13B4603E0628B013262831B68002B74
:101B8000F9D141F002012046218304F0B0FA002887
:101B90007AD041F0200176E0042B0AD121F0070130
:101BA00089B22046218304F0A2FA10B141F020014D
:101BB0002183218B01F0070AAA454FD00027B9469F
:101BC000AAE7236921F0070141F00601062DD3F8A9
:101BD000009021832DD1B9F1000F3FD041F00801D1
:101BE000218388F31188BFF36F8F20463949C84796
:101BF00029E021F00701236941F0040189B2042D95
:101C0000D3F804902183E6D000274FF0040A3E4623
:101C100082E721F00701236941F0050189B2052D12
:101C2000D3F808902183D6D000274FF0050A3E460E
:101C300072E700274FF0060A3E466DE72B4687E71E
:101C4000B9F1000FD1D1EFF31188202383F312886B
:101C5000BFF36F8F238B23F008032383258BEA06C2
:101C60002ED525F01003238305F007056669218B27
:101C7000002EBFF670AF00232768C4E9003321F0BF
:101C8000070141F001012183218B4FF0000901F090
:101C9000070AAA457FF440AF002F9CD041F008010D
:101CA000218388F31188BFF36F8F002FC8D03D6860
:101CB000394633465246204604F045FA2F46F4E7AB
:101CC000AB067FF51BAF25F02003238305F0070546
:101CD00000E700BF7361000070B5114B0D461C6832
:101CE000DCB1104B196800238B4202DB6FF001005E
:101CF00070BD224612F8106B864202D014460133A2
:101D0000F2E7E06810B96FF01200F1E704F06DFF40
:101D10000028F8D000202C60EAE76FF00C00E7E71D
:101D200014000020E86F000070B588B005460C462E
:101D3000C0B269461646FFF7CFFF00281BDB0098AC
:101D4000C8B143682268029383680195CDE90336E0
:101D50000023CDE906230593C56804F0AEFA6DB102
:101D60002846084901AA04F07AFC079808B9059B9F
:101D7000236008B070BD6FF01500FAE76FF0120035
:101D8000F7E700BF5963000008B5054804F0A2F961
:101D9000044804F09FF9BDE80840034804F09AB9EC
:101DA0006278000093780000C6780000014802F0D5
:101DB0008FBA00BF8C70000030BFFFF7FDBF00BFBF
:101DC000154B9A6A12F0007F9A6A14BF1E201D20DC
:101DD00012F0807F9A6A18BF1F2012F4801F9A6A3F
:101DE00018BF022012F4002F9A6A18BF212012F4A3
:101DF000802F9A6A18BF222012F4003F9A6A18BFF7
:101E0000232012F4803F9A6A18BF24206FEA02420E
:101E10006FEA12429A62704700ED00E010B5194B6C
:101E20000246986A9C6A10F4805F14BF172016203F
:101E300014F4006F9C6A18BF1820A40509D5986B8C
:101E4000986A000404D51AB19A6A22F400429A6290
:101E500019200C4B9A6A12F4806F9A6A18BF1A20E4
:101E6000D2050CD49B6A13F4005F18BF1C20054AEE
:101E7000936A43F47F43936200230B7010BD1B20D1
:101E8000F5E700BF00ED00E010B51C4B0246986A74
:101E90009C6A10F0100F14BF1120102014F0080FCE
:101EA0009C6A18BF1220A40709D5586B986A0006CF
:101EB00004D51AB19A6A22F080029A6213200F4B5D
:101EC0009A6A12F0010F9A6A18BF142012F0200FBC
:101ED0009A6A18BF1520D40658BF9B6A074B9A6AA6
:101EE000920642BF5A6A22F400525A629A6A42F03B
:101EF000FF029A6200230B7010BD00BF00ED00E0EE
:101F000070B5444B06465B6800258AB0C3F30803EE
:101F100085F31188BFF36F8F02F07F40B0F17F4FE0
:101F200011D102F00C0008280DD010074CBF0E464E
:101F300001250022033B8DF80720032B05D8DFE89D
:101F400003F01E5C60592E46F3E700249DF807302D
:101F50009BB92022314602A804F06DFA099B002D9E
:101F600053D0C3F3080222B96FEA53236FEA432325
:101F70000993204602A904F013FA0AB070BD254B5C
:101F8000DA6A9107E1D4DA6A002ADEDBDA6A520003
:101F9000DBD55A69B16942F480725A61BFF34F8F41
:101FA000BFF36F8F5A6931F8021C22F480725A61B4
:101FB000BFF34F8FBFF36F8F4DF60272914209D07E
:101FC0009A6AD2B242B101200DF10701FFF75CFF1E
:101FD0000446BBE73468B9E79A6A12F47F4F05D02C
:101FE00001200DF10701FFF719FFF1E79B6AB3F537
:101FF000803FAAD3FFF7E4FEEAE700200DF10701D6
:10200000E4E700200DF10701EDE723F4FF7323F06F
:102010000103ADE700ED00E0044B5A6942F0100205
:102020005A615A6942F480625A61704700ED00E0DB
:10203000EFF30880EFF3098101B57246FFF760FF07
:1020400001BD00BF002080F31488BFF36F8F002014
:1020500080F30A8880F30B8801F02CFA00200E49E7
:102060000860BFF34F8F0D4880F3088800F01AF81E
:10207000202080F311880A484FF40061401880F353
:102080000988EFF314800221084380F31488BFF31A
:102090006F8F00F07FF8000094ED00E0F83F002023
:1020A000F80F002072B6002383F313884FF0FF303F
:1020B0000C4A03F120010133102B42F82100F8D122
:1020C00000234FF0FF30074A03F160010133102B6A
:1020D00042F82100F8D162B6BFF34F8FBFF36F8F84
:1020E000704700BF00E100E01EF0040F0CBFEFF3EB
:1020F0000880EFF30980816911F8021C0229FFD0E2
:1021000001B504F053F901BD40B2002807DB0123FB
:102110004109034A00F01F00834042F82130704714
:1021200000E100E040B200280CDB0122064943092F
:1021300000F01F008240203341F82320BFF34F8F6F
:10214000BFF36F8F704700BF00E100E0054B42090D
:1021500053F82220012300F01F0003FA00F0104082
:10216000704700BF00E100E040B2002801F101012A
:10217000ACBF00F16040064B4FEA4111C9B2ABBFA2
:1021800000F5614000F00F0080F80013195470470B
:1021900014ED00E0144A08B5144B22F07F029A6057
:1021A000BFF34F8FBFF36F8FD3F8882022F47002F4
:1021B000C3F88820D3F8882042F4A002C3F888200E
:1021C0004FF04042C3F83422BFF34F8FBFF36F8FFD
:1021D0000023E1EE103A01F029FF01F06BFF00F05F
:1021E00031F801F02FFF00BF0000000000ED00E01B
:1021F0001E4680B50C46074615460023E1EE103A10
:1022000083F30B88DFF824C0ACF5205E8EF30B88D7
:102210008CF309884FF0000005498847204629467D
:102220003246B84703488047FEE700BFF83F00202A
:10223000CD630000DB6300001022014B1A61704780
:1022400000ED00E0002320210348C2180133412B98
:1022500082F80013F9D1704700E100E008B5EFF310
:102260000583064A103B02EBC30152F8330049686C
:102270008847BDE8084004F0A4B800BF8C6D00009A
:10228000014B1860704700BF180000200122024B6C
:102290000020C3F8402570470090035020B1034B45
:1022A000800143F001031847704700BFB06F000082
:1022B000084B70B5C31A0D4607499B100446594395
:1022C0004022064804F0D7F82B4601462046BDE8D8
:1022D00070401847540E0020B76DDBB6286D000023
:1022E000402373B50B4C0093041B0B460D460A4963
:1022F000A41061430646094A094804F0E7F8011EA4
:1023000005DA30462B4602B0BDE87040184702B0EF
:1023100070BD00BF540E0020B76DDBB63B650000FA
:10232000286D000010B5EFF31184202383F3128889
:10233000BFF36F8F074A136823F00201DB071160B8
:1023400002D4012004F0E5FB84F31188BFF36F8F02
:1023500010BD00BFA40E002070B50022012104466C
:102360000520FFF701FF0F4801F0CEF90E4B984210
:1023700015D101F0D9F926690C49304603F007FF61
:1023800000280BDB012535642469084904F11C0091
:1023900003F0FDFE002801DB0020E56470BD6FF056
:1023A0000400FBE7792400000000AD0B94700000EE
:1023B0000C22104B014602FB0033002030B4D3E95D
:1023C0000E529863EFF31180202484F31288BFF338
:1023D0006F8F1C6C04F0C00444F002041C6480F392
:1023E0001188BFF36F8F1DB12B4630BC02481847D0
:1023F00030BC7047540E0020286D000010B4EFF37D
:102400001182202383F31288BFF36F8F184801686D
:1024100041F002040460C80708D482F31188BFF3B6
:102420006F8F01205DF8044B01F092B94FF05021FD
:10243000D1F80C04D1F80C14C907EED5EFF31180D4
:1024400083F31288BFF36F8F0A490B6C03F0C0034C
:1024500043F002030B6480F31188BFF36F8F82F3A4
:102460001188BFF36F8F00205DF8044BFFF7A0BF0A
:10247000A40E0020540E002010B1012804D0704793
:10248000034B1B6C5B0701D1FFF792BF704700BF86
:10249000540E00202DE9F843012207463449D1E8C3
:1024A000EF3FC1E8E02F0028F9D133B93149324874
:1024B0004B60CB608A6003F07DFE7B1E012B2DD824
:1024C000012F07D14FF05023D3F81C3403F003033E
:1024D000022B23D004F0CAFB054608BB274B1B7810
:1024E000F3B14FF0502302220646C3F808234FF001
:1024F00050244FF00008DFF88890D4F81824D4F85E
:102500001834D20315D503F00303022B01D0012F99
:102510000FD135B386F31188BFF36F8FBDE8F88311
:10252000EFF31186202383F31288BFF36F8F012509
:10253000DDE7304603F059FFD4F81835DBB2012B44
:10254000DBD1D4F80421002AD7D0C4F80481D4F810
:1025500004210222C4F818252022C9F88021A36092
:10256000CBE74FF050230222C3F80423D6E700BF85
:10257000500E0020400E0020700E0020F10F0020B1
:1025800000E100E008B5074804F02FFB38B1064829
:10259000FFF776FE0448FFF769F8002008BD6FF0EA
:1025A0001200FBE7646D0000AD2500000A2838B575
:1025B0000446074D04D1AB680D2128465B68984757
:1025C000AB6803485B68E1B29847204638BD00BF5E
:1025D000646D0000024B0B6001231360704700BF65
:1025E000A80E002000487047E870000010B504F005
:1025F000F4FA034C206004F0EDFA6060002010BD96
:10260000A80E0020F8B50E461946304617461D465E
:1026100003F0A3FFB8B146EA050414F0030412D195
:102620004DB12B19032BA6EB040006D8074AD2F8AC
:102630000034DB07FBD50020F8BD3B1B196801F017
:10264000B7FC043CEDE76FF01500F5E70090035090
:1026500038B545682B69B3B11035284601F066FBE3
:10266000044680B90146284601F02EFB084B9842EB
:102670000BD122462846074901F00EFB22460521D0
:102680000D20FFF771FD002038BD6FF00400FBE75F
:102690000000AD0B99260000430970B507D10B4B24
:1026A000596821B101250C68094E854001B970BDFA
:1026B0008A682A4002D030464B6898471CB123688C
:1026C00021461C46F2E72346FAE700BFB00E002081
:1026D0003C6D00002DE9F04340F206354668D00617
:1026E00048BF0320337B02EA050558BFC2F3401000
:1026F00087B001F01F07B5F5837F144647EA4317FB
:102700008DF8030041D00FD8062D18D007D8B5B1E9
:10271000022D3CD06FF0150007B0BDE8F083B5F591
:10272000807FF7D101250AE040F20222954230D0A5
:10273000B5F5407F2FD0B5F5007FEBD10225220300
:102740002BD5012372688B409360326962BB07F01E
:102750001F037F0975D13D4A84F4803102EB830267
:10276000D2F80032C1F30041C4F3404423F4E163E2
:1027700044EA410423F007031C4344EA800444EA8A
:102780000524C2F800420020C6E70725D7E7042544
:10279000D5E70525D3E70325D1E7630341BF01232F
:1027A00072688B40D360D0E71036394630460DF161
:1027B000020201F077FA14F4403F80460CD139460A
:1027C000304604F000FA224B9845DCD130469DF8A3
:1027D000021001F0B5FAD6E74FF0000901AB394617
:1027E000304603AACDE90439CDE90199CDF80C9022
:1027F00001F02CF9164B98428CD114F4003315D00B
:102800009DF8033084F48034C4F300448DF80E3016
:1028100039464B46304603AA8DF80C508DF80D40D2
:1028200001F0C2F90A4B9842CDD073E7CDE90433E9
:1028300039460DF10303304603AA039301F006F96C
:10284000F0E7803352F82330FFDE00BF00258450CC
:102850000000AD0BF0B5406801F01F04057B87B0A8
:1028600044EA45140569002D5FD0B2F5001F00F160
:10287000100506D12146284604F0A7F9002007B02C
:10288000F0BD0027B2F5800F01AE0197776037D118
:10289000B3F1007F14BF052304238DF80430002317
:1028A000CDE904630393836823FA01F111F0010178
:1028B00018D1B2F1A07F15D104F01F03620903F112
:1028C000800338D11D4A52F82330DB070AD40DF1BA
:1028D000030632462146284601F0E4F9184B984297
:1028E00019D002962146284603AA01F0AFF8154BED
:1028F00098421DD101222146284601F02DFABDE75C
:10290000B3F1C06F05D0B3F1007F14BF01230223E0
:10291000C3E70323C1E73146284601F017FA094B04
:102920009842DED06FF00B00A9E76FF08500A6E7B4
:102930006FF01500A3E751F82330FFDE0025845027
:102940000400AD0B0000AD0B2DE9F04740F2FF167F
:10295000594FDFF868C1DFF868E100EB810181427F
:1029600002D10020BDE8F087046814F4804FC4F35E
:10297000C325C4F3080340F08C80640CB34208BF45
:102980004FF0FF337D5D192C00F28680DFE804F004
:102990000D13191C1F251C84848484366084848450
:1029A00084848484848463787B7EC2F80C355C1CC8
:1029B0005BD10430D3E7C2F814355C1CF9D0002495
:1029C0005CE0C2F80835F2E7C2F81035F5E75C1CA8
:1029D000C2F80835EDD0002404E05C1CC2F80C35C8
:1029E000E7D001245FEA531859D14FF00109DFF80D
:1029F000CC8009FA03FAC8F80CA008E0C2F8083540
:102A0000002DDAD15C1CD4D000240625A146D0F8D4
:102A100000A00AF40048B8F1000F1CBF4FF00009F5
:102A2000012403F01F085B093FD10CEB8808D8F89C
:102A30000032CAF3412A03EA0E0343EA8A0343EA57
:102A4000052343EA090343EA4403C8F80032B0E728
:102A5000C2F80C35D4E7C2F86035B3F1FF3F046823
:102A6000A7D0C4F30044002CBBD05C091AD10124C8
:102A7000DFF8488004FA03F9C8F80890A146C6E7D1
:102A8000C2F86435E9E7C2F86835E6E7C2F86C35A4
:102A9000E3E76FF0150065E76FF0850062E700235C
:102AA000DB60FFDE00239B60FBE7002308F180086A
:102AB00053F82830F5E700BF2E7900000025845038
:102AC000F0F8FCFF2DE9F04104460D46076904F0DB
:102AD000CDF84FF0200890B92A4B1B787BB16426C3
:102AE000606803F063FED0B9012003F0B0FF013E3F
:102AF000F6D1F4E786F31188BFF36F8FEFE7EFF3BA
:102B00001186314688F31288BFF36F8F606803F037
:102B10004DFE80B986F31188BFF36F8FEFE7EFF3B7
:102B20001186314688F31288BFF36F8F606803F017
:102B30003DFE0028DED03B691D706268386913686D
:102B4000C3F844050120C3F848050020C3F820015C
:102B5000D3F82051C3F858015268D3F85801D2066F
:102B600008D5082062681268C2F800054FF4800298
:102B7000C3F8042301229A6081F31188BFF36F8F99
:102B8000BDE8F081F10F00202DE9F7434FF0000878
:102B9000476805693C680646C4F800852860D7F890
:102BA0000C904146484601AA03F0D2FD00283CDBC8
:102BB000019BD9F8002019791868FFF7C5FE002895
:102BC00033DB6B7A3169012B03D0032B2BD14FF010
:102BD0001008AB7A032B26D195F80BC0BCF1000F7F
:102BE00002D0BCF1010F1ED12A7A12B1022A1AD1E9
:102BF0000E226B687068B3F5164F006800F0B28063
:102C000034D8B3F5165F00F0B0801AD8B3F5966FDC
:102C100000F0AD800CD8B3F5967F00F0AB80B3F533
:102C2000167F00F0AA806FF0850003B0BDE8F08346
:102C3000B3F5166F00F0A480B3F5965FF3D15C4B4B
:102C400043E0B3F5E14F00F09E8008D8B3F5615F33
:102C500000F09B80B3F5964FE5D1564B35E047F633
:102C6000122E7345DFD14FF400032EE0B3F5613F20
:102C700000F08D8015D8B3F5963F00F08B800AD810
:102C80004DF6C02E734500F08780B3F5614FCAD171
:102C90004FF46B0319E0B3F5E13FC4D14FF0EB7390
:102CA00013E0B3F5612F7AD009D8DFF820E173453E
:102CB00078D0B3F5E12FB6D14FF0E86305E0DFF847
:102CC00010E17345AFD14FF08053C0F824357368DD
:102CD00048EA0C081B6842EA0802C3F86C250B1D81
:102CE000D5E9010183E803007B68990712D505F156
:102CF000180000F0B7FD304B984256D1287E04F101
:102D00000C0204F5907103F0A4FE01202B7E984084
:102D100000F0F4FC0823C4F800353B7A53B9C4F83A
:102D20001031D4F810316B69C4F834350123C4F87C
:102D3000383523607B6800209A075CBF4FF48073AE
:102D4000C4F804337B68DB0644BF4FF48003C4F847
:102D500004332B69C4F844350123C4F84805A36043
:102D6000E36062E74FF41D03AFE7144BADE74FF4A8
:102D70009E23AAE74FF4A033A7E74FF41C33A4E740
:102D80004FF41D23A1E70E4B9FE70E4B9DE74FF03D
:102D90006C739AE70C4B98E74FF4650395E74FF097
:102DA000706392E74FF080638FE76FF004003CE7B9
:102DB00000B0130000A04E000000AD0B0050270033
:102DC00000C0750000F03A0000903A0190D0030076
:102DD00040420F000123834070B5DC430B4AD2E828
:102DE000EF1F01EA0405C2E8E65F002EF7D14FF4B9
:102DF000803282400648C0F80823BFF35F8FBFF3DC
:102E00006F8F0B4214BF0120002070BDC00E002048
:102E10000050015070B40E4922F07F46D1E90034D1
:102E2000D01AC31844F10004C1E90034A6F5001318
:102E3000B3F5400F09D2074B1B681A0A1B069C19F1
:102E4000054B42F10005C3E9004570BC01F092B9A1
:102E500040010020C40E002048010020D9B1012308
:102E60000D4A8340D2E8EFCF4CEA030CC2E8E1CF31
:102E70000029F7D14FF48033084A8340C2F8043365
:102E8000074BD3E8AF3FC340DB0742BF4FF400120C
:102E9000044BC3F800217047C00E002000500150C1
:102EA000BC0E002000E100E00D4B1868010A00068E
:102EB000BFF35F8F0B4BD3F80435181841F10001B5
:102EC000B3F5801F0AD2084BD3E90023904271EB7F
:102ED000030303D210F1807041F10001704700BF7D
:102EE000C40E002000500150480100202DE9F04F91
:102EF00085B016461F4604469DF840A0FFF76AFFBE
:102F00000190FFF7D1FFB04271EB070352D23B4B68
:102F1000301A67EB0101984271F100014DD2384B34
:102F200003EB0413D3E902239F4208BF964258D013
:102F30004FF48038334908FA04F8204626F07F4BD6
:102F4000C1F8488303F097FC4FF00309584604F199
:102F50005005AD00ADB205F1502504F5A87305F597
:102F600080350293029A20F07F4341F82230C1F865
:102F70004483D1F80435244AC01A033820F07F4036
:102F800090422ED9286868B1D1F80435A3EB0B0024
:102F900020F07F40B0F5000F039322D9204603F0C4
:102FA0006AFC039BBAF1000F07D109EB030009F19A
:102FB0000109D7E7BAF1000F09D06FF015052046D7
:102FC0000199FFF74BFF284605B0BDE8F08F0123BC
:102FD0000E4AA340D2E8EF0F1843C2E8E10F0029E0
:102FE000F8D107490E982301C8500F9B01EB04123A
:102FF0000025C2E902675360E1E700BF01008000DD
:103000003001002000500150FDFF7F00BC0E002069
:103010007FB500254FF0FF304FF0FF31194C1A4BB0
:103020000226C4F80833C4F84833184BC4F80855CE
:10303000C3E902014FF480334FF40012C4F80433A3
:10304000134B0121C4F804631520C3F880212A46DC
:10305000FFF78AF81520FFF757F801230D4AA36000
:10306000236013600C4B0D4A009328460023CDE9E2
:103070000155FFF73BFF3046FFF70CFA284604B036
:1030800070BD00BF0050015003000F003001002050
:1030900000E100E0C00E0020152E0000FFFF7F00C1
:1030A0002DE9F7432E4BD3F8042390070BD5D3F823
:1030B000042142B10022C3F804212A4AD3F8043182
:1030C000136801331360264AD2F80433D90326D596
:1030D000254BD3E8EF1F21F00100C3E8E40F002CDB
:1030E000F7D1CB0702D4D2F84031C3B100251C4C34
:1030F000C4F84051D4F84031FFF7D6FEEFF3118207
:10310000202383F31288BFF36F8F184BD3E9026734
:10311000B042B94106D282F31188BFF36F8F03B07A
:10312000BDE8F0834FF0FF38D3E900104FF0FF39CE
:103130001D60C3E902894FF48033C4F84833C4F8F2
:103140004051D4F8403182F31188BFF36F8F0029CA
:10315000E5D0009032463B4628468847DFE700BF6F
:1031600000500150C40E0020BC0E00203001002091
:1031700030B5431C124C85B005D08442A8BF04462C
:10318000012CB8BF0124FFF78FFE0E4B0C4DD3E985
:103190000013401AB0F5000F0FD22218AA4228BF20
:1031A0002A46002052180849CDE90100009143F158
:1031B0000003FFF79BFE05B030BD2A46F1E700BFD4
:1031C000FFFF7F0040010020152E000008B5FFF72B
:1031D0006BFE024B1B68C01A08BD00BF40010020F7
:1031E000012310B5074C15206360FEF79BFF4FF4D9
:1031F0000012054BC4F80833C4F84833034BC3F836
:10320000802110BD0050015003000F0000E100E0DC
:1032100040EA0103C3F30E0330B58BB940F2151534
:10322000094CC90BC0F3C730994201D1002030BD11
:10323000C218D2B202F5C07244F822500133F3E74B
:103240006FF01500F3E700BF0030005030B5816823
:1032500085B0103921F00704054603F076F81022F6
:103260000146684603F0F2F810226846064903F06A
:10327000E2F810236A462146284603F034F8003865
:1032800018BF012005B030BD5073000030B50D46A9
:10329000816887B0102302AA1039044603F00EF8A3
:1032A000002802DA012007B030BD1022204602A912
:1032B00003F00CFB00283AD110221E4902A803F0AB
:1032C000AAF800280CBF012302232B70204603F02C
:1032D000E9FA012301460DF10702204602F0EEFF54
:1032E0000028DFDB9DF80730204603F00F021B09A2
:1032F0006A702B7101220DF1070103F0E7FA10B992
:103300006B78042B03D901236B7000232B71A26807
:103310002046183A22F00702083AA91C03F0E9FAFD
:103320000028BFD12046E91C03F03CFBBBE7032388
:10333000CBE700BF50730000F0B5354F85B04600B5
:103340000546694657F8260003F032FB044610B1E3
:10335000FF2005B0F0BD013657F8260002A903F0A2
:1033600027FB012837D12A4649212A4802F098FF35
:10337000294B8DF80C40029300229DF800609DF8C7
:103380000870264C3146207803F092FA50B3394643
:10339000607803F08DFA28B3A378042B03D09DF84E
:1033A000031099421ED1E378042B03D09DF80B1033
:1033B000994217D12379042B10D16279022A1DD1A9
:1033C000174B18482A46492102F06AFF6079831E8C
:1033D000022BBED9BCE70028CED0B9E79DF8021079
:1033E0009942EAD00132032A04F10604CAD10E48F8
:1033F0002A46492102F054FF0120AAE7032A05D0FA
:103400000A4B0B49042A08BF0B46DAE7094BD8E7F9
:10341000A07100006D79000003010303027A00002F
:103420004F790000B8790000DC7900005479000081
:10343000667900004A79000008B5EFF31083012B8C
:103440000C4A07D1126ABFF34F8F511C4A424A41BE
:10345000104608BD03F0D9FA00B172B6126ABFF384
:103460004F8F531C5A425A4103F0CFFA0028EFD035
:1034700062B6EDE70080FF0008B5EFF31083012B83
:103480000B4A06D1D269BFF34F8F02F001021046FA
:1034900008BD03F0BAFA00B172B6D269BFF34F8F1C
:1034A00002F0010203F0B1FA0028F0D062B6EEE7B4
:1034B0000080FF0010B503F0A8FA30B14FF05023A0
:1034C0000022C3F81421C3F8182103F0ADFA28B183
:1034D0000122644BC3F8382AC3F878254FF47F02E1
:1034E000D2F83031D2F83421BFF34F8FC3F30B033E
:1034F000092B05D1012A1EBF01225A4BC3F878259A
:1035000003F092FA18B10E22574BC3F8E42E03F0E1
:103510007CFA30B10022534BC3F80C270122C3F8C8
:1035200010270022D30003F57F03D3F80013BFF365
:103530004F8F013108D0D3F800130132D3F8043390
:10354000B2F5807F0B60EDD1EFF31084FFF794FFAD
:1035500000284DD0BFF34F8F444BD3F80024012AED
:10356000FBD1C3F80425D3F80024012AFBD1012C98
:1035700003D003F04AFA00B172B6FFF77DFF58B1ED
:103580003B4AD36923F00103D361BFF34F8F374A1E
:10359000D2F80034012BFBD1FFF74EFF68B1344A5B
:1035A000136A23F0FF0343F020031362BFF34F8F2E
:1035B0002E4AD2F80034012BFBD1012C03D003F0AA
:1035C00024FA00B162B60022284BC3F80425D3F8D0
:1035D0000024012AFBD1BFF34F8F2649264BCA682E
:1035E00002F4E0621343CB60BFF34F8F00BFFDE7EF
:1035F000FFF722FF0028ADD11E4AD2F88C3043F4E9
:103600004063C2F88C304FF47F03D3F83021D3F8F5
:103610003431BFF34F8FC2F30B02092A16D1013B9D
:10362000022B02D8154AD35C83B1114814490368B0
:103630000E4A8B420CBF5A230023C2F8103EC36AC5
:103640008B420CBF5A230023C2F8003E094AD2F82D
:10365000883043F47003C2F88830BFF34F8FBFF354
:103660006F8F10BD0040005000A003500090035029
:103670000080FF0000ED00E00400FA05147A00006D
:10368000FA50FA5030B50468ACB1B4FA84F30122B0
:10369000C3F11F03DBB29A4024EA0202D0E8EF5FD5
:1036A000A54204D1C0E8EC2FBCF1000FF6D1EAD15D
:1036B00002480B7030BD0248FCE700BF0000AD0BB4
:1036C0000200AD0B10B50368CB40DB0710D401231B
:1036D0008B40026843EA0201D0E8EF4F944204D1E4
:1036E000C0E8EC1FBCF1000FF6D1F2D1014810BDCB
:1036F0000148FCE70000AD0B0400AD0B014BC3F823
:103700000405704700700150044B1A7922B9012258
:1037100018601A710248704702487047C80E0020AE
:103720000000AD0B0C00AD0B08B5084B1B6833B1A6
:103730000520FEF70BFD10B90520FEF7E5FC4FF064
:1037400050230122C3F8182508BD00BFC80E002071
:1037500010B510B1012847D010BD4FF05023D3F859
:103760001814D3F81824C90322D502F00303022B3E
:1037700005D0012B02D0002003F072F901234FF095
:1037800050220220C2F8183508224FF4827300211B
:1037900003F1502319601C68012402F150221460C7
:1037A000164A126822B34FF05023C3F80403D3E73C
:1037B000D3F81424D207E1D5D3F81C2402F0030275
:1037C000013A012AD7D80D4A12681AB10222C3F869
:1037D0000423C1E7D3F80421002AFBD00022C3F858
:1037E0000421D3F80431B7E700224FF48073CEE709
:1037F0001A68002AFCD019601B68ADE7C80E0020CB
:103800004FF0502310B5D3F8002152B10020C3F877
:103810000001D3F800210122C3F80823104B1B68D4
:1038200098474FF05023D3F8042182B10022C3F807
:103830000421D3F80421D3F81824D3F81824022142
:1038400002F00302012A03D1C3F818159A6010BDD3
:10385000C3F80813024B0120BDE810401B6818474D
:10386000C80E002001460148FFF70CBF540000209D
:10387000036803F01F025B090260024818BF0020C2
:10388000704700BF0025845070B50D4C00F108034F
:1038900034F813300546DA050E4607D5C3F3432343
:1038A00004EBC302526854F833309847A3682BB135
:1038B00031462846E268BDE87040184770BD00BF39
:1038C00058000020024611F0010004D003490B6AA1
:1038D00013600B6203B90020704700BF00258450BD
:1038E00010B4134AC0B2083032F81030D9051CD5D4
:1038F000C3F3432123F4F85322F81030002002F1DF
:103900000E0434F8023F13F4807F03D0C3F3432343
:1039100099420AD001302028F3D1002342F83130F7
:1039200004485DF8044BFFF7CDBE5DF8044B7047CB
:1039300058000020B0000020F0B505460020012608
:10394000044607468C420BD1114BD3F87C2132B18F
:103950000022C3F87C21D3F87C3140F00040F0BD58
:10396000E3B29B0003F580729B0806FA03F31D4245
:103970000BD002F1A04202F55042D2F800C0BCF1D7
:10398000000F02D01760126818430134DAE700BF55
:1039900000D00050CBB2024608460D49083331F83A
:1039A0001330990611D599070FD4012110685B0BCC
:1039B0009940C0F80813126802EB8303D3F810256E
:1039C00022F00302C3F810257047002103F0ECB881
:1039D00058000020F7B5194ECDB2083536F815302D
:1039E0000746DB070C4626D5FFF7D4FF36F815301F
:1039F0009A0608D55A0B3B6803EB82030022C3F8F2
:103A00001025C3F810252046FFF76AFF002301A800
:103A100026F815300194FFF72BFF019B00EB830084
:103A2000D0F80022064B134043F00203C0F80032E6
:103A3000044803B0F0BD0448FBE700BF5800002075
:103A4000F0F8FCFF0000AD0B0400AD0B2DE9FF41C9
:103A5000136807460C461646FBB1DFF84481CDB229
:103A6000083538F8152002F02202222A22D000223E
:103A70002046CDE900228DF80E208DF80F200DF1A3
:103A80000E010DF10F0203F046F838F8153023F05F
:103A9000020343F0010328F8153073684BB31A781A
:103AA0005868DFF8FCC0E3B208333CF813108D0708
:103AB00002D5B0B138481FE021F02001C904C90C7B
:103AC0002CF8131068B1032AF4D870683D68406878
:103AD00090F800E005EB8E058AB9C5F81025C5F809
:103AE00010253CF8131021F01C0141EA82022CF849
:103AF0001320B3682BBB294804B0BDE8F081D5F88A
:103B0000108541EA4E3128F00308C5F810853D685C
:103B100041F0200105EB8E05D5F810052CF81310A7
:103B200020F4473020F44070C5F810052002D5F885
:103B3000107500F4F85040EA02403843C5F810050B
:103B4000CFE72046D3E90067FFF7CAFE002ED2D0A8
:103B5000134DD5E90023964203D19F4201D10022A3
:103B600009E010480DF10F01FFF78CFD0B4B984257
:103B7000C2D19DF80F20E4B205EBC20308345F60A8
:103B800035F8143045F8326043EA422343F4807339
:103B900025F81430AFE700BF0400AD0B0000AD0BFB
:103BA00058000020B00000202DE9FF4107460C46D8
:103BB0001E4612B3DFF8D480CDB2083538F8153080
:103BC000980701D4990621D413F01C0F02D0537822
:103BD000012B1BD001238DF80F3000232046CDE9A7
:103BE00000230DF10F01931C013202F094FF38F80D
:103BF000153043F0030328F81530002E44D0234D30
:103C0000E1B2083135F81120930703D4204804B0FD
:103C1000BDE8F081002096F800E03B6822F0200229
:103C2000D20403EB8E03D20CC3F8100525F8112043
:103C3000C3F8100596F801C04FEA8E08BCF1000FDA
:103C400022D03868B6784044D0F810354FEA0C4C92
:103C500023F4981323F4F853C0F81035230203F427
:103C6000F8530CF4403C3605D0F8107543EA0C03C9
:103C700006F48016334342EA4E323B4342F02002C0
:103C8000C0F8103525F811200248C0E75800002080
:103C90000400AD0B0000AD0B014BC3E902127047ED
:103CA00058000020054BC9B2083133F8113099068D
:103CB00043BF5B0B02481370024870475800002056
:103CC0000000AD0B0400AD0B70B5154D064695F820
:103CD00060401CBB2146402205F1100002F0B6FBFB
:103CE000214630682E6D8E420ED10023C0F87C3103
:103CF000D0F87C3140F30730FEF706FA012309487B
:103D000085F86030AB6570BDCBB29B0003F5807267
:103D10007C2B04BF845083580131E4E70248F2E76A
:103D2000580000200000AD0B0C00AD0B034B93F8C6
:103D30006000003818BF0120704700BF5800002005
:103D40000148FFF7BFBC00BFAC0000200148FFF7EF
:103D500099BC00BFAC00002073B503680C46D3F8D3
:103D600004130029A4BF4FF00041C3F804131E49F7
:103D7000E3B2083331F8133099061AD513F002066E
:103D800017D15B0B05689C0004F580716E50695873
:103D900001682144D1F8104544F00104C1F81045F0
:103DA0002AB10122016802FA03F3C1F8043302B018
:103DB00070BDC3F38203042B11D0052B11D001A8D1
:103DC0000194FFF755FD019A0369D34003F0010305
:103DD000991C204602B0BDE8704002F0E5BE032108
:103DE000F7E70221F5E700BF580000202DE9F3476F
:103DF000534B544FD3F80403396DC0B240F0004028
:103E0000FFF79AFD051E18DA00236846F96D009346
:103E10004FF00108FFF756FD97F85C30DA0757D4EA
:103E2000396D4FF00040FFF787FD6846F96DFFF7E9
:103E300049FD0028F0D125F000450124002D66D170
:103E400002B0BDE8F08794FAA4F4B4FA84F4E00870
:103E500004F1080337F8139004F007021DF800304E
:103E600008FA02F223EA02030DF8003001A80194D7
:103E7000FFF7FEFC019B4FEA9901803350F8236065
:103E8000C9F3820A4B07D146C6F3014624D5204622
:103E90005146FFF7F9FC01A80194FFF7E9FC019BEB
:103EA000F6B2803350F82330C3F301439E4207D16A
:103EB0000021204602F078FE3146204602F074FED2
:103EC00001A80194FFF7D4FC019B08FA03F30362F5
:103ED000009C002CB7D1A3E7022E0CD10321204671
:103EE00002F062FE0AF00503012BE9D149462046A3
:103EF000FFF7CAFCE4E70221204602F055FEBAF1C2
:103F0000030FF3D0032EDBD1BAF1020FEDE795FAE0
:103F1000A5F3B3FA83F304FA03F29B0003F1A04381
:103F200003F55043D3F81005D3F81015C0F304205F
:103F3000C1F3014125EA0205FFF7A6FC7EE700BFB9
:103F400000D00050580000200022034BC3F8842505
:103F5000C3F80425704700BF00900350044AD2F80C
:103F60000834DB07FBD50160BFF35F8F704700BFEC
:103F70000090035008B5C0F30B0383B90222094B2C
:103F8000C3F88425C3F804254FF0FF320260D3F84C
:103F90000024D207FBD5FFF7D7FF034808BD03482D
:103FA000FCE700BF009003500000AD0B0A00AD0B12
:103FB000012208B5054BC3F88425C3F80425FFF793
:103FC000CDFFBDE80840FFF7BFBF00BF0090035022
:103FD00038B5094B53F82040013053F82050A54222
:103FE00000D838BD636823B1204602F023FE0834B0
:103FF000F5E723689847FAE7A8710000012208B5A1
:10400000084B03201A70FFF7E3FFFDF7BDFE042005
:10401000FFF7DEFFFCF7FEF9034A137B23F00103F1
:10402000137308BDF10F00205001002008B50348AC
:10403000034A0021121A02F015FE08BD30010020CB
:10404000F40F002008B50020FFF7C2FF164B03F560
:10405000006282F3088883F30A880025E023134C6A
:1040600084F82230E57725766576A57684F82050A9
:10407000636A43F4E023636284F82350FDF7CCFFC6
:10408000FEF7DAF84FF0FF33A362E36202F0ACFD13
:104090000120FFF79DFF0220FFF79AFF2B462A46DB
:1040A00029460348FEF7A4F8F80F002000ED00E0D1
:1040B000FD3F000008B50648064A0749121A02F0FB
:1040C000D3FDBDE80840054A0549064802F0CCBDCD
:1040D000000000202E010020187A000000000000DF
:1040E000187A000000000020034B1B680BB9FFF793
:1040F0006DB80020704700BFD00E002030B570B101
:104100000B4B5B6898420AD0036843B1D3E90421A2
:10411000D0E90445121941EB0501C3E90421D0E9B6
:10412000003213605A600023C0E9003330BD00BF85
:10413000BC00002010B50E4B1C689C4204D1FFF758
:10414000D3FF6FF0004010BDFFF7CEFF002CF8D07A
:10415000D4E904321B1A62EBE072B3F1004F72F142
:104160000001EEDA002AACBF18460020EBE700BFE2
:10417000BC0000202DE9F84FEFF31186202383F3D4
:104180001288BFF36F8FDFF8B4902A4D4FF0000A0A
:104190002860D9F800004FF0000B484508BF002008
:1041A000254C3746D4E9001E2B6880B3D0E904863D
:1041B0004FEAE37C43457CEB060206DAB8EB0302E8
:1041C00066EB0C06C0E9042621E018EB01014EEB7A
:1041D000E873C0E904ABC4E90013FFF78FFF87F36E
:1041E0001188BFF36F8F83689847EFF311872023FF
:1041F00083F31288BFF36F8F2B68D9F80000A3EB0D
:10420000080348453E462B60CBD1D4E9001E59181F
:104210004EEBE373C4E9001300242C60FFF78AFF20
:104220002146FEF7A5FF87F31188BFF36F8FBDE826
:10423000F88F00BFD00E0020D0010020BC0000206D
:1042400010B50A4C23681BB101232360002010BD68
:1042500000F046F80028F7D00138062803D8044BB0
:1042600053F8200010BD034810BD00BFD40E00203D
:10427000C0710000FE8FFFFFBFF34F8F0549064B53
:10428000CA6802F4E0621343CB60BFF34F8F00BFF4
:10429000FDE700BF00ED00E00400FA0530B44FF088
:1042A000FE320025074B084C08494968C3F8002432
:1042B000C3F80424C3F80824C3F80C24C4F8005538
:1042C00030BC08470010845000008450C400002017
:1042D000024BD0E90012C3E900127047C40000206D
:1042E00038B500F02FF820B1032400F063F8204621
:1042F00038BD00F031F898B900F0ACF898B90F4D1E
:10430000D5F828391B0EF02B08D1D5F8242A0C4BF0
:104310009A420AD0072400F017F8E6E70624FAE7E5
:104320000424204638BD0024F5E7012000F092F86F
:1043300004460028F7D1C5F80C0AD8E700108450CD
:104340000000E0200020704700207047014BC3F8B8
:10435000040A70470010845010B5114800F048F866
:1043600000B110BD0F4800F043F80028F9D10E4C01
:10437000204600F03DF80028F3D10C4B0C481C609F
:1043800000F036F801460028EBD100F02DF8044685
:1043900008B1204610BD00F03FF82046FAE700BF04
:1043A000DC000020D8000020D4000020CC00002039
:1043B000D000002008B5084800F024F8074800F0B5
:1043C00021F8074800F01EF8064800F01BF8BDE889
:1043D000084000F00BB800BFDC000020D80000202F
:1043E000D4000020D000002000207047704700BF9C
:1043F00008B5034B02681B6810689847002008BD89
:10440000F400002008B5034B02685B681068984709
:10441000002008BDF400002070B5094C094D20694A
:10442000AB68984718B1084B08485B68984700216B
:10443000074AEB6811602069BDE87040184700BF6B
:10444000E0000020F4000020C4000020DC71000027
:10445000D80E0020F8B51A4D1A4E0446B2682869E5
:104460009047E8B9184F3B684CB1A3B1012B19D064
:10447000013B3B602869F36898470020F8BD43B9C9
:104480000121124AC2F800151149D1F81029002A59
:10449000FBD101333B60F368286998470020F8BDE1
:1044A0000C48F8BD0A4AD2F81039002BFBD1074A54
:1044B0006FF07E40C2F80035FFF748FF3B68D7E752
:1044C000E0000020F4000020D80E002000008450FE
:1044D00000108450E98FFFFF10B5044650B16368A7
:1044E00013F0685F05D0064A934202D00023626051
:1044F000236010BD034B04485B689847EFE700BF9B
:104500002C5F5CA9C4000020FC710000C8B14368A6
:104510000D4A934213D013F0685F0ED0012350E888
:10452000002F194640E8001C9CF0000FF7D1012A2B
:10453000F5D0BFF35F8F00207047044870470448F0
:1045400070476FF4E04070472C5F5CA9E98FFFFF74
:10455000EA8FFFFF034680B1426809498A420AD0C8
:1045600012F0685F05D0BFF35F8F002210461A601B
:10457000704704487047044870476FF4E040704744
:104580002C5F5CA9E98FFFFFEA8FFFFF10B504469F
:1045900020B10023034A2360626010BD0248FFF788
:1045A0007DFEF6E73A00003A2472000030B102685E
:1045B000034B04489A4208BF0020704702487047E6
:1045C000DD55AABB8208F0007108F00038B50D4631
:1045D0000446B0B1A0220021043002F066FB95B180
:1045E0000822294604F1640002F065FB082205F167
:1045F000200104F1840002F05EFB0020034B2360E5
:1046000038BD0348FCE70348FAE700BFDD55AABB05
:104610007108F0008308F0002DE9F74305460E46C7
:1046200099461146FFF7C2FF0446002840F08480F7
:10463000002E00F08580002900F08480B9F1200F61
:1046400040F0828005F14404082205F10408204668
:1046500002F031FB05F1240708223146404602F002
:104660002AFB06F120010822384602F024FB02A9A9
:1046700041F8049D4FF4807002F011FB002865D1D1
:104680004FF48073324A0121136093600823314A4A
:1046900000F034FB0121052308462F4A00F02EFBD1
:1046A0000823424601211C2000F028FB08233A463B
:1046B0000121032000F022FB2246082301210220D1
:1046C00000F01CFB0823254A01211A2000F016FBEC
:1046D0000523234A01211B2000F010FB0823214A57
:1046E0000121142000F00AFB08231F4A0121152094
:1046F00000F004FB082305F164020121162000F0FC
:10470000FDFA082305F184020121172000F0F6FAD2
:104710000823164A01210B2000F0F0FA00F04AFBB2
:104720000446019800F0D8FA114B002C18BF1C4623
:10473000A421284602F0BBFA204603B0BDE8F0836E
:104740000C4CF9E70C4CF7E70C4CF5E7084CEFE79D
:1047500090108450887200000073000048720000BE
:10476000EC720000AC720000CC72000068720000B5
:104770008408F0007608F0008008F0008108F0005E
:10478000C2690C4B1A60826943F8042C426943F8F1
:10479000082C026943F80C2CC26843F8102C82687C
:1047A00043F8142C426843F8182C026843F81C2C78
:1047B000704700BF5C1684500C4B1B68C3610C4BE8
:1047C0001B6883610B4B1B6843610B4B1B680361C8
:1047D0000A4B1B68C3600A4B1B688360094B1B684C
:1047E0004360094B1B680360704700BF5C16845030
:1047F0005816845054168450501684504C168450C9
:1048000048168450441684504016845030B10268D3
:10481000034B04489A4208BF002070470248704783
:10482000DD55AABB0202F0000002F00038B50446D4
:1048300068B1051D7021284602F039FA2846202269
:10484000044902F030FA0020034B236038BD0348CE
:10485000FCE700BF14730000DD55AABB0002F000A6
:104860002DE9F04385B015466F46274B04460E46AA
:104870000FCB87E80F002DB94FF00009484605B06F
:10488000BDE8F0832046FFF7C1FF81460028F5D13F
:10489000231D0193636AA3BB236F8BB1C3F140084F
:1048A000A84528BFA84604F13000314618444246C6
:1048B00002F0F9F9236F464443442367A5EB08054A
:1048C000226F402A06D104F13001384600F0B4FBD3
:1048D0000023236705F03F0835F03F0505D031463A
:1048E0002A46384600F0A8FB2E44B8F1000FC3D08A
:1048F0004246314604F1300002F0D5F9C4F8708028
:10490000BCE7DFF80890B9E7A06F00000C02F000E8
:104910002DE9FF4104466F46134B0E460FCB87E847
:104920000F002046FFF772FF8046B0B9CEB1636A30
:10493000251D01953BB90123226F636204F130010B
:10494000384600F079FB2B46043E243453F8042B00
:1049500012BAA34246F8042FF8D1404604B0BDE88D
:10496000F081DFF80880F8E7A06F00000502F00092
:10497000084B1B681B0EF02B08D1074B1A68074B1E
:104980009A4205D10020064B1860704705207047F9
:104990000620704728198450241A84500000E02013
:1049A0000C1A8450002230B5134640F6FC754900BD
:1049B000023802F1A15404F5823490424FEA840493
:1049C00002F10102CABF236025605B181E2AF0D1E4
:1049D000034A13600B445360024B034A1A6030BD14
:1049E000781084508410845020F80F001E4B30B58E
:1049F0001A4685B0196800910099CC07FAD500F1E4
:104A0000A15000F582308000016813680193019B7A
:104A1000D807FAD5154B164C186820231F3090FB89
:104A2000F3F0144D0138002810DA00230130400162
:104A300053B14FF00042A0F12001134204D10138DC
:104A400088424FEA5202F8D105B030BD1368039393
:104A5000039BDB07FAD5431823602B680293029B64
:104A6000002BE3D10138DEE7B4108450AC10845041
:104A7000E4108450DC108450F0B51D6885B001F05E
:104A80001F040DB91F2C28D1174D2E462F680197F2
:104A9000019FFF07FAD500F1A15000F58230800098
:104AA000006835680395039DED07FAD51F2C00EBD0
:104AB000611018BFC9430D4D18BF01F01F012860D8
:104AC0000B480068029002981CBF00FA01F11160C7
:104AD0004FF0000108BF1060196010684300C00F5C
:104AE000136005B0F0BD00BFB4108450E4108450D2
:104AF000DC1084500C4B890118603F3020F03F00DF
:104B00004030586099600948D960196159619961CC
:104B10001C3382B0196002680192019AD207FAD55B
:104B2000196002B0704700BF90108450B4108450D8
:104B300038B5A0F12003B3F5426F05462CD88F2875
:104B400026D800F1470300F16604DB064FEA54144F
:104B500000D0013464013F34A409013411B1A142F1
:104B60001AD30C464FF48050E300B0FBF3F020283A
:104B700028BF202002B110600122084B21461A6094
:104B8000FFF710FF28462146FFF7B4FF002038BD8D
:104B900000F11F046409DDE70148F8E71C188450A0
:104BA0002221F000464BF0B51D4689B01C680194E7
:104BB000019CE407FAD5434B002413449B001A6878
:104BC0000B181E2B88BFC0F11E011F320B18520993
:104BD0005343B3F5806F84BF4FF48061B1FBF2F1B2
:104BE000274688BF091ADFF8E4E000F1A150DFF89A
:104BF000E0C000F58230A14233DC2B680493049BB3
:104C0000DB07FAD5304B1B68296805910599CF075A
:104C1000FAD52E4C2E49236000231E46934203F101
:104C2000010040D11946002620F0010228488A429E
:104C30003CD8296806910699CE07FAD52549096816
:104C4000286807900798C007FAD5216000210C4614
:104C50001F488B422DD100201D499A422CD809B003
:104C6000F0BD2B680293029BDB07FAD503199B006A
:104C70001B682E680396039EF607FAD5CEF800301F
:104C80000023934203F1010306D1164623F00103EA
:104C9000B34204D80134AEE7CCF80070F1E7CCF8A9
:104CA00000700136F4E70E600346B7E70660013195
:104CB000BDE704600131CCE708600133CDE700BFF8
:104CC000B4108450240421147C108450D4108450D7
:104CD000D81084507810845008B540B1202801467F
:104CE0004FF0070228BF20210020FFF75BFF0022C2
:104CF000014B1A6008BD00BF1C188450F0B5294D47
:104D000085B02C462E680096009EF607FAD500F175
:104D1000A15000F58230800005682068019001985C
:104D2000C707FAD52048214F056002EB8306B2423F
:104D300029D100275A1C1D4E22F001029A4227D881
:104D400023680293029BDE07FAD5194B0B449B00A4
:104D50001B681F335B099A4213D2216803910399A0
:104D6000C907FAD500211544056008469B1A0F4A69
:104D70008B4210D800205A1C0C4922F001029A42A2
:104D80000CD805B0F0BD52F804CBC7F800C0CEE790
:104D900037600133D2E710600131E9E70860013381
:104DA000EDE700BFB4108450D4108450D810845064
:104DB000240421142DE9F041814BA0B01D689868AE
:104DC00020331E461A680192019AD707FAD57D4B07
:104DD0007D4A1A6032680292029AD407FAD57B4A59
:104DE0001A607B4A1446116803910399C907FAD5E2
:104DF000784A1168C1F3402137680497049FFF0780
:104E0000FAD5754F1F6027680597059FFF07FAD5EC
:104E10001768002900F0CF80B90540F1CC803168D7
:104E200006910699CF07FAD56C4919602168079158
:104E30000799C907FAD51168C1F340213768089767
:104E4000089FFF07FAD5664F1F6027680997099FDB
:104E5000FF07FAD51268002900F0AF80910540F1F4
:104E6000AC8032680A920A9AD207FAD5564A1A607A
:104E700032680B920B9AD707FAD55A4A1A603168F2
:104E80000C910C99CC07FAD55749196031680D91EE
:104E90000D99C907FAD55549196031680E910E99D7
:104EA000CF07FAD55249196031680F910F99CC0795
:104EB000FAD550491960504B1E4619681091109947
:104EC000C907FAD53F4C4D4B236033681193119BB2
:104ED000DB07FAD54A4B236033681293129BDF0736
:104EE000FAD5484B23603A4B9846196813911399A9
:104EF000C907FAD5324F386033681493149BDB0727
:104F0000FAD5226033681593159BD807FAD53E4B26
:104F1000236033681693169BD907FAD53B4B236061
:104F200033681793179BDA07FAD5394B2360336838
:104F30001893189BDB07FAD5364B23603368199317
:104F4000199BD807FAD5344B236033681A931A9B00
:104F5000D907FAD5314B236033681B931B9BDA07C3
:104F6000FAD52F4B236000F01DFC08BBD8F80030A9
:104F70001C931C9BDB07F9D53D6033681D931D9B7B
:104F8000D907FAD5274B236033681E931E9BDA0797
:104F9000FAD5254B2360D8F800301F931F9BDB0701
:104FA000F9D50C4B1B6813F4805F204B08BF1846E3
:104FB00020B0BDE8F0811E48FAE71E48F8E700BFC0
:104FC000901084508010845000100251C01F72292C
:104FD000B410845088108450C0CF0129C01F0E29FE
:104FE000C03F002940010249003184A80000164951
:104FF000400108A180440888B0108450C0447088E3
:1050000080077A41C0077E4100006A498006164940
:1050100040006E49000200210082202140822021B0
:105020008082242140A161A100C861510308F100E0
:105030000108F1000208F100324B2DE9F74F8046DC
:105040009246994644681A68002AFCD12E4B9B462A
:105050001A68002AFCD14FF0FF30019100F094FC57
:10506000802000F097FC01230720284A284DA2F554
:105070009E722B60C2F83C011360636A254F264E76
:105080003B60A36A20463360D8F8003042F8043C05
:10509000D8F8083098470199D9F80030002BFBD197
:1050A000BAF1000F20D104221C4B1A60D9F800304D
:1050B000002BFBD1DBF800A0BAF1000FFAD1D8F831
:1050C0000C30204698473B6863623368A362144BF8
:1050D000C3F800A0C3F844A1D9F80030002BFBD1DD
:1050E0002B6003B0BDE8F08F236A4020012B04BF82
:1050F0000B4A13600B4B1960C3F804A000F050FC7E
:10510000D4E700BF10198450201C8450001984502B
:1051100018188450CC178450D0178450C817845066
:1051200084168450281C8450544B10B5194698B0EE
:105130001A680192019AD207FAD5514B514A1A6066
:105140000A680292029AD407FAD54F4A1A600A688E
:105150000392039AD007FAD54C4818600A68049263
:10516000049AD207FAD54A4A1A600A680592059A43
:10517000D407FAD5474A1A600A680692069AD207F7
:10518000FAD5454A1A600A680792079AD407FAD5F1
:10519000424A1A600A680892089AD207FAD5404A29
:1051A0001A600A680992099AD407FAD53D4A1A602A
:1051B0000A680A920A9AD207FAD53B4A1A600A6824
:1051C0000B920B9AD407FAD5384A1A600A680C92E7
:1051D0000C9AD207FAD5364A1A600A680D920D9ACF
:1051E000D407FAD5334A1A600A680E920E9AD2078B
:1051F000FAD5314A1A600A680F920F9AD407FAD585
:105200002E4A1A600A681092109AD207FAD52C4AD0
:105210001A601A4B19461C681194119CE407FAD5C0
:10522000174B1860086812901298C407FAD51A60D4
:105230000A681392139AD007FAD5124A1A600A68BC
:105240001492149AD207FAD51E4A1A600A68159267
:10525000159AD407FAD51C4A1A600A681692169A4B
:10526000D007FAD5194A1A600A681792179AD20716
:10527000FAD5174A1A6018B010BD00BFB01084509C
:105280008010845000936521000431904096659011
:105290000083612100C3302100C3649000816190CC
:1052A00000461021008111210041442100C3202922
:1052B0000C4610C80086312100C3602140C1282956
:1052C000409665210013319040962529594614C80F
:1052D00040043249494B10B5194694B01A680092FF
:1052E000009AD207FAD5464B464A1A600A680192DC
:1052F000019AD407FAD5444A1A600A680292029ABF
:10530000D007FAD5414818600A680392039AD20779
:10531000FAD53F4A1A600A680492049AD407FAD56B
:105320003C4A1A600A680592059AD207FAD53A4AA9
:105330001A600A680692069AD407FAD5374A1A60A4
:105340000A680792079AD207FAD5354A1A600A689E
:105350000892089AD407FAD5324A1A600A68099264
:10536000099AD207FAD5304A1A600A680A920A9A4C
:10537000D407FAD52D4A1A600A680B920B9AD20705
:10538000FAD52B4A1A600A680C920C9AD407FAD5FF
:10539000284A1A600A680D920D9AD207FAD5264A51
:1053A0001A600A680E920E9AD407FAD5234A1A6038
:1053B0000A680F920F9AD207FAD5214A1A600F4B4A
:1053C00019461C681094109CE407FAD50C4B186021
:1053D000086811901198C407FAD51A600A681292E9
:1053E000129AD007FAD5174A1A600A681392139ACC
:1053F000D207FAD5144A1A6014B010BDB010845008
:10540000801084508090652100040990409665903A
:10541000808061218020082180206490008161903B
:1054200000461021008111210041442180202029C3
:10543000024610C8008609218020602140212829C9
:105440004096652140962529594614C8504B10B501
:105450001C4696B01A680192019AD207FAD54D4BB4
:105460004D4A1A6022680292029AD207FAD54B4A34
:105470001A604B4A42EA804022680392039AD2079C
:10548000FAD5186022680492049AD007FAD5454AE2
:105490001A60A2F5800242EA814122680592059ACB
:1054A000D207FAD5196022680692069AD007FAD573
:1054B0003D4A1A6022680792079AD107FAD53B4AFB
:1054C0001A6022680892089AD207FAD5384A1A60F8
:1054D00022680992099AD007FAD5364A1A602268DA
:1054E0000A920A9AD107FAD5334A1A6022680B92B7
:1054F0000B9AD207FAD5314A1A6022680C920C9A9C
:10550000D007FAD52E4A1A6022680D920D9AD1075B
:10551000FAD52C4A1A6022680E920E9AD207FAD552
:10552000294A1A6022680F920F9AD007FAD5274AA3
:105530001A60216810911099C907FAD51A60144BA6
:105540001A46196811911199C807FAD5114B2049CB
:105550001960116812911299C907FAD51D4919608D
:10556000116813911399CC07FAD50B49196011688A
:1055700014911499C807FAD5174919601168159143
:105580001599C907FAD5154A1A6016B010BD00BFA3
:10559000B010845080108450400441900086292926
:1055A000D81001C8401441904014212940146521AD
:1055B0000034409000310C90C0400C90C030202945
:1055C00040960D9000416090031645C80086112159
:1055D00000416021594644C84014459040142D9024
:1055E000264870B5054688B004680094009CE6071C
:1055F000FAD5234C23480460234C44EA83432C68A7
:105600000194019CE407FAD50360930143EA8242C6
:1056100042F0104444F4C0442B680293029BDE071E
:10562000FAD504602B680393039BDB07FAD5174B6D
:1056300003608B0143EA814141F0104343F4C043CE
:105640002E680496049EF607FAD503602B6805932E
:10565000059BDE07FAD5046041F058412B6806939C
:10566000069BDC07FAD5016042F058422B6807938D
:10567000079BDB07FAD5026008B070BDB0108450FC
:10568000C021022980108450807100988061189098
:10569000354B8EB019461A680092009AD207FAD597
:1056A000324B334A1A600A680192019AD007FAD540
:1056B000304A1A600A680292029AD207FAD52E4A34
:1056C0001A600A680392039AD007FAD52B4A1A6027
:1056D0000A680492049AD207FAD5294A1A600A681D
:1056E0000592059AD007FAD5264A1A600A680692EA
:1056F000069AD207FAD5244A1A600A680792079ACE
:10570000D007FAD5214A1A600A680892089AD20787
:10571000FAD51F4A1A600A680992099AD007FAD581
:105720001C4A1A600A680A920A9AD207FAD51A4ADB
:105730001A6008680B900B98C007FAD51A600A68BF
:105740000C920C9AD007FAD5144A1A600A680D9286
:105750000D9AD207FAD5124A0E211A6000200D23A5
:105760000F220EB0FFF73CBFB01084508010845061
:105770008043012940633921807001298020542110
:1057800000D13490C0403490C0302029C0530D90D7
:1057900000413890832308C880E31021004138215C
:1057A000CF4308C801232DE9F04192B0CDE903337E
:1057B000624B1D461A680592059AD207FAD5604BCE
:1057C000604C2360604B19461A680692069AD70708
:1057D000FAD55E4B1A68D60400F1A8802A680792B1
:1057E000079AD007FAD55A4A22600A680892089A9E
:1057F000D207FAD51E68C6F30036002E40F0988016
:105800001220FFF7F3F807461320FFF7EFF887425F
:105810008CBF12201320FFF7E9F8471EFFF738FF6F
:1058200003AB01AA39461220FFF726F904AB8046E4
:1058300002AA39461320FFF71FF900EB480002289F
:1058400032D003283ED0012874D12B680993099BDC
:10585000DB07FAD53F4B23602B680A930A9BD807D6
:10586000FAD53D4B23602B680F930F9BD907FAD5D0
:105870003A4B23602B681093109BDA07FAD5384B0C
:1058800023602B681193119BDB07FAD5354B2360FE
:10589000013F25D51023192218210020FFF7A0FE73
:1058A000304612B0BDE8F0812B680B930B9BD907F3
:1058B000FAD52D4B23602B680C930C9BDA07FAD595
:1058C0002A4BCFE72B680D930D9BDB07FAD5284BAE
:1058D00023602B680E930E9BD807FAD5254BC1E7A2
:1058E00003AB01AA39461220FFF7C6F804AB044601
:1058F00002AA39461320FFF7BFF810EB440402D187
:10590000FFF712FCC4E7FFF7E5FC022C08D0032CDC
:1059100009D0012C10D117211620FFF797FDB7E70A
:1059200015211420F9E70F210E20F6E7124EB7E7F4
:10593000124EB5E7124EB3E7124EB1E7B0108450E5
:1059400000084A5180108450B4108450881084504C
:1059500000084E5100065A4940065E490004424183
:105960000014424940042E49000652494006564957
:1059700000063A4940063E490608F1000708F100D2
:105980000408F1000508F100014B1860704700BFE2
:10599000081A8450014B1860704700BF041A8450E5
:1059A000034A13681842FCD0024A10601846704738
:1059B000001A8450081A845070470020704730B590
:1059C000836804468B42154685B00ED96368C0686B
:1059D000194401AA00F03FFE28B96268019B9B1A96
:1059E0002B60029B6B6005B030BD6FF02100FAE7C1
:1059F00070472DE9F7430E4617469946044628B9E5
:105A00004FF0FF38404603B0BDE8F0830029F7D0DF
:105A1000002AF5D0CB680D8938461D440423294659
:105A20000DEB030200F04AFC80460028E8D146F660
:105A30000812BDF804107389914225D1BDF80610F3
:105A40009942DDD1042338460DEB0302294400F0CE
:105A500035FC0028D4D146F60713BDF804209A423D
:105A6000CED1C4E900679DF82830A4F80890A3724D
:105A70007389BDF806202B44E360738913442B44DB
:105A8000043563612561BDE7002BE4D0B8E72DE95B
:105A9000F3410E4617461D46044620B94FF0FF302D
:105AA00002B0BDE8F0810368002BF7D04368002BFB
:105AB000F4D04FF6FF78D4E904239A4216D2236833
:105AC0005B8923B1E368934204BF04332361042359
:105AD000216960680DEB030200F0F0FB0028DDD1C6
:105AE000A37A2BB1D4E903329A4201D30120D7E73C
:105AF0002389BDF80610434501F1040203D0BDF827
:105B000004C09C450BD115B1BDF804302B8023692E
:105B1000043333603980236913442361C0E7236968
:105B200013442361C7E748B103683BB143682BB115
:105B3000C068884294BF0020012070474FF0FF30BA
:105B4000704773B50C46064611460223204601AA4B
:105B500000F031FA0546E8B9019A1F2A0ED9A2F1E0
:105B60002001304620222368194400F064FC236899
:105B7000019A13442360284602B070BD0146C2F169
:105B80002002304600F062FC019A2168C2F1200038
:105B90003044EAE76FF00205EDE74FF4C073584375
:105BA0003030704710B5044600F0C8FB4FF4C072A7
:105BB000A368303B02FB103010BD70B50D460446A3
:105BC00000F070FE2A46A0F1080104232046BDE83B
:105BD000704000F073BB13B50446019100F062FE03
:105BE0000423A0F108010DEB0302204600F09DFE06
:105BF00002B010BDFFF7FEBFFFF7FCBFFFF7FABF13
:105C0000FFF7F8BFFFF7F6BFFFF7F4BFFFF7F2BFEC
:105C1000FFF7F0BFFFF7EEBF704770B513460E46B3
:105C20001546002102460446FBF7A0F950B92B4661
:105C30000121204604F12C02FBF798F910B1002E47
:105C400008BF002070BD73B5044600200D461646FF
:105C5000FAF76CFC6946C0B2FCF73EF830BB2C2367
:105C600003FB0544E368258900981D440423294665
:105C70000DEB030200F022FBC0B946F60813BDF895
:105C8000042064899A42009815D1BDF806309C42E0
:105C90000CD1042361190DEB030200F00FFB28B9AE
:105CA00046F60713BDF804209A4207D0009800F08A
:105CB00004FB02B070BD002CF2D0F7E7BDF806106F
:105CC000214429443160F1E737B580250446426A12
:105CD00001A903200195FCF727F858B9019B092079
:105CE000226DA36201A90195FCF71EF8054628B1B3
:105CF000092500E00125284603B030BD019B206A3C
:105D0000636500F01BFBE065F5E70123036003F129
:105D1000012343600023C0E9023370474379012B1C
:105D200007D10368012B04D10079431E5842584122
:105D30007047002070477FB506460D46032001A935
:105D4000FBF7CAFF38BB0198FFF72CFFF16D044643
:105D5000284600F0D1F80444019800F0EFFA064616
:105D6000019800F0F2FA082201460DEB020000F063
:105D70006DFB2B7921468DF808300198334602AA35
:105D800000F0B1FA041E019818BF012400F095FA42
:105D9000204604B070BD0124FAE700F0B9BA2DE93D
:105DA000F8430E46002107460846FAF7BFFB0446B3
:105DB00001210020FAF7BAFB33789C4221D09842A7
:105DC00021D101252C2303FB0575F86DAC6AFFF783
:105DD000E4FE4FF000080746013C6B6A304603EBD7
:105DE000C40253F83410D2F804901B684A46C91A0A
:105DF000C844FFF7D2FFB84504F1FF34EDD3BDE846
:105E0000F8830025DEE70120F9E737B515460C4693
:105E10000920694600F0CCFDE979012903D0002270
:105E2000204600F0D9FD9DF80330012B02D1204619
:105E300000F0B1FDA9682046FFF7CDFE2046FDF732
:105E400005FA002003B030BD73B50D460646FBF7DA
:105E500093F90446E86058B302282ED1032001A923
:105E6000FBF73AFF58BB2A4631460198FBF7E4F8A6
:105E70000446D0B9019800F015FD012301460DF14B
:105E80000302019800F01AFA0446A0B90122019811
:105E90000DF1030100F01AFD10B101238DF803305C
:105EA0009DF8033003F00F03EB71019800F005FA41
:105EB000204602B070BD0124F7E70724F8E701246B
:105EC000F6E738B5436A0446C06D5D68FFF765FEC6
:105ED00000230246A06A01382B449A4201D90138B6
:105EE000FAE738BD436A00205A68034613448B42E0
:105EF00000F10100FAD3704710B543790279012B04
:105F000006BF00230C46CB0102F1FF3201FB023336
:105F1000026818BF4C00013A04FB023010BD70B596
:105F20000368CD1A002D02DC6FF05F0070BD93F99D
:105F300000601C78002E0ADB5C1C04601B78136078
:105F40000368C91A13688B42EED80020EEE704F00C
:105F50007F04013C032C2BD8DFE804F0020A142153
:105F6000012DE1D05B781360036802330360E7E73B
:105F7000022DD9DDB3F801305BBA9BB21360036820
:105F80000333F3E7032DCFDD9C785D782402DB78C3
:105F900044EA05442343136003680433E6E7042D11
:105FA000C2DDD3F801301BBA136003680533DDE7A7
:105FB0006FF06300BAE770B404680E1B002E07DDB3
:105FC00026789E4208D10134046070BCFFF7A7BF59
:105FD0006FF05F0070BC70476FF06100FAE738B592
:105FE00003230446FFF7E7FF18B9136813B96FF0EE
:105FF000670038BD013B136023681A78002AF6D188
:1060000001332360F5E72DE9F34190461F4601AACD
:10601000302305460E46FFF7CEFF0446F0B92B6845
:10602000F61A002E34DD42461B78284642F8043B1F
:106030002E68019B1E4431460623FFF7BCFF044631
:1060400060B92B68D8F80420C8F808309918B14214
:10605000296007D10C213846FBF738FA204602B0F8
:10606000BDE8F0819B5C3A4642F8043B2B68314620
:10607000013328462B60FFF752FF60B92B687A681E
:10608000BB601344B34218BF6FF065042B60E5E7B3
:106090006FF05F04E2E70446E0E7F8B5B1F1005FB6
:1060A0000546144600AF10D26E46D31D23F00703F9
:1060B000ADEB030D684600F0BEF96946224628465E
:1060C000FEF7CEFBB546BD46F8BDFEF7C9FBFAE7C5
:1060D000002070470FB407B504A951F8040B0191D3
:1060E000FBF7B6FA03B05DF804EB04B07047038B1E
:1060F00013F0070305D10368002B0CBF0020032019
:106100007047022B05D1408BB0FA80F04009800027
:106110007047012B05D10368002B0CBF0020052020
:1061200070470020704710B50C4600B111B96FF0F0
:10613000150010BD081D00F094F80028F9D1A368DF
:10614000032BF6D9F3E72DE9F0410D460746194632
:10615000281D90461E4600F095F8044638B1334697
:10616000424629463846A446BDE8F0416047BDE8AE
:10617000F08110B4EFF31182202484F31288BFF36E
:106180006F8F41615DF8044B0121FBF797BC38B577
:106190000C46054658B151B10B6843B14B6833B159
:1061A0001C22002100F052F900202C6138BD6FF054
:1061B0001500FBE770B505460E46FFF7B4FF041E59
:1061C00014DBEFF31182202383F31288BFF36F8F68
:1061D0004FF6FF716B8B2C8B8B4204F0070407D1B9
:1061E00082F31188BFF36F8F6FF00A04204670BDF1
:1061F000022C0CD101336B8382F31188BFF36F8FB4
:106200000023224631462846FFF79DFFEEE7062C85
:1062100014D8DFE804F004131313041A0400002355
:1062200033606B683BB9C5E90066ACB9022128460A
:10623000FBF744FCDAE71E606E60F6E782F3118834
:10624000BFF36F8F6FF00404D0E782F31188BFF3C0
:106250006F8F6FF08504C9E782F31188BFF36F8FEA
:10626000C4E7034658B1426802F00302012A03D092
:10627000032A04D1026812B10020986070476FF0C1
:10628000150070474268034602F00302032A4FF0EC
:106290000002816014BF104600685A607047704762
:1062A0000FB407B504A951F8040B0191FBF7D0F91D
:1062B00003B05DF804EB04B070477047002930B4B8
:1062C000044618460BDBA5680844A84207D8E068D6
:1062D0006468214484682468A44630BC60476FF039
:1062E000150030BC7047002930B4044618460BDB5B
:1062F000A5680844A84207D8E06864682144846817
:106300006468A44630BC60476FF0150030BC70472D
:106310000029034610B410460BDB9C680844A042D9
:1063200007D8D8685B68194483685DF8044B9B689C
:1063300018476FF015005DF8044B704708B5C0684A
:106340008368DB689847006808BD08B5C068836843
:10635000DB689847007908BD70B54C680368A342B4
:1063600001D2012070BD8A682244934201D30020EB
:10637000F8E74E69D1E90325B54203D36FF00B036B
:106380008B61F4E71B1B42F835304368086902EB68
:10639000C00253600B6901330B61E2E7FEE770470F
:1063A000012801D1EFF3058300F035BC01460068F8
:1063B000FFF7F6BF08B5FBF7FFFCBDE8084000F0AB
:1063C00000B8704700210120FFF7EABF61B662B64E
:1063D00080F31188BFF36F8F7047EFF31180202394
:1063E00083F31288BFF36F8F704772B6002383F375
:1063F0001188BFF36F8FBFF34F8F20BF80F31188D9
:10640000BFF36F8F62B67047034600201A5C02B973
:1064100070470130FAE710B55AB10139841810F805
:10642000012B11F8013FA04201D09A42F7D0D01AB7
:1064300010BD1046FCE710B5431E0A44914200D13E
:1064400010BD11F8014B03F8014FF7E70346C9B23D
:106450000244934200D1704703F8011BF9E74FF063
:10646000FF3070470C220369C9B201FB0233186C7C
:1064700000F00700704770B5C9B20369EFF31185EA
:10648000202484F31288BFF36F8F0C2606FB01349F
:10649000246C14F0C00408D0A24206D085F3118801
:1064A000BFF36F8F4FF0FF3070BD012271430B447B
:1064B0001A6485F31188BFF36F8F43680B445B68E0
:1064C00098470020F0E78022FFF7D5BFF8B5069F78
:1064D0000469C9B2EFF31186202585F31288BFF352
:1064E0006F8F0C2569430C44256C05F0070CBCF13B
:1064F000010F0BD1276486F31188BFF36F8FC4E9B6
:106500000E2343685B5898470020F8BD05F0C0058E
:10651000AF4286F31188BFF36F8F0CBF6FF0770027
:106520004FF0FF30F1E713B580240094FFF7CEFF62
:1065300002B010BD6FF08500704710B41C240069D4
:10654000CBB203FB040000215DF8044B1047002090
:10655000FDF7FEB8002000F0DCBA38B505460C4661
:1065600000F035FB002D07DBA84205D9401B844213
:106570008CBF0020012038BD0020FCE770B50C4620
:10658000154600F027FB294606462046FFF7E5FFA3
:10659000B8B1B4FBF6F306FB134393B9B5FBF6F3BE
:1065A00006FB13536BB9AE4201D9002070BD00F059
:1065B00011FB06462046FDF7DDFCAD1B3444F9D146
:1065C000F3E76FF01500F1E770B50D461946284660
:1065D00016461C46FFF7C1FF38B124B122462946B2
:1065E0003046FFF728FF002070BD6FF01500FBE775
:1065F0002DE9F3411C460023904682682360A36086
:106600000D461369694601AA9847019B5A1E0192DB
:1066100023B96FF0150002B0BDE8F0810098A268C0
:1066200047682168676085B9A8EB02030668B34232
:1066300028BF334603FB07111A442160A260026899
:106640009A4206D808300090DFE76B1AB3FBF7F3E5
:10665000ECE70020DFE713460022FFF7C9BF2DE972
:10666000F0470024836886B0884691461B6902AAD9
:1066700001A99847A2462546029BAB4202D806B024
:10668000BDE8F0870026019F07EBC5077B680493F0
:106690003A680AEB0603B24202D89A460135EBE7A4
:1066A00049460394059303A8C0470028E7D0049BFC
:1066B00001361C44ECE7436800205B681B690B60F3
:1066C0007047436802EA01005B6821EA02019860B2
:1066D0000020D9607047436800205B68996070476C
:1066E000436800205B68D960704743685A68536804
:1066F00021EA03000B4090600020D360704710B582
:1067000003695868F8B1884219D19C680868A142A9
:10671000586000D19860002008602AB15A680A6069
:106720009A68596002B99960002010E0814206D150
:106730000868206098688142EDD19C60EBE70446D0
:1067400000680028F2D1002AE8D16FF0150010BDD2
:1067500030B543681360057A446804EBC504A3426E
:1067600002D36FF0010030BD5C798C4201D0083358
:10677000F0E70020F7E743681B68D3F88004C3F80C
:1067800080047047436802691B68D3F8100150B158
:106790000020526912780A70C3F81001D3F8102152
:1067A00001221A6070474FF0FF30704702680346BD
:1067B000D2F8580140B95B689B0706D4D2F8200193
:1067C000003818BF012070470120704742681368E5
:1067D000D3F80413C90517D5D3F82011A1B1EFF3ED
:1067E0001181202080F31288BFF36F8FD3F820012E
:1067F00030B10020C3F82001D3F820010120D86077
:1068000081F31188BFF36F8F5268D20614D5EFF36E
:106810001182202181F31288BFF36F8FD3F85811B2
:1068200011B10021C3F800154FF48001C3F808131B
:1068300082F31188BFF36F8F704710B504460022B2
:1068400001210920FBF790FC0920FBF75DFC2046A5
:10685000BDE81040FCF798B910B5044600220121AC
:106860000820FBF781FC0820FBF74EFC2046BDE822
:106870001040FCF789B9002200F150039B009BB245
:1068800003F1502303F580331A601B687047FDF74E
:10689000D7BC08B5FBF78AFAFFF781FDBDE80840D1
:1068A000FDF7CEBC8068183820F00700103870471C
:1068B000042809D0052803D1481E18BF01207047BD
:1068C000431A5842584170470120704738B5154661
:1068D0000C4661B15AB1FFF738FD2146254411F845
:1068E000013B834203D1A942F9D1012038BD0020E8
:1068F000FCE738B50C460123114622460546FFF752
:10690000DDFC00280FDB012221462846FFF7DEFFD1
:1069100038B92378012B14BF0223012300202370F0
:1069200038BD0323FAE70120FAE72DE9F7431D46B6
:1069300006460F469046FFF701FD6C1E0444404298
:106940000440082C1AD83046FFF7FFFC81462A463F
:1069500041466846FFF76FFD4946621B0DEB050097
:10696000FFF774FD23466A4639463046FFF7BBFC05
:10697000003818BF012003B0BDE8F0834FF0FF30AE
:10698000F9E707B501238DF8042001AAFFF7CDFF31
:1069900003B05DF804FB81680122183921F007017A
:1069A000FFF7EFBF8268183A22F00702FFF7A1BF96
:1069B00013B50C46C0B201A9FBF78EF950B92146B8
:1069C0000198FCF763FC04460198FFF776FC20462B
:1069D00002B010BD0124FAE713B541EA02110446E2
:1069E0008DF80710FFF75EFF012301460DF1070246
:1069F0002046FFF79AFF02B010BD816801221839C6
:106A000021F007010839FFF7BCBF4FF47F03D3F82B
:106A10003001D3F83431BFF34F8FC0F30B00A0F136
:106A200009035842584170474FF47F02D2F8303181
:106A3000D2F83401BFF34F8FC3F30B03092B03D1FB
:106A4000431E58425841704700207047004700F0ED
:106A5000C7B840F00040C1F88000C2F8800070471D
:106A6000F7B5044618B1012824D003B0F0BD4FF0AB
:106A700050230222C3F8082301220646DA60C3F835
:106A80000401D3F80431012342F210754FF050276E
:106A90008DF80730DCB1012CE7D1D7F80C3403F4C2
:106AA00080338EBB002BE0D00120FFF7D0FF013DEB
:106AB000F3D1DAE74FF050230022C3F808035860FF
:106AC000C3F80021D3F800310DF10706DBE7D7F852
:106AD000183403F480333EB9002BC6D00120FFF7F1
:106AE000B6FF013DF3D1C0E7D7F8182402F0030246
:106AF0003270002BB9D09DF807000128B5D1FFF7FF
:106B0000A6FF013DC6D1B0E7D7F80C2402F0010280
:106B1000EEE7FFF7A5BFF7B51646DDE90847019098
:106B200001A81D46FCF7A4FE019BB6F1000C18BF9E
:106B30004FF0010C00EB83000B1E18BF0123002D4A
:106B400043EA4C0314BF4FF00C0C4FF0000C002C28
:106B500043EA0C0314BF4FF4E06C4FF0000C002F1D
:106B600043EA0C0314BF4FF4403C4FF0000CD0F844
:106B7000002243EA0C0322EA030301B109780EB1B3
:106B80003678760019430DB12D78AD0031430CB144
:106B90002478240229430FB13F783F040C433C433F
:106BA000C0F8004203B0F0BD1FB50DF10F03019313
:106BB00000238DF80F101A4619460093FFF7ABFF1C
:106BC00005B05DF804FBFCF705BFFCF7E3BE4FF42E
:106BD000801070474FF4805070474FF480707047BA
:106BE00008B1FBF75BBB7047704740B1C36858788A
:106BF00010F001001EBF1878B0FA80F0400970470D
:106C0000EFF31183202383F31288BFF36F8FFEE726
:106C100008B5FFF7F5FF10B5EFF31184202383F3D8
:106C20001288BFF36F8FFFF7F3FF84F31188BFF370
:106C30006F8F10BD10B5D0E9003433B90020E26881
:106C4000537843F00103537010BD20469847002845
:106C5000F4D00028B8BF4042FF28A8BFFF20E36857
:106C60001870ECE7FFF7F2BBFFF7E5BBEFF3058029
:106C7000003818BF012070472DE9F041069F0446F7
:106C800015461E46FDF7A2FC38B93B46324629465A
:106C90002046BDE8F041FDF7BFBCBDE8F0810A46E3
:106CA0000021FDF745BFFFF7C6BBFFF7CFBB0A4684
:106CB0000021FFF7CBBB01EB820204388A4201D1ED
:106CC0000020704752F8043D1BBA40F8043FF5E736
:106CD000A894FF7F010000008D220000000000004A
:106CE00059230000286D0000512600003C6D000073
:106CF0008F6800000000000059680000646D00000B
:106D00003B680000506D0000852500000000000079
:106D10001130000000000000936800000000000037
:106D2000ED250000786D0000F4780000A0700000F0
:106D3000B870000024010020540E002022790000C9
:106D4000F07000000871000028010020B00E002043
:106D5000367900002C710000947100002A01002097
:106D60001C00002040790000607100009471000058
:106D70002C010020380000200B79000000000000EA
:106D8000D470000026010020000000000000000078
:106D9000C563000000000000C563000000000000A3
:106DA000C563000000000000C56300000000000093
:106DB000C5630000013800004D6A000000000000BB
:106DC000C563000000000000C5630000646D0000A2
:106DD000CD670000506D0000CD670000000000008E
:106DE000C563000000000000C56300000000000053
:106DF000C5630000ED3D00004D6A0000000000008A
:106E0000C563000000000000C56300000000000032
:106E1000C563000000000000C56300000000000022
:106E2000C563000000000000C56300000000000012
:106E3000C563000000000000A13000000000000059
:106E4000C563000000000000C563000000000000F2
:106E5000C563000000000000C563000000000000E2
:106E6000C563000000000000C563000000000000D2
:106E7000C563000000000000C563000000000000C2
:106E8000C563000000000000C563000000000000B2
:106E9000C563000000000000C563000000000000A2
:106EA000C563000000000000C56300000000000092
:106EB000C563000000000000C56300000000000082
:106EC000C563000000000000C56300000000000072
:106ED000C563000000000000C56300000000000062
:106EE000C563000000000000C56300000000000052
:106EF000C563000000000000C56300000000000042
:106F0000C563000000000000C56300000000000031
:106F1000C563000000000000C56300000000000021
:106F2000C563000000000000C56300000000000011
:106F3000C563000000000000C56300000000000001
:106F4000C563000000000000C563000000000000F1
:106F5000C563000000000000C563000000000000E1
:106F6000C563000000000000C563000000000000D1
:106F7000C563000000000000C563000000000000C1
:106F8000C563000000000000C563000000000000B1
:106F9000C56300003E74000003000000FFFFFFFF18
:106FA000020000000000000081470000B947000017
:106FB0000338FDD8704700000300000009000000FE
:106FC00001000000F5770000DC6F00000300000006
:106FD0000900000003000000090000005B00000041
:106FE00000800050009000500A00000000000000E7
:106FF0000000000000C00000786D000001000000EB
:1070000000C0000000400000786D00000200000099
:107010000000010000020000786D00000300000085
:107020000000010000800700786D000004000000EF
:107030000000010000800000786D000005000000E5
:1070400000020100007E0700786D000006000000CD
:1070500000020100007E0000786D000007000000C3
:107060000080010000000700786D000008000000AB
:107070000080010000000700786D0000090000009A
:107080000080080000800700786D0000000000000C
:107090009D630000E1220000B1220000000000001A
:1070A000FD23000025230000FF7800004F6500004D
:1070B000556500000579000035650000C7640000D3
:1070C000276500000000000065640000000000006B
:1070D00000000000C9650000052600007D65000075
:1070E000E5250000D525000004000000FF00000099
:1070F000FFFFFFFF0025845000000000000000009B
:1071000000D0005000000000D5260000B766000047
:10711000C3660000D7660000E1660000EB66000071
:1071200055280000FF66000000000000009000509D
:1071300002000000000000003C71000000900050C0
:1071400048710000010000005071000004000000C0
:107150001D000000100004001C06020011060600BD
:10716000008000500200000000000000707100006C
:10717000008000507C71000001000000847100005C
:10718000040000001B0000000E0004001A060200AC
:107190000F06060085670000C52A0000776700001B
:1071A0000300000009000000D86C0000D86C00004B
:1071B000106D0000186D0000286D0000286D0000A3
:1071C000FF8FFFFFFF8FFFFFFE8FFFFFFE8FFFFF91
:1071D000FD8FFFFFFC8FFFFFFC8FFFFF436F756C80
:1071E00064206E6F74206C6F636B20706F776572B4
:1071F0002073617665206D75746578006D757465B2
:10720000785F667265652063616C6C656420776980
:107210007468204E554C4C20706172616D657465C8
:107220007200000043616E277420696E69746961A1
:107230006C697A65206D757465782C207761732090
:107240004E554C4C0D0A0000FFFFFFFFFFFFFFFFF4
:10725000FFFFFFFF00000000000000000000000032
:1072600001000000FFFFFFFFFCFFFFFFFFFFFFFF2C
:10727000FFFFFFFF00000000000000000000000012
:1072800001000000FFFFFFFF512563FCC2CAB9F3F4
:10729000849E17A7ADFAE6BCFFFFFFFFFFFFFFFFCD
:1072A00000000000FFFFFFFF0000000096C298D81A
:1072B0004539A1F4A033EB2D817D0377F240A4631F
:1072C000E5E6BCF847422CE1F2D1176BF551BF3728
:1072D0006840B6CBCE5E316B5733CE2B169E0F7CFB
:1072E0004AEBE78E9B7F1AFEE242E34FFFFFFFFF70
:1072F0007F0000008000000000000000000000008F
:10730000FFFFFFFF7F000000800000000000000082
:107310000000000067E6096A85AE67BB72F36E3C49
:107320003AF54FA57F520E518C68059BABD9831F50
:1073300019CDE05B010002001000110020002100C7
:107340002200230024003000310032003300FFFF10
:1073500077C295F360D2EF7F3552500F2CB679800B
:1073600025633A205374617274696E6720626F6F8F
:10737000746C6F616465720A0025633A20556E6112
:10738000626C6520746F2066696E6420626F6F7432
:1073900061626C6520696D6167650A0025633A204A
:1073A000426F6F746C6F6164657220636861696EAF
:1073B0006C6F61642061646472657373206F6666CC
:1073C0007365743A20307825780A0025633A204A9C
:1073D000756D70696E6720746F20746865206669CA
:1073E00072737420696D61676520736C6F740A0035
:1073F00025633A2050726F74656374206D63756203
:107400006F6F7420666C617368206661696C656477
:107410002C2063616E63656C207374617274757087
:107420002E0A0025633A204E657665722073686FD8
:10743000756C642067657420686572650A006D6309
:1074400075626F6F740025633A20696E76616C69AE
:107450006420666C6173682049442025643B206584
:10746000787065637465642025640A002A8648CEB6
:107470003D030107002A8648CE3D02010025633AFC
:1074800020556E61626C6520746F2064657465724E
:107490006D696E6520666C61736820736563746FD7
:1074A00072206F662074686520696D61676520745D
:1074B0007261696C65720A007072696D617279003F
:1074C0007365636F6E646172790025633A20496D5C
:1074D00061676520696E2074686520257320736C70
:1074E0006F74206973206E6F742076616C696421FB
:1074F0000A0025633A202564207374617475732033
:107500007772697465206661696C73207065726654
:107510006F726D696E672074686520737761700A99
:107520000025633A204661696C656420746F206FA2
:1075300070656E20666C61736820617265612049B8
:10754000442025642028696D6167652025642073C7
:107550006C6F74202564293A2025642C2063616EA9
:107560006E6F7420636F6E74696E75650A002563B3
:107570003A204661696C65642072656164696E6772
:1075800020736563746F72733B20424F4F545F4D9D
:1075900041585F494D475F534543544F52533D2532
:1075A00064202D20746F6F20736D616C6C3F0A0036
:1075B00025633A204661696C65642072656164697F
:1075C0006E6720696D6167652068656164657273C7
:1075D0003B20496D6167653D25750A0025633A20AA
:1075E0004661696C65642072656164696E672062DA
:1075F0006F6F74207374617475733B20496D61679C
:10760000653D25750A0025633A2070616E69632126
:107610000A0025633A2044657465637465642069D3
:107620006E636F6E73697374656E742073746174C6
:107630007573210A0025633A2043616E6E6F7420D2
:10764000757067726164653A206E6F7420612063A3
:107650006F6D70617469626C6520616D6F756E74B9
:10766000206F6620736563746F72730A0025633A36
:107670002043616E6E6F7420757067726164653A45
:10768000206D6F726520736563746F727320746808
:10769000616E20616C6C6F7765640A0025633A2027
:1076A00043616E6E6F7420757067726164653A2015
:1076B0006E6F742073616D6520736563746F7220E3
:1076C0006C61796F75740A0062616400676F6F6442
:1076D00000756E736574005072696D61727920690E
:1076E0006D6167650025633A2025733A206D6167F7
:1076F00069633D25732C20737761705F74797065C1
:107700003D307825782C20636F70795F646F6E65EB
:107710003D307825782C20696D6167655F6F6B3D22
:10772000307825780A005365636F6E646172792042
:10773000696D6167650025633A20426F6F7420733D
:107740006F757263653A207072696D61727920732A
:107750006C6F740A0025633A20426F6F7420736F58
:10776000757263653A206E6F6E650A0025633A2074
:107770005374617274696E672073776170207573DA
:10778000696E67206D6F766520616C676F726974D2
:10779000686D2E0A0025633A204E6F7420656E6F67
:1077A0007567682066726565207370616365207413
:1077B0006F2072756E2073776170207570677261CB
:1077C00064650A0025633A207265717569726564A3
:1077D00020256420627974657320627574206F6E51
:1077E0006C792025642061726520617661696C6125
:1077F000626C650A003059301306072A8648CE3D70
:10780000020106082A8648CE3D0301070342000410
:107810002ACB403CE8FEED5BA44995A1A91DAEE84A
:10782000DBBE1937CD14FB2F245737E5953988D99E
:1078300094B9D65AEBD7CDD5308AD6FE48B24A6A2B
:10784000810EE5F07D8B6834CC3A6AFC538EFAC128
:107850002D0020002B00307800305800286E696C15
:1078600029002A2A2A20426F6F74696E67204D43CF
:1078700055626F6F742076322E312E302D6465760E
:107880002D646166323934366130663037202A2AF9
:107890002A0A002A2A2A205573696E67206E5246EA
:1078A00020436F6E6E6563742053444B2076322EF6
:1078B000372E302D356362383535373063613433D8
:1078C000202A2A2A0A002A2A2A205573696E67204C
:1078D0005A6570687972204F532076332E362E39D0
:1078E000392D313030626566633730633734202A92
:1078F0002A2A0A00636C6F636B40353030300068B1
:1079000066636C6B006C66636C6B00666C617368BD
:107910002D636F6E74726F6C6C65724033393030EA
:1079200030006770696F4038343235303000000104
:107930000203040506077561727440393030300067
:10794000756172744038303030007065726D00744B
:10795000657374004255473B2063616E277420684D
:10796000617070656E007265766572740025633AA9
:10797000205365636F6E6461727920696D6167651C
:10798000206F6620696D61676520706169722028CB
:1079900025642E2920697320756E726561636861A4
:1079A000626C652E20547265617420697420617365
:1079B00020656D7074790A0025633A20496D61670E
:1079C0006520696E6465783A2025642C20537761C0
:1079D0007020747970653A2025730A0025633A2077
:1079E000496D61676520696E6465783A2025642C6D
:1079F000205377617020747970653A206E6F6E65E0
:107A00000A00040104030402040104010403010345
:107A1000030401040000010088EACD1F55555515E7
:107A2000AAAAAA1A4D640000D1600000EC6F000001
:107A30005F6400000000000000C2010000010300BC
:107A400000000000EE0F0020ED0F002000000000FD
:107A50000000000000C2010000010300000000005F
:107A6000F00F0020EF0F002000000000FFFF0000DB
:107A70000000000000000000000000000000000006
:107A800000000000000000000000000000000000F6
:107A900000000000000000000000000000000000E6
:107AA00000000000000000000000000000000000D6
:107AB00000000000000000000000000000000000C6
:107AC00008000000FF0000000000000001000000AE
:107AD00000000000BC000020BC00002000000000EE
:107AE00079420000D4000020F0000020E8000020CF
:107AF000E4000020E00000201C0100201401002010
:107B00000C01002000000000040100208D45000051
:107B1000D94400000D45000055450000DC0E002052
:107B20003A00003AE00E00203A00003AE40E00204D
:107B30003A00003AE80E00203A00003A0000000047
:0A7B400000000000000015E015E051
:020000040001F9
:100000003DB8F3960000000000020000C0EC0100C3
:1000100000000000000000000000000000000000E0
:10002000FFFFFFFFFFFFFFFFFFFFFFFFFFFFFFFFE0
:10003000FFFFFFFFFFFFFFFFFFFFFFFFFFFFFFFFD0
:10004000FFFFFFFFFFFFFFFFFFFFFFFFFFFFFFFFC0
:10005000FFFFFFFFFFFFFFFFFFFFFFFFFFFFFFFFB0
:10006000FFFFFFFFFFFFFFFFFFFFFFFFFFFFFFFFA0
:10007000FFFFFFFFFFFFFFFFFFFFFFFFFFFFFFFF90
:10008000FFFFFFFFFFFFFFFFFFFFFFFFFFFFFFFF80
:10009000FFFFFFFFFFFFFFFFFFFFFFFFFFFFFFFF70
:1000A000FFFFFFFFFFFFFFFFFFFFFFFFFFFFFFFF60
:1000B000FFFFFFFFFFFFFFFFFFFFFFFFFFFFFFFF50
:1000C000FFFFFFFFFFFFFFFFFFFFFFFFFFFFFFFF40
:1000D000FFFFFFFFFFFFFFFFFFFFFFFFFFFFFFFF30
:1000E000FFFFFFFFFFFFFFFFFFFFFFFFFFFFFFFF20
:1000F000FFFFFFFFFFFFFFFFFFFFFFFFFFFFFFFF10
:10010000FFFFFFFFFFFFFFFFFFFFFFFFFFFFFFFFFF
:10011000FFFFFFFFFFFFFFFFFFFFFFFFFFFFFFFFEF
:10012000FFFFFFFFFFFFFFFFFFFFFFFFFFFFFFFFDF
:10013000FFFFFFFFFFFFFFFFFFFFFFFFFFFFFFFFCF
:10014000FFFFFFFFFFFFFFFFFFFFFFFFFFFFFFFFBF
:10015000FFFFFFFFFFFFFFFFFFFFFFFFFFFFFFFFAF
:10016000FFFFFFFFFFFFFFFFFFFFFFFFFFFFFFFF9F
:10017000FFFFFFFFFFFFFFFFFFFFFFFFFFFFFFFF8F
:10018000FFFFFFFFFFFFFFFFFFFFFFFFFFFFFFFF7F
:10019000FFFFFFFFFFFFFFFFFFFFFFFFFFFFFFFF6F
:1001A000FFFFFFFFFFFFFFFFFFFFFFFFFFFFFFFF5F
:1001B000FFFFFFFFFFFFFFFFFFFFFFFFFFFFFFFF4F
:1001C000FFFFFFFFFFFFFFFFFFFFFFFFFFFFFFFF3F
:1001D000FFFFFFFFFFFFFFFFFFFFFFFFFFFFFFFF2F
:1001E000FFFFFFFFFFFFFFFFFFFFFFFFFFFFFFFF1F
:1001F000FFFFFFFFFFFFFFFFFFFFFFFFFFFFFFFF0F
:10020000F80B0020690801003D090100D15A0100E6
:10021000F15A0100115B0100515B0100315B0100EB
:10022000000000000000000000000000092901009B
:100230003D090100000000003D0901003D090100E9
:10024000000000000000000000000000F133010089
:10025000000000003D090100000000000000000057
:100260003D0901003D0901003D0901003D09010072
:10027000000000003D0901003D0901003D090100A9
:100280003D0901003D0901000000000000000000E0
:100290003D0901003D0901000000000000000000D0
:1002A0003D09010000000000000000003D090100C0
:1002B0003D0901003D0901003D0901003D09010022
:1002C0003D0901003D0901003D0901003D09010012
:1002D0003D090100000000003D0901000000000090
:1002E0003D090100000000003D0901000000000080
:1002F0003D090100000000000000000000000000B7
:10030000000000003D0901000000000000000000A6
:1003100000000000000000000000000000000000DD
:10032000000000003D090100000000000000000086
:1003300000000000000000000000000000000000BD
:100340003D09010000015F5F00000000FE0B00009E
:100350009929010080060000000000000000000054
:10036000000000000000000000000000401200201B
:100370000000000001015F5F030100001F01000099
:1003800085060100000000000000000001000000E0
:10039000010000000000000000000000000000005C
:1003A0000000000070000000545F010080000000A9
:1003B000000F000001000000D104010001015F5F97
:1003C000040100001F010000F3070100000000000D
:1003D000000000000000000001000000000000001C
:1003E0000000000000000000000000005F5F01004E
:1003F000400000000507000001000000DF060100CA
:1004000038B50025054C29462046D4F80024C4F808
:10041000045405F006FCC4F8005438BD200C00203C
:1004200013B511460022CDE9002242680346382A5E
:10043000046844D194F82820022A19D01AB900F08F
:1004400047F902B010BD21482468D0F80404013AED
:10045000CDE90040082A35D8DFE802F0050A0E137E
:10046000181D22272C006A46184600F02EF9E8E7EE
:10047000184600F018F9E4E76A46184600F016F945
:10048000DFE76A46184600F00BF9DAE76A461846D5
:1004900000F00FF9D5E76A46184600F00DF9D0E7ED
:1004A0006A46184600F00BF9CBE76A46184600F09A
:1004B00009F9C6E76A46184600F00EF9C1E76FF081
:1004C0008000BEE76FF08500BBE700BF200C002076
:1004D0002DE9F04F05680446A1B0002D40F0AA8038
:1004E0002022294602A805F09CFB12AF20222946B3
:1004F0000AA805F096FB38222946384605F091FBFC
:10050000E26904F11C039846B2B10426E26A04F1E0
:100510002C03EAB10425EEB96FF08306304621B012
:10052000BDE8F08F002EF1D053F8041D3246013E95
:100530000029F7D01646E9E70326F5E7002DEAD0B3
:1005400053F8041D2A46013D0029F7D01546E2E77D
:100550000325F5E738233A460021606805F09EFB45
:100560003828D9D14FF00109CDE90270334F0DF190
:10057000080A04F1100B4E45D7F800141CD10DF1F8
:1005800028094B46002008EB850EC64533D108B13B
:10059000C7F80014A3683146C7F804340AAA2B46EA
:1005A00002A8FFF73DFF00270646BD4209F10809F2
:1005B00038D1FFF725FFB1E75BF8043FC1F5806252
:1005C000D81C20F00300904204D9FFF719FF6FF008
:1005D0008C06A3E70844CA19C7F8000449466068B6
:1005E000019205F05BFB019ACAF80C0009F10109C0
:1005F0004AF8082FBFE758F804CFC1F5806A0CF11C
:10060000030222F00302524503F1080305D87818CB
:1006100043E9020C11440120B7E70028D5D0C7F800
:100620000014D2E7394659E90223606805F04BFB14
:100630000137BAE76FF0850670E700BF200C002095
:1006400008B528220021024805F0EBFA002008BD79
:100650002810002010B5044C0F222046034905F055
:10066000BBFA204610BD00BF51100020F607010064
:1006700008B50121024803F091FA002008BD00BF2F
:100680005010002008B5FFF7DBFF40B9FFF7E2FF8D
:10069000FFF7EEFF18B9BDE8084003F0EDBA08BD5A
:1006A0006FF0850070476FF0850070476FF0850030
:1006B00070476FF0850070476FF0850070476FF0EE
:1006C000850070476FF0850070476FF085007047B8
:1006D000D1E9000103F0B0BA6FF085007047F0B5C2
:1006E00003680546B3F57D7FA7B007D040F2F53229
:1006F000934207D06FF0850027B0F0BD01F0A4FC55
:100700000020F9E700243C22214607A8CDE9024455
:10071000CDE90444069405F084FA3C22214617A84A
:10072000169405F07EFAEA69019405F11C0302B300
:100730000426EA6A05F12C033AB30424731E012B44
:1007400052D8012C50D80423002168680DEB030215
:1007500005F0A4FA04281AD06FF08000CCE7002E30
:10076000E7D053F8041D3246013E0029F7D0164663
:10077000DFE70326F5E7002CE0D053F8041D2246FE
:10078000013C0029F7D01446D8E70324F5E7022EF0
:1007900016D16E69402E29D806AF33463A4601215C
:1007A000686805F07BFA8642D6D1CDE9027602A9C7
:1007B00044B92246019801F01EFE044620469BE7FC
:1007C0000021F5E72B6A402BC6D816AACDE90423F1
:1007D000019804AA01F00FFEDDE90423044600217C
:1007E000686805F070FAE9E7012085E76FF0890095
:1007F00082E7002070474D62656420544C532033DB
:100800002E352E3000000000000000000000000027
:1008100000000000000000000000000000000000D8
:100820005430000001000000407C010080100020D6
:100830004A000000407C0100200C00200000000065
:10084000407C0100000C002000000000A8110020E6
:10085000C4050000200C002018010000000C00203E
:100860000800000002F03EBC08B572B6002383F316
:100870001488BFF36F8F83F30A8883F30B88BFF369
:100880005F8F254B5A6A22F480325A62D3F8942043
:1008900022F00102C3F89420BFF34F8FBFF36F8F94
:1008A0001E4A9A6000F058F81D4B83F309881D4BCF
:1008B00083F30A8883F30B881B4B15A1D1E9000150
:1008C000C3E9000100F0EEF8184B19498B4212D32E
:1008D0000020184B18498B4218D302F0CFFF18683C
:1008E00050F82240586840F822400132986882420D
:1008F000F5D30C33EAE70022F8E71C6844F822003D
:1009000001325C68A242F8D30833E4E70022F8E73A
:10091000A5EDF5FEA5EDF5FE00ED00E000020100FD
:10092000F80B002000040020F80B0020280801002C
:100930004C0801004C08010064080100EFF3088036
:10094000EFF309812DE9F00F6B46724600F094F940
:1009500008B0FFF787FFFEE738B572B6002383F3D0
:10096000138883F311884FF0FF30274A03F12001E9
:100970000133102B42F82100F8D100234FF0FF344F
:10098000214A03F160010133102B42F82140F8D1D4
:10099000012200251D4B29465A60C3F84843C3F87D
:1009A000084303F580535A60C3F84843C3F808432B
:1009B000A3F55043C3F800558022C3F808431448F8
:1009C00005F02FF929468022124805F02AF9124B2A
:1009D0002946C3F800558022C3F808430F4805F0A4
:1009E00020F9802229460E4805F01BF90D4BC3F86B
:1009F00008454FF05023C3F8084362B6BFF34F8F4A
:100A0000BFF36F8F38BD00BF00E100E00040015030
:100A100080800050808100500090005080900050F5
:100A2000809100500070015008B5EFF31083012B46
:100A30000C4A07D1126ABFF34F8F511C4A424A41F8
:100A4000104608BD01F042FB00B172B6126ABFF356
:100A50004F8F531C5A425A4101F038FB0028EFD007
:100A600062B6EDE70080FF0008B5EFF31083012BBD
:100A70000B4A06D1D269BFF34F8F02F00102104634
:100A800008BD01F023FB00B172B6D269BFF34F8FEE
:100A900002F0010201F01AFB0028F0D062B6EEE786
:100AA0000080FF00694A10B5D2F8D03043F002034D
:100AB000C2F8D03001F00AFB30B14FF050230022D1
:100AC000C3F81421C3F8182101F00FFB28B101224B
:100AD0005F4BC3F8382AC3F878254FF47F02D2F869
:100AE0003031D2F83421BFF34F8FC3F30B03092BFE
:100AF00005D1012A1EBF0122554BC3F8782501F00C
:100B0000F4FA18B10E22534BC3F8E42E01F0DEFACA
:100B100030B100224E4BC3F80C270122C3F8102736
:100B20000022D30003F57F03D3F80013BFF34F8FE8
:100B3000013108D0D3F800130132D3F80433B2F5F1
:100B4000807F0B60EDD1EFF31084FFF78DFF00285D
:100B50004DD0BFF34F8F404BD3F80024012AFBD177
:100B6000C3F80425D3F80024012AFBD1012C03D0BB
:100B700001F0ACFA00B172B6FFF776FF58B1374A10
:100B8000D36923F00103D361BFF34F8F324AD2F808
:100B90000034012BFBD1FFF747FF68B12F4A136ADE
:100BA00023F0FF0343F020031362BFF34F8F2A4A61
:100BB000D2F80034012BFBD1012C03D001F086FACE
:100BC00000B162B60022244BC3F80425D3F80024F8
:100BD000012AFBD1BFF34F8F1C49214BCA6802F495
:100BE000E0621343CB60BFF34F8F00BFFDE7FFF719
:100BF0001BFF0028ADD1154AD2F88C3043F4406376
:100C0000C2F88C304FF47F03D3F83021D3F834315D
:100C1000BFF34F8FC2F30B02092A16D1013B022BFF
:100C200002D8104AD35C83B10C480F4903680A4AC2
:100C30008B420CBF5A230023C2F8103EC36A8B427A
:100C40000CBF5A230023C2F8003E10BD00ED00E0A7
:100C50000040005000A00350009003500080FF00AF
:100C60000400FA05C0340100FA50FA507C22014910
:100C700004F0B2BFDC18002038B51D46364B374CA7
:100C80005B68C3F308032360EFF30383C4E9012027
:100C90006365C2F3801302F00C020C2AE16036D1C6
:100CA0000BB9EFF3898120222D48216104F094FFD4
:100CB00025B1202229462B4804F08EFF264B9A6A44
:100CC000A265D96AE165986B206602F4004060660F
:100CD000586BA06602F08000E0669A62D962D3F891
:100CE000E42021482267D3F8E810616702F0400150
:100CF000A167C3F8E4200E2101F009FA2268D31E8F
:100D0000042B1CD8DFE803F0090F1215180013B9E3
:100D1000EFF38881C7E70146C5E70C211348BDE81A
:100D2000384001F0F4B912211148F8E70B211148BD
:100D3000F5E70D211048F2E70E211048EFE70F2AE2
:100D400098BF1421BDE8384089BF25210C480D48C3
:100D5000103A01F087BB00BF00ED00E0DC18002076
:100D6000F018002010190020C3340100D134010014
:100D7000DD340100EF340100FA34010007350100D1
:100D800015350100293501002DE9F34106460F46CE
:100D90000C4DD5F82C80C04710F00104FBD139462A
:100DA00030466B69984740B9C047C307FCD42B6AEB
:100DB000019302B0BDE8F0411847204602B0BDE8FB
:100DC000F08100BF5035010010B5094C0020A36828
:100DD0009847236902209847A46A4FF4E131012023
:100DE000A0472346BDE8104001211520184700BF49
:100DF00050350100064B82B01868002382B262F3BE
:100E00000F03000C60F31F43184602B0704700BF89
:100E100098350100014B1869704700BF841000200D
:100E2000014B5869704700BF8410002010B5044C76
:100E3000204600F0B5FE002084F8200010BD00BF61
:100E40008410002038B50C4D0C4695F8203013B9AD
:100E50004FF0FF3038BD0A460146284600F02AFF11
:100E6000064B984205D00B3B9842F1D100206C61B3
:100E7000F0E76FF00100EDE7841000200B00AD0BF0
:100E8000F0B51B4E054696F820300C4691B01BB9C4
:100E90004FF0FF3011B0F0BD00F06043B3F1005FE0
:100EA00021D100230A460146304600F0EFFB114BEA
:100EB00098421AD00B3B9842EAD1346111E0A71B4B
:100EC000402F28BF4027A9193A46684604F084FEFF
:100ED00039466846FFF7D4FF0028DBD14036B442DC
:100EE000EDD80020D6E70026F9E76FF00100D1E742
:100EF000841000200B00AD0BC3B2012B10B540F0E5
:100F000096804DF6C023994270D028D8B1F5615F24
:100F10006FD011D8B1F5965F6DD008D8B1F5966F46
:100F20006BD0B1F5166F6BD06FF007005DE0B1F5D7
:100F3000165FF9D1454B33E047F61223994262D050
:100F400007D8B1F5964F61D0B1F5E14FECD1404BE8
:100F500026E0B1F5164FE7D14FF41D0320E03D4BDD
:100F6000994255D011D8B1F5E13F54D007D8B1F529
:100F7000614F53D0B1F5963FD6D1374B10E0B1F564
:100F8000613FD1D14FF06C730AE0B1F5612F48D0C9
:100F9000324B994248D0B1F5E12FC5D14FF0E8630B
:100FA00010F4E06F46D110F4404103D0B1F5804F0A
:100FB00043D1102110F4405203D0B2F5805F3FD1ED
:100FC0000E2210F4403003D0B0F5403F3BD1012059
:100FD000234C20766276E361A1760A4324681043AD
:100FE000C4F82435C4F86C05002010BD4FF4650327
:100FF000D6E71C4BD4E71C4BD2E74FF49E23CFE738
:101000004FF41D23CCE74FF40003C9E7174BC7E7A4
:101010004FF08063C4E74FF0EB73C1E74FF46B030D
:10102000BEE74FF07063BBE74FF08053B8E76FF057
:101030000300DAE76FF00800D7E76FF00A00D4E7A3
:101040006FF00900D1E76FF00B00CEE700502700EA
:1010500000C0750090D0030000903A0140420F009C
:101060008410002000F03A0000B0130000A04E00F1
:1010700010B58EB02422002105A804F0D2FD4FF057
:10108000FF33CDE90133CDE903334FF0EB730B931D
:101090000723104C01A8D4E902128DF8363001F074
:1010A00054F801460022204600F03AFA0A4B9842D2
:1010B0000DD10C9B002023831B0CA3760B9BC4E952
:1010C0000400E361012384F820300EB010BD6FF0FE
:1010D0000100FAE7841000200000AD0B7FB5002569
:1010E0000C46C0F808511646D0F80821D0F8002266
:1010F00022F02002C0F80022104AC0F8082301F0B4
:1011000074F8A560256104F14C03D3E8EF1F21F4C6
:101110007F0121F47041C3E8E21F002AF5D11022BB
:101120002946684604F07DFD042368468DF80030AA
:101130000196D4E90013984704B070BD10020A006C
:1011400000F01F03400909D1074A02EB8303D3F8DB
:101150000012064A0A40C3F800227047002280337A
:1011600052F82330FFDE00BF00258450F0F8FCFF6A
:101170002DE9F04F804690F804A05020664F0E46AF
:1011800000FB0A70416885B049B113F0020304D036
:10119000836B002B00F0B2800123009300E00091EC
:1011A0004FF0500909FB0A73DB6CD90600F1A680E9
:1011B0004FF0010BB3180293029BB34200F0A780DB
:1011C00006F06043039398F80450D8F8004009FBF8
:1011D00005739A6B9AB9039BB3F1005F40F0998055
:1011E000019200F0A1FD09FB0572D16C204601F0CF
:1011F000010100F0C8FF28B900F09EFDE3E70123DC
:101200000193EEE7516C33460029BCBFD4F84C156E
:101210005164019A42B109FB05713078D1E90E237E
:10122000D054D1E90E3213441BB1C4F84435C4F88C
:1012300048B50022C4F82021D4F82011C4F8582160
:10124000D4F85811C4F85021D4F850210822C4F819
:101250000025009AE2B14FF48003C4F80433C4F8C7
:1012600008B000F069FD502303FB0A7251680029A1
:101270004BD1D26C120748D503FB0A734C33D3E829
:10128000EF1F21F00801C3E8E21F002A36D0F6E77D
:10129000C4F808B0019300F04FFD09FB0572D16C52
:1012A000019B01F001012046019300F06CFF844690
:1012B000019BD4F84C05D4F84425BCF1000F0DD1A6
:1012C0009342F0D005EB850507EB0515D1B100F091
:1012D0002BFD2946204600F0CDFFC2E705EB850532
:1012E000934207EB0515F1D10028EFD100F01CFD6A
:1012F0002946204600F0BEFF00F01EFD074805B05D
:10130000BDE8F08FC4F80CB0E1E7013654E70448BB
:10131000F5E70448F3E700BF581900200800AD0BBB
:101320000000AD0B0400AD0B430904D10123034AB7
:1013300083409360704700239B60FFDE002584504C
:1013400000F01F0340090BD1084A02EB8302D2F8D8
:101350000012074B0B4043F00303C2F80032704702
:101360000022803352F82330FFDE00BF0025845076
:10137000F0F8FCFF2DE9F84391F8303005460C46B3
:1013800090F804800F6853BB5023DFF85091781C0D
:1013900003FB0893DE6C46F00072DA6404D0384632
:1013A000FFF7C2FFFFF7CCFF6068411C01D0FFF7D9
:1013B000C7FE94F82C30012B11D1502303FB089366
:1013C000E06846F02066421CDE6401D0FFF7B8FEFC
:1013D000A068431C03D0FFF7A7FFFFF7B1FF94F805
:1013E0002F0038B950223D4B02FB0833DA6C42F033
:1013F0008072DA6494F82CC094F82D1094F82E20A2
:101400002B68D4F828E041EA0C010A43E668D4E9E5
:101410000198C3F824E5C3F86C2550B9BCF1010F5D
:10142000C3F80C75C3F8149504BFC3F80885C3F856
:101430001065D3F8682503F26458012A08BFDA6002
:10144000D3F86425012A13D1082149F64046244FD8
:10145000C3F8001547F001075A60D8F800309BBB6D
:101460002B68D3F88024C3F880240022C3F8002519
:1014700000212B6894F83220C3F81011D3F8100122
:10148000C3F82011D3F82001C3F82411D3F82401A4
:10149000C3F84411D3F84401C3F85811D3F85811D4
:1014A00043F307335201002BD2B212DB0D49C818A7
:1014B00080F800230122580903F01F0302FA03F306
:1014C00041F82030BDE8F8834020B847013EC4D140
:1014D000C6E7054903F00F03CA54F3E75819002083
:1014E000A035010000E100E014ED00E000F01F0372
:1014F00040090BD1084A02EB8302D2F80012074BD5
:101500000B4043F00203C2F80032704700228033E0
:1015100052F82330FFDE00BF00258450F0F8FCFFB6
:101520002DE9F3479046502290F80490514C02FB6D
:1015300009FA04EB0A070D4697F8481006460029F9
:1015400040F0858009EB890004EB001004F069FB92
:101550002B69AA6944F80A306B69BB6302B1013A8E
:10156000502303FB0943DA632A6A042A81BFEA692C
:101570009A610022DA6195F83130B8F1000F37D066
:1015800083F001073F0233B1502303FB0943DA6CB8
:1015900042F00102DA64502303FB09440123C4F83A
:1015A000048084F848303468D4F84C2112BB2946B2
:1015B0003046FFF7DFFE0822002334688DF807303D
:1015C000C4F800250DF10702C4F84425C4F84835D5
:1015D00001230A25A360E360D4F85831002B38D1E9
:1015E000254B402043F001039847013DF4D128E00A
:1015F0004746C8E708224FF06409C4F80025636035
:101600001D4B43F0010AD4F84431F3B9D4F8243126
:10161000DBB94FF42070D047B9F10109F3D14B4643
:101620000022C4F84C21D4F84C11C4F81021D4F88D
:101630001011C4F84421D4F84411C4F80025002B3B
:10164000B5D10E4802B0BDE8F0870123E8E70C48A9
:10165000F8E70023C4F820319845D4F82021C4F8D5
:101660000035084B08BF00231F4333680648C3F802
:101670000473E7E758190020A03501000100AD0B05
:101680000C00AD0B10020A000000AD0B2DE9F04775
:1016900084460F469E4616460579002A51D04FF0E3
:1016A000500ADFF8AC80D0F800900AFB058ADAF81F
:1016B000044074B96BB9DAF82C50002D43D1CAF844
:1016C0002C20FFF755FD0446CAF82C502046BDE8F3
:1016D000F0871EF0030F07D0734632463946BDE847
:1016E000F0476046FFF744BD07F06043B3F1005F89
:1016F0004FF0500414D104FB058400F015FBE26A9E
:101700001AB1144C00F018FBE0E7C4E90A7605EBC7
:101710008505484608EB051100F0B7FD0E4CF1E7D2
:1017200004FB0584A36B83B100F0FEFAE36A002B8F
:10173000E7D1E36C012243F00203C4E90A76E364D3
:10174000E5E7064CC2E7034CC0E7054CBEE700BF27
:10175000581900200B00AD0B0000AD0B0600AD0BBF
:101760000A00AD0B2DE9F84350230679284D046893
:1017700003FB0653D4F80473DA6AC4F8087322B979
:101780002448C4F80473BDE8F88306EB860005F12D
:101790004C024FEA001802EB0012D2E8EFCF4CF0F7
:1017A000080CC2E8E0CF0028F7D10122E26031B393
:1017B000D96C01EA02094946204600F0E4FC002801
:1017C000FAD000F0B1FAB9F1000F1CD1D4F82031F1
:1017D00053B10123E360D4F85831002BFBD02046ED
:1017E00005EB080100F046FD00F0A6FA0023C4F85E
:1017F0002031D4F82021502202FB0655EB62064826
:10180000C4F80473BFE7D4F85831002BE7D1EBE7F5
:10181000581900200500AD0B0000AD0B2DE9F84371
:1018200090F80480484F08EB8806360106F14C0515
:1018300004683D44D5E8EF3F43F48052C5E8E02F0B
:101840000028F7D1DB047BD4480705D5502303FBE0
:1018500008739B69002B75D03C4B3E44C4F8083399
:101860000823C4F800350023C4F81031D4F810213F
:10187000C4F84C31D4F84C21C4F844310A03D4F8EC
:1018800044318B0303F4804302F4005249031343B1
:1018900001F400410B43D5E8EF2F1A43C5E8E12FCF
:1018A0000029F8D14FF0500909FB0879D9F8083020
:1018B000BBB9D9F8043063B9D5E8EF3F23F47F030F
:1018C00023F47043C5E8E23F002AF5D12048BDE883
:1018D000F8830321304600F063FCD9F80830002B70
:1018E000EAD0D4F80433590713D5502303FB087307
:1018F0005A6872B1DB6C1A030BD5D5E8EF3F23F4BD
:101900000023C5E8E23F002AF7D10621304600F067
:1019100047FC502303FB0873DB6CDB0401D40D4848
:10192000D5E7D4F84C310BB901232360502303FBD6
:1019300008735B68002BF2D0044BC4F80433EEE765
:101940000548C4E70548C2E75819002010020A00FC
:101950000200AD0B0000AD0B0B00AD0B0800AD0B92
:101960002DE9F84F056801F06043D5F804A3B3F101
:10197000005F90F804B089461746C5F808A37CD1EB
:101980005023404E03FB0B639A6852B15B68002BF7
:101990005ED1D5F81021002A5AD0C5F81031D5F8FB
:1019A0001031502404FB0B64E269C4E90297002A59
:1019B0003CD00BEB8B0897424FEA081824D24FF02B
:1019C000000B3A46A1694846C4E902BB04F004F999
:1019D000E269A069D21BC119E26104F0C7F863682B
:1019E0006BB1B04449463A46404600F0EAFBE36C2E
:1019F000990404D55A4641462846FFF76FFB224812
:101A0000C5F804A3BDE8F88F4846A16904F0E4F8DE
:101A1000E36963620023E3611C4B9844D8E8EF3F1D
:101A200043F40023C8E8E23F002AF7D1502303FB28
:101A30000B63586ADA689968DB6C121A0144C5F8BE
:101A40003415C5F83825DA04D9D501232B60D6E73B
:101A5000502303FB0B6633698BB9F36CC5F83495DF
:101A60005B04C6E90497C5F83875C8D5D5F80032C7
:101A700043F02003C5F80032C1E70548C0E7054838
:101A8000BEE700BF581900200000AD0BA4190020CC
:101A90000A00AD0B0B00AD0B50232DE9F0413C4D7E
:101AA00090F80480046803FB0853DB6CD4F8000250
:101AB00003F48223B3F5805F68D1D4F80463C4F8DB
:101AC000086309B9830656D4D4F8003223F0200302
:101AD000C4F800324FF4842308EB8801090101F1B6
:101AE0004C072F44D7E8EF0F1843C7E8EC0FBCF1C1
:101AF000000FF7D12AB9502303FB08535B68002B72
:101B000041D1244BC4F8083301236360D4F8443135
:101B1000002BFBD00023C4F84C31D4F84C21C4F87E
:101B20001031D4F81021C4F84431D4F84431502392
:101B300003FB0853DA6C12F400421FD1DA6120462D
:101B400000F053FB502303FB08550023AB602B61CF
:101B5000D7E8EF3F23F47F0323F47043C7E8E23F65
:101B6000002AF5D126F4202626F404760A48C4F883
:101B70000463BDE8F0814FF48033ADE7204629448B
:101B800000F045FBDBE701236360EFE70348F0E784
:101B90005819002010020A000000AD0B0500AD0B23
:101BA0002DE9F8432F4A03680679C3F8082343F365
:101BB0000733002B04460DDB01215A0903F01F03F4
:101BC000994002F12003284A42F82310BFF34F8FB7
:101BD000BFF36F8F012220461146FFF75DFF012101
:101BE0002046FFF7BFFD50212279204D236801FBDD
:101BF0000252D46CD3F80C05E201D3F81495D3F853
:101C00000875D3F8108509D54FF0FF32C3F80C25BD
:101C1000C3F81425C3F80825C3F81025A30116D569
:101C2000411C01D0FFF762FCB9F1FF3F02D04846EA
:101C3000FFF75CFC22010AD5B8F1FF3F02D0404615
:101C4000FFF754FC7B1C02D03846FFF74FFC5023B3
:101C5000002203FB0653DA6483F848205A60BDE88B
:101C6000F88300BF10034A0000E100E0581900208B
:101C700010B5502402790B4B04FB02335B686BB93F
:101C80000368D3F810211AB9D3F80025082A07D021
:101C900011B1D3F83C350B60034810BD0348FCE795
:101CA0000348FAE7581900200000AD0B0800AD0BFF
:101CB0000B00AD0BF7B505461646FFF751FE164B68
:101CC0000446984222D1032128462F79FFF7A6FD2A
:101CD000124B984201D0A0421BD15022104B02FB64
:101CE00007335B6893B90C4C284601A9FFF7C0FF86
:101CF000A042F9D1019BB34207D3012228461146E5
:101D000003B0BDE8F040FFF7C7BE064C204603B065
:101D1000F0BD0446FAE700BF0000AD0B0B00AD0BB1
:101D2000581900200800AD0B72B6024A136801333F
:101D300013607047A8190020034A1368013B136021
:101D400003B962B6704700BFA8190020003A18BF57
:101D50000122003918BF012103688900074841EAC0
:101D60004201186359605A6842F001025A60BFF399
:101D70004F8FBFF36F8F0020704700BF04AAFF0092
:101D80000722024BC3F80423704700BF0030005005
:101D9000084BD3F80801D3F80021003818BF012000
:101DA00080000AB140F00100D3F804310BB140F0DB
:101DB00002007047003000500022074BC3F800219A
:101DC000D3F80011C3F80421D3F80411C3F8082193
:101DD000D3F80831704700BF0030005000231720AF
:101DE0000C49012B03F1010201D81346F9E703F571
:101DF000C073202A41F823001346F2D10023172094
:101E0000044A03F5E0710133202B42F82100F8D198
:101E1000704700BF0030005010B59DF80840C00B5F
:101E200043EA0423064CC90B43EA0213884200D953
:101E300010BDC2B202F5C07244F822300130F5E79D
:101E40000030005010B59DF8084000F1604043EAB2
:101E5000042301F16041074C400B490B43EA021394
:101E6000884200D910BDC2B202F5E07244F82230B7
:101E70000130F5E700300050C0F30E03C3F5004316
:101E8000B3FA83F3C3F11B03064AC0F3C730DBB2D6
:101E900040F4807043F48073C2F80005C2F8043542
:101EA000704700BF0030005043030148184470479A
:101EB000FF1FF81F054BC0F30730090241F0300146
:101EC00000F5007043F82010704700BF003000504C
:101ED000044BC0F30730090200F5007043F82010EE
:101EE000704700BF0030005008B5FFF751FF044BAA
:101EF000162118600348BDE8084000F008B900BF8B
:101F0000EC1F0020A63501000C22014903F064BE3D
:101F1000EC1F002010B501F050FA044690B901F012
:101F2000E1FE044680B90A4A2E21D368094823F00D
:101F300008031B041B0C43F0BF6343F40033D3605E
:101F400000F0E5F8204610BD45F22354FAE700BF43
:101F500000ED00E0BC350100024B1860024B002090
:101F600019607047FC1F0020F81F00201FB5274C88
:101F7000426923685A6282699A62C269DA62026AB5
:101F80001A63426A5A63826A9A63C26ADA63026BAC
:101F90001A64426B5A60826B9A60C26BDA60026CA0
:101FA0001A61426C5A61826C9A61C26CDA61026D8C
:101FB0001A62826D5A65C26D9A65026FDA65026EA9
:101FC0001A66826E5A66426F9A66EFF388825A6486
:101FD000EFF389829A644268DA64EFF394821A65B7
:101FE000026801A81A67FFF78FFF2368019ADA6673
:101FF00001221A70064B1C686408640020462146C2
:102000002246234603F0C1FE04B010BDFC1F002091
:10201000F81F002000B5A1B001A8FEF727FE029B23
:1020200063B15B060AD4019B23F00203052B05D1A3
:10203000044B1B6813B101A8FFF798FF21B05DF8AE
:1020400004FB00BFF81F0020BFF34F8F0549064B6C
:10205000CA6802F4E0621343CB60BFF34F8F00BF46
:10206000FDE700BF00ED00E00400FA05F8B54368A5
:102070000C2B26D14B68042B23D14FF0FF3304687F
:102080000E6821683360E1B1A268D2B10623012055
:1020900001F0EBF8A8B961680B4BD3E9005CA942E9
:1020A0000AD3A26865448F18AF4205D8206803F0B0
:1020B00093FD00203060F8BD0130042803F10803CF
:1020C000EBD10220F7E700BFEC3501004FF47F03AE
:1020D000D3F83001D3F83431BFF34F8FC0F30B0086
:1020E000A0F109035842584170474FF47F02D2F8DB
:1020F0003031D2F83401BFF34F8FC3F30B03092BF8
:1021000003D1431E58425841704700207047FEF7E4
:102110003BBE012070476FF003007047002382B080
:102120000193019802B070476FF0030070470023DD
:1021300082B00193019802B07047022814BF6FF07B
:10214000030000207047FEF79BBE30B501EB820212
:10215000914200D130BD51F8044B04F07F037F2B36
:102160004FEA144408BF4FF0FF33032CF0D8DFE8E8
:1021700004F0020406080360EAE74360E8E78360CE
:10218000E6E7C360E4E70346D0F8580130B931B957
:10219000D3F82001003818BF012070470120704794
:1021A00030B504460D4685B010220021684603F084
:1021B00038FDD4E9001368468DF80050984705B003
:1021C00030BD7FB504460E461546002110226846F4
:1021D00003F027FD012368468DF80030CDE9016545
:1021E000D4E90013984704B070BD10B50446FFF75A
:1021F0009BFDD4F8583133B1D4F8043313F4800381
:1022000008BFC4F80035BDE81040FFF795BD70B5B4
:102210000D4604460522AA21D0F83C65A86903F0C2
:1022200000FD0522AB69C4F83435C4F83825002216
:10223000C4F81021D4F810110121E162D4F8101172
:102240000029FBD0C4F84C21D4F84C11C4F810215B
:10225000D4F81021D4F83C259642EA6109D15A1EDF
:10226000043312F8011FAA2903D19A42F9D100239D
:10227000EB6170BDD0F8583133B1CB6CC3F3003291
:10228000DB0458BFC0F80025704770B5CE6C0D4612
:1022900006F001010446FFF776FF38B94FF48003DA
:1022A00046F00406EE64C4F8043370BDD5E90A367E
:1022B0005AB1296CEA6B761A964228BF1646194421
:1022C0003246A86B03F088FCAB6B4FF0FF326A64B8
:1022D0001BB1C4F84435C4F848650023C4F8203164
:1022E000D4F82021C4F85831D4F85821C4F850311A
:1022F000D4F850310823C4F800354FF48003C4F8F3
:1023000004330123A360D0E74B6830B513F01F05F9
:102310002DD102680C681068C0F30720844226D2D1
:102320005068556094600C7C23F01F0304F0010496
:102330001C438B7CDB0003F018031C434B7C5B00CD
:1023400003F006032343D3608B68013B23F01F0493
:10235000CB685B0003F00E03234343F001031361DA
:102360005060BFF34F8FBFF36F8F284630BD012001
:10237000FCE7036800205A68C9B258609960D860C9
:1023800018615A60704770B50546002403681E68DE
:10239000C6F30726B44201D1002070BD214628466D
:1023A000FFF7E7FF0134F5E7C0037047C00300F50E
:1023B000FF407F307047002070471F2070474FF468
:1023C0000040704700F57F40C03040037047402018
:1023D00070475F2070474FF40050704700207047EF
:1023E00008B5FFF717FE72B620BFFDE70020704763
:1023F0000020704770470B4670B5114618B103288E
:1024000006D0032070BD1846BDE87040FFF72EBE11
:102410005A68082A01D00220F4E74C68042CFAD14B
:102420001D684FF0FF330E68296833600029F2D031
:102430006B68002BEFD026237422012000F015FFDB
:102440000028E8D1224623230120696800F00DFF0F
:1024500004460028DFD1D5E90001FFF77DFD30609B
:102460002046CFE730B50C46154685B038B139B1B6
:10247000FFF74DFE041E03DA204605B030BD0446CA
:1024800040F60D23ADF80E3009230B4901A805F0E5
:102490000F028A5C2D091A54013B012BF7D147F634
:1024A00030030C21ADF80430FFF731FE0028B4BF33
:1024B00004462418E0E700BF0C36010008B5154BB0
:1024C00083F30A88144800F063FF00BBFFF722FD86
:1024D000E8B9FFF783FFD0B9FFF788FF98B9FFF796
:1024E00089FF00F0C1FE35210C48FFF710FE00F017
:1024F00007FC26210A48FFF70AFE00F039FA00F02F
:1025000095FE002008BDFFF773FF0028E7D000F01C
:10251000E9FDEEE700040020AC1900201C360100A4
:10252000513601002DE9F04F93B00093574B81468F
:10253000D3F800B00BB2002B0D461646C1F302686B
:10254000C1F3024A04DA6FF0800013B0BDE8F08FE7
:102550008B42C36001D10020F7E708EB0A03042B8C
:10256000F1D8CC0F64014FEAC80731463A46DBF890
:10257000080044F0020300F078FE01460028E2D192
:10258000202202A803F04DFB3A46314602A84FEA4A
:10259000CA0603F021FB32460099DBF8080044F03C
:1025A000060300F062FE07460028CCD10146202237
:1025B0000AA803F036FB324600990AA802AE03F0DF
:1025C0000BFB33460137B84514D91A46BC460DE01B
:1025D000D2F808E0D16818687144884203D259687B
:1025E00008448645AFD30CF1010C0832C445EFD145
:1025F0000833E7E715F0006F18BF202409F118072A
:1026000007EB880844F00203474513D1202C26D15C
:10261000002D02DBC5F3C0456C0109F128050AAEA7
:1026200005EB8A0A44F0060455451AD1009BC9F807
:102630007C3090E77268DBF8080056F8081B0193BD
:1026400000F013FE00287FF47EAF56F8042C019BA7
:1026500047F8042F56F8082C38633A62D4E7002470
:10266000DBE77268234656F8081BDBF8080000F029
:10267000FCFD00287FF467AF56F8043C45F8043FA2
:1026800056F8083C28642B63CEE700BFB019002041
:102690002DE9F0411F461A4B0D461646D3F800802F
:1026A00000F0D7FE044608B900F01CFDE368002BDB
:1026B00001DA00F017FD032D01D900F013FD04EB42
:1026C0008504E569E36CED1A16D006233A463146D7
:1026D000D8F8080000F0C9FD08B100F003FDBD42C4
:1026E00028BF3D46E36CE16B2A461944304603F0AF
:1026F00073FAE36C2B44E3642846BDE8F08100BF25
:10270000B01900202DE9F0411D461A4B0F46164620
:10271000D3F8008000F09DFE044608B900F0E2FC0A
:10272000E368002B01DA00F0DDFC032F01D900F093
:10273000D9FC04EB8704E36AE26E9B1AAB4201D238
:1027400000F0D0FC02232A463146D8F8080000F0F9
:102750008CFD08B100F0C6FCE36EE06D2A46314600
:10276000184403F039FAE36E00202B44E366BDE819
:10277000F08100BFB01900202DE9F04105464FF06F
:1027800001080E4E0E4B37685C681CB9284637604E
:10279000BDE8F0812268936813F400700CD1A3693E
:1027A000012B09D0D368346023B19847002801DA9F
:1027B00000F098FCC4F81880246AE6E7B0190020FD
:1027C000B419002038B5044610B96FF0800038BD48
:1027D0008368002BF9D01A68002AF6D05D68002DB6
:1027E000F3D00B4BE861A8691D6020B92B68DB684A
:1027F00053B90123AB61A36804F10C001B681B698A
:10280000984701232360E2E798470028F1DADCE7E4
:10281000B01900204268024B08461A60704700BF9A
:10282000B0190020002330B505680446AA68C0E945
:10283000063312F4406F85B01CD012F4006202D04F
:1028400000F082F90246A96A2B6968460B440731F9
:1028500023F0070321F00701CDE9021300930023C1
:1028600005490193EB6800F06BFA684600F0D4FD6F
:10287000024B1C6005B030BD79270100B019002063
:1028800001F00C0370B50C2B0CBF154605464A062B
:102890000C461ED58B0658BF2835AB6913F8026C61
:1028A00084F00803C3F3C003C6F38012934201D03F
:1028B00000F018FC16F0A00F1CD176B1032E15D035
:1028C00032461C210D48FFF7CDFD6FF083032B60CE
:1028D0000AE000F007FC2026E2E700F007FB0446D0
:1028E0000146074800F094FD204670BD284600F0E0
:1028F0000DFAF9E732461F210248E4E77736010076
:10290000F80B002093360100EFF308807146EFF3D7
:102910000982EFF30B830CB406B4FFF7B1FF8646D0
:10292000009900F0080001F00801401A02DC12DBF7
:1029300004B070471EF020031CBF2DE9F00FBDF15D
:10294000080D0A4C254626462746A046A146A24623
:10295000A34630B4704704B030BC1EF020031CBF47
:102960001DF1080DBDE8F00F04B07047A5EDF5FEB0
:10297000084BDA6882F07F4282F47F0242F48042A0
:10298000DA6000221A765A76DA76DA77602283F8ED
:102990002220704700ED00E0009A0A4B9A420FD1C6
:1029A0000122904301460246034604460546064678
:1029B00007468046814682468346844686460447CB
:1029C000FEE70000A5EDF5FE2DE9F041044618B93B
:1029D00043F6DA30BDE8F0810029F9D0836800259C
:1029E00013F4406F14BF01230023134F43F002037D
:1029F000DFF848800B6000F13006236AAB4201D853
:102A00000020E7E71421A369E26906EB830301FBD9
:102A100002330C226A4399188968090709D59B5823
:102A2000BB4201D04345D3D1186810B10121FFF753
:102A300041FA0135E1E700BFB4100020AC100020DE
:102A400070B5324C86B03248FFF79DFC23680125F3
:102A50005A1C01932F4B2260DA681B694FF44076B1
:102A6000039300232A4801A902920495ADF814604B
:102A70008DF81630FFF748FC18B143F6DA3006B08F
:102A800070BD23688DF816005A1C0193224B204814
:102A90000293224B01A9CDE903352260ADF8146001
:102AA000FFF732FC0028E8D123688DF816005A1C85
:102AB00001931B4B164802931A4B01A9CDE903352C
:102AC0002260ADF81460FFF71FFC0028D5D1236801
:102AD0008DF816005A1C0193134B0D480293134BAB
:102AE00001A903930223049340F201132260ADF87D
:102AF0001430FFF709FC04460028BED12A462946B7
:102B00000348FFF723F92046B9E700BFBC190020AE
:102B1000A81000202437010060370100805F010009
:102B20002008010020080100000C0020200C0020DB
:102B3000014B1868704700BF24370100014B1B6828
:102B40001868704724370100014B1B6858687047AC
:102B50002437010008B5FFF7C7F9FFF72DF90A4B35
:102B60005A68103AD3B2120609D401215A0903F067
:102B70001F03994002F16003044A42F82310BDE8A4
:102B8000084000F0AFBA00BF00ED00E000E100E057
:102B90000020034BD8765A6A42F470225A6270477A
:102BA00000ED00E00349044BCA68002092B21343D1
:102BB000CB60704700ED00E00800FA0500224FF0FE
:102BC000FF300D4B02F1A0010132102A43F8210021
:102BD000F8D1D3F88022002022F00802C3F8802226
:102BE000D3F88022D3F8802222F40072C3F8802226
:102BF000D3F88032704700BF00E100E008B5FFF76E
:102C0000BFF80822024BC3F880211A60002008BDDB
:102C100000E100E0064BD3F8D02022F00102C3F817
:102C2000D020D3F8D02042F00202C3F8D020704761
:102C300000ED00E037B50124FFF7D0F8174D22462C
:102C400005234FF4813016490094FFF7E5F822463A
:102C500007234FF0005013490094FFF7F3F8D5E92C
:102C60000101072300220094FFF7D6F80723002272
:102C70000D490E480094FFF7E5F82969E868013925
:102C8000FFF7FAF8062300224FF4082008490094C1
:102C9000FFF7C2F8002003B030BD00BF24370100A9
:102CA000FF7F0100FF7F0020FFFF03200080002046
:102CB000FFFF0F0038B500240E4D002155F8040B1E
:102CC0000134FFF705F91C2CF7D10020012240F256
:102CD0000111094BC3F88004C3F88424C3F8C0046D
:102CE000C3F8C424054AC2F840154FF48072C3F8F3
:102CF000402438BDB436010000300050009003502D
:102D00000122014B1A607047C019002010B504461B
:102D1000094B2289186861680623806800F0A5FACB
:102D200028B9064B1B68012B01D100F087F86FF022
:102D30008603236010BD00BFB0190020C019002019
:102D40002DE9F84305461E460068134B9046AA68D5
:102D5000A0F1080440E90233503890420F4601D2F6
:102D600000F0C0F9A4F1480948220021484602F0C9
:102D700058FF002344E9073344F8143C4FF08073B4
:102D800044F8043C6FF0020344E9036744F8208CE4
:102D9000C5E90093BDE8F883A5EDF5FE30B5094C13
:102DA000024661680023084640B105686D68954297
:102DB00005D11BB1826860609A60816030BD0346B6
:102DC0008068F1E7441A002038B504462AB10B6840
:102DD0009B68DB0512D5002038BD0B4B1D680DB973
:102DE00000F080F900222B6899692C338A4203D0C5
:102DF00053F8040FA04204D19142ECD16FF0FC00D3
:102E0000EAE70132F2E700BFB019002070B50446CE
:102E10000E461546002130220C3002F002FF064B10
:102E200020461B68A6606360656100F001FA00231C
:102E30002061236070BD00BFB0190020044B1B68E7
:102E40001BB11B680BB1586870474FF0FF307047DB
:102E5000B0190020064B10B51C680CB900F042F9FF
:102E600023689B6813F4406F14BF0120002010BD3D
:102E7000B01900202DE9F843904607460C46FFF7AD
:102E8000E9FF024624B96FF080042046BDE8F883CC
:102E90006300F8D5144B04F01F0153F82150002DA6
:102EA000F1D02B6829465868FFF78EFFB0B9C4F3FC
:102EB0000721284600F0BBFA04460028E3D1EFF3CF
:102EC000108972B600F0C1F9064689F3108840B146
:102ED00042462946FFF79AFF3E60D6E76FF081042D
:102EE000D3E76FF08204D0E7C41900202DE9F04148
:102EF00000F0AAF90023134E134F73607B6000F0BB
:102F0000E5F8DFF84880304600F022F80446A8B122
:102F100039468023424600F07FF80546204600F0FF
:102F2000CBFA206804F10801FFF74EFD08B100F06C
:102F3000D9F829462046FFF775FCE4E7BDE8F041E3
:102F400000F071B9B4190020441A0020C4190020FF
:102F5000F8B5054608B900F0C5F82A4E346814F1F2
:102F6000290F4CD8284B196804F128038B4246D20C
:102F7000236AA26903EB43030C321344606AE269DB
:102F8000024402EB820213449B00E31801D29942EF
:102F900001D200F0A7F823681C4A1B0C1B049342C3
:102FA00001D000F09FF82388B3F5817F01D300F0B2
:102FB00099F86368002B01DA00F094F8144A176856
:102FC00007F124031360134A1268934201D900F0F9
:102FD00089F8236AA26903EB43030C32616A134444
:102FE000E2693C600A4402EB82021344326802EB5D
:102FF00083026B6832603B626F603846F8BD002721
:10300000FBE700BFC41000204837010000005F5FED
:10301000C0100020443701002DE9F74F0F469046BD
:103020000646009300B109B900F05CF8D6F800A09C
:10303000DAF818200AF1300303EB820BDAF81C40AF
:10304000204B1D6854B10C2202FB04541C601E4B23
:103050001B689C4201D900F045F82C4625464FF0EC
:103060000009DAF81C204A4500D91CB9002003B039
:10307000BDE8F08F142303FB09B20023C5E9002645
:103080009268AB60930516D5B8F1000F02D0009B93
:10309000802B03D0019200F025F8019A12F0E00F86
:1030A000D0B202D158F820201AB1019000F01AF8DD
:1030B000019848F820507A6809F10109AA607D60FA
:1030C0000C35CEE7BC1000204037010008B5FFF7F3
:1030D0002FFD034B9860FFF731FD80F3888808BD12
:1030E00000ED02E0FFF77CB98230012808B506D870
:1030F000FFF7B0FE18B9BDE80840FFF7F3BF08BD01
:10310000F8B506460D4600F0A4F9044608B9FFF7E5
:10311000E9FFA7680FB9FFF7E5FFE368991C20D026
:103120005A1C21D1A5B315F1820F13D102232360BC
:10313000EFF3108672B629462046FFF76BFB054673
:1031400086F310882368022B24D1204600F086F8ED
:103150002846F8BD15F1830FEAD0FFF7C3FF00251D
:10316000E6E702232360FAE7002BF6DB204600F0B7
:1031700094F93B689B689B0501D50223236015F1F8
:10318000810FD5D16369002BD2DBFFF7ABFFCFE70F
:103190003546F4E700232360DAE708B5FFF720F9A6
:1031A0006FF0830008BD2DE9F3410E46174698469F
:1031B0000546FFF74FFE00F060F92946024601A8D8
:1031C000FFF758FE044660B943463A463146019837
:1031D000FFF7A8F9044640B16B0002D5019800F052
:1031E0003DF8204602B0BDE8F0810198FFF7EAFA09
:1031F0000446F6E740F20110704770B50546FFF748
:1032000029FE06462846FFF7C9FD044608B90020F6
:1032100070BD014632462846FFF7D6FD0028F6D19C
:103220002368D868F4E76FF00200704700DF70474A
:103230004FF480507047B0F5805F03D1EFF30B80FF
:1032400080387047002070477047EFF30B8000F123
:10325000800383F30B88704700207047EFF30B83E4
:10326000803B83F30B88704770472DE9F0410E4691
:103270001546002A4AD0C4074BD480F00204C4F398
:103280004004A40003F00602062A4AD144F00104D7
:1032900022462946304602F0AFFBB8BB46E800F2B2
:1032A00005EB0608100E120208F1FF3747E800F39D
:1032B0004FEA136166D51B0264D5884262D046E8A6
:1032C00000F547E800F7FFF776F82D0E85424FEA44
:1032D000176734D3FFF771F8874230D82846FFF7D5
:1032E00065F82246C6F101010144304602F084FB34
:1032F000002847D00135AF4218D83846FFF754F8B8
:103300002246A8EB000102F077FBD8B30020BDE80D
:10331000F081EFF39484A40004F0040444F0120458
:10332000B0E7990731D544F00804B1E72846FFF724
:103330003BF80646FFF743F822460146D5E7FFF77C
:1033400046F885421ED3FFF744F887421AD828462C
:10335000FEF7AAFD2246C6F101010144304602F003
:103360004BFB78B10135AF4203D83846FFF72AF856
:10337000C6E72846FFF726F80646FFF72CF8224650
:103380000146EBE76FF07F00C1E74CF2DA20BEE7C1
:1033900010B50446FFF73EFCFFF74CFC10B143F6B6
:1033A000DA3010BDFFF786FC0028F8D1FFF748FBA4
:1033B0000028F4D102232360F3E708B5FFF7E8FB08
:1033C00010B143F6DA3008BDFFF7ECFB0028F8D166
:1033D00000F01CF80028F4D162B6FDF7F5FCFFF709
:1033E000EDFB0028EDD1FFF709FC0028EBD0E8E762
:1033F000EFF30880EFF309812DE9F00F6B46724679
:10340000FDF73AFC08B0FFF7A5FBFEE70020704788
:1034100004460D46A54628470368283383F30988E8
:10342000836883F30B88BFF36F8F4068704703682E
:103430009A68DB6812F4806F05D18B422CBF0020A4
:103440006FF0FA0070478B420CBF00206FF0FA005B
:10345000704710B5FFF7EFFE0446FFF7FDFE50B9C9
:10346000FFF7ECFCA3685B681B685B68834218BFCE
:103470000024204610BD0024FBE738B5054648B1BE
:1034800000F01BF8B5EBD07F044601D0FFF72AFE11
:10349000204638BDFFF7D2FCF4E7002310B500F159
:1034A000280252F8041F19B1C16F146C19444C6002
:1034B0000833202BF5D110BD70474FF0FF30704717
:1034C000000001464154414C204552524F523A208F
:1034D00000486172644661756C740D0A004D656D3B
:1034E0004D616E616765206661756C740D0A0042FE
:1034F00075734661756C740D0A0055736167654696
:1035000061756C740D0A005365637572654661756B
:103510006C740D0A00526573657276656420457897
:1035200063657074696F6E2000506C6174666F72B1
:103530006D2065787465726E616C20696E74657259
:103540007275707420284952516E293A200000008B
:10355000F50D010013210100711001002D0E010075
:103560003B21010047210100450E01001721010008
:10357000150E0100210E0100F90E01001D210100B0
:10358000292101002F2101001D000000100004006E
:103590001C000200110006000302020200000000ED
:1035A0000338FDD87047506C6174666F726D2045AA
:1035B0007863657074696F6E3A0D0A00416C6C2017
:1035C00070696E732068617665206265656E206340
:1035D0006F6E66696775726564206173206E6F6EC9
:1035E0002D7365637572650D0A000000000001000F
:1035F000000200000002FF002C0000003001FF006C
:10360000080000004001FF000C00000030313233A0
:103610003435363738394142434445461B5B313BEC
:1036200033346D5B536563205468726561645D205B
:1036300053656375726520696D61676520696E69A0
:103640007469616C697A696E67211B5B306D0D0A64
:10365000001B5B313B33346D426F6F74696E6720C2
:1036600054462D4D2076322E302E302D6E6373321F
:103670001B5B306D0D0A00556E6B6E6F776E2053BD
:10368000504D20535643207265717565737465649F
:103690003A2000556E6B6E6F776E20535643206E46
:1036A000756D626572207265717565737465643AD3
:1036B00020000000004000500050005000800050EA
:1036C00000A0005000B0005000E0005000F000509A
:1036D0000000015000100150004001500050015006
:1036E000007001500080015000B0015000C0015036
:1036F00000D0015000E0015000F0015000000250E5
:1037000000100250002002500030025000400250D1
:10371000006002500080025000A002500090035050
:10372000002584500080010000800100FF7F080018
:10373000007C01000080010000800800FFFF0F00F6
:103740002C1200201412002000040100FFFFFFFFD4
:10375000FFFFFFFFFFFFFFFFFFFFFFFFFFFFFFFF79
:10376000009A204B9A4208D110B502F07DFA02F07F
:10377000A9F906BC96460C46744702F0B9FA009ABD
:10378000184B9A4208D110B502F07AFA02F09AF971
:1037900006BC96460C46744702F0AAFA0CB4029A8C
:1037A000104B9A420CD14FF0004319430CBC10B59A
:1037B00000F09EF802F086F906BC96460C46744767
:1037C00002F096FA009A074B9A4202D1064908681D
:1037D000744702F08DFA009A024B9A4200D1744766
:1037E00002F086FAA5EDF5FE801000200348044B98
:1037F000834202D0034B03B118477047A811002041
:10380000A8110020000000000548064B1B1AD90F24
:1038100001EBA301491002D0034B03B118477047D5
:10382000A8110020A81100200000000010B5064CCF
:10383000237843B9FFF7DAFF044B13B10448AFF321
:1038400000800123237010BDC0180020000000007C
:10385000745F010008B5044B1BB104490448AFF381
:103860000080BDE80840CFE700000000C418002039
:10387000745F0100A3F5803A704700BF174B002B1F
:1038800008BF134B9D46FFF7F5FF00218B460F46FF
:103890001348144A121A02F0C4F90E4B002B00D040
:1038A00098470D4B002B00D09847002000210400C2
:1038B0000D000D48002802D00C48AFF3008002F044
:1038C00077F820002900FEF7F9FD02F05DF800BF4F
:1038D000000008000000000000000000F80B0020BD
:1038E000A8110020B82800200000000000000000FF
:1038F0002DE9F84304460D4616461F46EFF30583AF
:10390000C3F308030BB1FFF7EDFBDFF834903B4640
:10391000204632462946D9F80080FFF744FCD9F802
:1039200000300446984506D0DB6901461869BDE8B9
:10393000F843FFF7E5BBFFF7D7FB2046BDE8F88368
:10394000B019002001680E4A0346914215D1C169A1
:10395000A2F11022A2F1EF1291420ED18268012A47
:103960000BD8C26812B101698A4206D0586928B1E1
:103970009B691B1A5842584170470120704700BF8D
:1039800055AA00FF0D4B70B59E68A6B13046FFF7F3
:10399000D9FF044678B9F3686BB935690DB920468B
:1039A00070BD2846FFF7CEFF28B9EB68B34202D1BD
:1039B0002E462D69F2E70124F1E700BF4C1A0020E2
:1039C0002DE9F041394E3468F368D4B1B468C4B11C
:1039D000002861D000295FD001FB00F5B5FBF0F0B5
:1039E000884259D1291D57D8AA070DD025F00302C6
:1039F00004321C4603E0616891424FD2A469002C56
:103A0000F9D12046BDE8F0812A46F2E7891A232938
:103A100004F12007D4E9050C1AD80123A360A0B152
:103A2000C0F818C0A36903B158610023C4E9053385
:103A30003369DB0702D5FFF7A5FFA0BB2A460021AB
:103A400038463C4602F0EDF8DBE7C6F80CC0E9E783
:103A500002F1200804EB08032039C3E9011E2169A3
:103A6000DFF84CE0DC60196144F808E0AEF1102E9C
:103A7000AEF1EF1EC3F81CE001B1CB60C3E9050C49
:103A800040B18361996901B14B6101212361C4E9AE
:103A90000121CAE7F360F5E70024B2E7D4F808E0B3
:103AA000BEF1000FB2D0012001F06EFF4C1A0020D1
:103AB00055AA00FFF8B5054600283AD0364E3368BF
:103AC000002B36D0B268002A33D0834203D8726804
:103AD0001344984202D3012001F056FFA0F12004C4
:103AE0002046FFF72FFF0028F5D155F8183C012B91
:103AF000F1D145F8180C55E90570DFB1BB68CBB9B9
:103B000055F81C2C7B68203213447B60386100B16F
:103B1000C76020220021204602F083F8386908B1EE
:103B200083682BB333699B0703D5FFF72BFF00286E
:103B3000D1D1F8BD40B3836833BB42686368134496
:103B4000203363600369D4E90521236192B9B9B9CF
:103B5000426981696261A161A2B19461A26902B105
:103B6000546103B1DC602022002102F05AF8D9E749
:103B70003C46E2E79161A1690029E9D04A61E7E7A3
:103B8000F160F8E7F460E9E7F36845F8083C03B151
:103B90005C61F460C6E700BF4C1A002038B50D46E2
:103BA000142200210446124802F03BF81149124841
:103BB00000F02CF8232D1AD914F003031FBF043D85
:103BC000ED18C3F10403E4182A460021204602F050
:103BD00028F8074B094AC3E900459C602260A2F11E
:103BE0001022203DA2F1EF126560E261DC6038BD79
:103BF0004C1A0020B53A0100C139010055AA00FF56
:103C0000014B1B68184700BFC8100020024B18600A
:103C1000024B002019607047CC100020C810002013
:103C200010B50A46044619B1024B00211B6898479B
:103C300010BD00BFD0100020054B0A46197819B1FD
:103C40000146181D02F08EB86FF08800704700BF63
:103C5000601A002010B5074C00F032F8204602F040
:103C600092F8201F0821FFF7DBFFBDE8104002F0AB
:103C700076B800BF641A002070B50C4D2B787BB964
:103C800002F06BF8044670B90126281D6E7002F030
:103C900067F8044638B900F00BF8044618B92E70DE
:103CA0000024204670BDFFF7D5FFFAE7601A002018
:103CB0000122024B002083F880257047681A0020FB
:103CC000F8B5074C2025264601272046276202F03A
:103CD00033F8013D04F12C04F7D186F88055F8BD86
:103CE000681A002010B50C4C236813B10B4B1B68ED
:103CF0002BB900F089FC30B90122084B1A6001236E
:103D00002360002010BD0138062801D9044810BDE9
:103D1000044B53F8200010BD042000200020002098
:103D2000FE8FFFFFDC5D0100144B2DE9F0430028FE
:103D300014BF04461C46124F236883B0BB4219D0FF
:103D400016460D4620464FF4147104F1040900F0A4
:103D500047F804F58E78484600F0CEF8404600F06B
:103D600019FA2B464A4640460649009600F034FBB5
:103D700008B92760002003B0BDE8F08308200020C8
:103D8000A5BCC95A7D3F010070B50D4C1D460028E9
:103D900014BF064626460B4B306882B098420DD1C0
:103DA00006F58E70002633460096144600F03EFB62
:103DB000002818BF34462C6002B070BD0248FBE7F3
:103DC00008200020A5BCC95AE88FFFFF38B131B1E7
:103DD000002201440346013081421A70FAD1704733
:103DE00038B131B1002201440346013088421A70D3
:103DF000FAD170472DE9F043202B1D460646884630
:103E000091468BB026D8DBB202AF8DF80480B04665
:103E100058F8041B8DF8053021B9404601F038F9F7
:103E2000044640B9012302224046336001A901F053
:103E300043F9044638B138462021FFF7D1FF204628
:103E40000BB0BDE8F0832A464946404601F034F9FC
:103E50000446F0E702AF1946104600233A4601F047
:103E6000B1FA04460028E6D12023B9461D46CCE726
:103E70002DE9F041D0F8F830A6B0002BD8BF02AE43
:103E800031DD05460027D0F80C4102AEA4F101084F
:103E90009022D5F8FC403146D0F8000101AB0197E3
:103EA000B8FA88F8A0474FEA5818044620B9019B91
:103EB00053B9B8F1000F16D030469021FFF790FFAC
:103EC000204626B0BDE8F081014632462846FFF77D
:103ED00091FF58B9D5F80431019A1344C5F804315B
:103EE000B8F1000FE8D16FF03C04E5E70446204646
:103EF00026B0BDE8F08100BF70B50025044614224D
:103F000004F588762946C0F8F850FC3001F089FEA7
:103F100008222946304601F084FE144B30461B68C7
:103F20009847204640F8045B01F098F8104B304663
:103F30001B689847C8B9D4F8F830AB420FDC03EBE4
:103F4000830204EB82022021C2F800010120C2E9B1
:103F5000421008490133C2F8FC10C4F8F830064B8F
:103F60003046BDE870401B68184770BDF010002057
:103F7000EC100020614F0100E81000202DE9F0470F
:103F8000202A88B07AD83F4B00F5887904461B6810
:103F900048461746884698470546F8B940F2011644
:103FA000D4F8F830002B65D02046FFF761FF0546B6
:103FB00038B9D4F8F830002B14DC013EF2D16FF0A0
:103FC0003B056E4620213046FFF70AFF2E4B484640
:103FD0001B689847002818BF6FF01D05284608B0D9
:103FE000BDE8F087D4E94132934203D3D4F80C21E1
:103FF000012A02D0013ED7D1E1E71F2BFAD96E4644
:1040000001462022304604F1040A01F00AFE31463E
:10401000504601F07BF805460028D3D1504601F008
:1040200031F8504601F01AF82946504601F030F8B0
:1040300005460028C6D150462022314601F03CF802
:1040400005460028BED1034632462021304601F005
:10405000B9F905460028B5D1D4F8F8303A46002B16
:10406000C8BF002340463146C8BFC4F8043101F040
:10407000B3FDA7E76FF03F056E46A3E76FF03B0582
:10408000ACE700BFEC100020E810002070B590B045
:1040900000287AD03E4C0D46402236210646204666
:1040A00001F0BFFD40225C21A01801F0BAFD2B1DDC
:1040B000A34203D904F144039D4252D32B682268E2
:1040C000534023602B68226C534023646B68626802
:1040D000534063606B68626C53406364AB68A26872
:1040E0005340A360AB68A26C5340A364EB68E268E2
:1040F0005340E360EB68E26C5340E3642B69226950
:1041000053402361226D2B695340236562696B69BB
:10411000534063616B69626D53406365AB69A2692B
:104120005340A361AB69A26D5340A365EB69E2699B
:104130005340E361EB69E26D5340E3650021304693
:1041400000F0A6FF044628B940223046104900F08E
:10415000B3FF044640216846FFF742FE204610B0F8
:1041600070BD631E04F13F01013D1F3415F8010FBE
:1041700013F8012F42401A7011F8012F2878A3423A
:1041800082EA00020A70F1D1D8E76FF07304E5E724
:104190005822002010B54FF49A720021044601F015
:1041A00040FD42F21072044BC4F8202104F59670D1
:1041B0001B68BDE810401847F01000202DE9F04FB3
:1041C00004468846914695B0002900F0A780002A51
:1041D0000CBF0126022600238DF80C30002C00F0C5
:1041E0009F80DFF844A104AF0AF1400B0021204674
:1041F00000F04EFF034648B1384620210193FFF7F7
:10420000EFFD019B184615B0BDE8F08F40225146E6
:10421000204600F051FF03460028EDD104F1F405DB
:1042200020222946204600F047FF03460028E3D11C
:104230000122204603A900F03FFF03460028DBD1FE
:10424000022E62D020460CA900F060FF0346002831
:10425000D2D10146204600F01BFF03460028CBD1F7
:1042600040225946204600F027FF03460028C3D1CC
:10427000202220460CA900F01FFF03460028BBD1D6
:104280003946204600F042FF03460028B4D13946A3
:104290002046FFF7FBFE03460028ADD12022294629
:1042A000204600F009FF03460028A5D120460CA9AE
:1042B00000F02CFF034600289ED10146204600F066
:1042C000E7FE0346002897D140225946204600F0D9
:1042D000F3FE034600288FD1202220460CA900F0CF
:1042E000EBFE0346002887D12946204600F00EFF4A
:1042F0000346002880D19DF80C200132D2B2B24290
:104300008DF80C20FFF472AF76E74A46414620460E
:1043100000F0D2FE0346002894D06DE701265AE74C
:104320006FF0730304AF67E7582200202DE9F041D6
:104330000446884615461F46D0F81801E0B013B170
:1043400000EB40004008B5F5807F3ED82844B0F52A
:10435000C07F3AD84FF4C0720021684601F061FC7A
:104360006946D4F82431D4F81821D4F828019847A4
:1043700070BBD4F8186157B1D4E9493072080DEB1D
:104380000601984720BBD4F8183106EB5306B8F164
:10439000000F00D08DB9324669462046FFF70EFF68
:1043A000054610B90123C4F8143131466846FFF7B9
:1043B00017FD284660B0BDE8F0810DEB06004146D0
:1043C0002A462E4401F008FCE5E76FF00405F0E70B
:1043D0006FF00805EDE700BF2DE9F047044604F152
:1043E000F4050F4691461E46DDF8208000F036FEAB
:1043F00029462046FFF74AFE08B1BDE8F087284667
:104400002022012101F00DFCD4F81831C4F82471E8
:10441000C4F8289113B92023C4F818314246314614
:104420002046BDE8F0470123FFF780BFB2F5806F5B
:1044300000F295802DE9F04F89B09A46129BB3F5B2
:10444000807F00F29080D0F82431164604460F4653
:104450004BB3D0F81C31012B05D0D0F81421D0F883
:1044600020319A421FDD514600232046129AFFF761
:104470005DFF014698B900231293002E5ED0DFF84D
:10448000EC9009F1400B0021204600F001FE202EA7
:104490003546014628BF202504F1F40890B10846AE
:1044A00009B0BDE8F08FBAF1000FE6D0129B002BE7
:1044B000E1D051461A462046FFF780FE014600280B
:1044C000DBD0ECE749464022204600F0F5FD0146EE
:1044D0000028E4D141462022204600F0EDFD0146AF
:1044E0000028DCD16946204600F010FE0146002875
:1044F000D5D1204600F0CCFD01460028CFD1594649
:104500004022204600F0D8FD01460028C7D1694668
:104510002022204600F0D0FD01460028BFD14146B0
:10452000204600F0F3FD01460028B8D138462A465F
:10453000414601F051FB761B2F44A4D15146204641
:10454000129AFFF73BFE01460028A8D10846D4F88E
:1045500014310133C4F8143109B0BDE8F08F6FF0A5
:104560000201084670476FF0040198E758220020C6
:10457000002130B58DB0282202A8019101F051FB35
:1045800002A800F047FF044610B120460DB030BD30
:10459000174D4FF0FF31286800F042F9044620B172
:1045A000144800F0D3F9012C18D0002000F068F96D
:1045B000D0B9114A02A901A800F0C4FC04460120A8
:1045C00000F05EF960B9286800F032F90028DCD00C
:1045D0000A4800F0BBF920460DB030BD0524F2E7D3
:1045E000074800F0B3F9EEE7064800F0AFF9E0E75E
:1045F000D4100020F85D0100D8220020505E010098
:10460000305E0100105E010030B583B000F05CF850
:1046100028B100F0ABF80324204603B030BD00F011
:1046200077F8D8B900F02CF9E0B9224CD4F8283941
:104630001B0EF02B0AD1D4F8242A1F4B9A4231D0FA
:1046400000F044F8072400F091F8E5E7062400F0B4
:104650003DF800F08BF8204603B030BD042420461E
:1046600003B030BD00F032F800F080F8FFF780FFB3
:10467000044698B9114D2B68002BCDD10246014656
:10468000FFF752FB50B968220D4901ABFFF77CFBE5
:1046900020B920460B4B2B6003B030BD05242046CB
:1046A00003B030BD012000F0EBF80028DAD1C4F8E7
:1046B0000C0ADBE7001084500000E020F824002002
:1046C000FC2400205AEA5A5A002070470020704704
:1046D000430504D54FF0FF32034BC3F80821024BCA
:1046E000C3F8080A704700BF00108450014BC3F89C
:1046F000040A70470010845008B100F06BB84FF402
:104700007500704708B100F04FB84FF4750070475E
:1047100010B5114800F070F800B110BD0F4800F05E
:104720006BF80028F9D10E4C204600F065F80028FF
:10473000F3D10C4B0C481C6000F05EF801460028D9
:10474000EBD100F02DF8044608B1204610BD00F072
:1047500079F82046FAE700BFE4100020E0100020BE
:10476000DC100020D4100020D810002008B5084824
:1047700000F04CF8074800F049F8074800F046F808
:10478000064800F043F8BDE8084000F00BB800BF51
:10479000E4100020E0100020DC100020D8100020E1
:1047A00000207047704700BF024610B4084CD4F890
:1047B000003A1342FBD021B1D4F804310B60C4F8A5
:1047C0000831034B0020C3F8082A10BC704700BF13
:1047D00000108450044AD2F8003A1842FBD0C2F8C4
:1047E000080A0020704700BF0010845001F0BEB9D5
:1047F0000A46002101F015BA08B5034B02681B6890
:1048000010689847002008BD1011002008B5034B20
:1048100002685B6810689847002008BD10110020EE
:10482000024B02689B681068184700BF10110020F7
:1048300008B5034B0268DB6810689847002008BD84
:104840001011002070B5094C094D2069AB689847DC
:1048500018B1084B08485B6898470021074AEB6885
:1048600011602069BDE87040184700BFFC100020AF
:1048700010110020F4100020685E01006425002063
:10488000F8B51A4D1A4E0446B26828699047E8B93F
:10489000184F3B684CB1A3B1012B19D0013B3B60D1
:1048A0002869F36898470020F8BD43B90121124AEE
:1048B000C2F800151149D1F81029002AFBD10133A3
:1048C0003B60F368286998470020F8BD0C48F8BDA4
:1048D0000A4AD2F81039002BFBD1074A6FF07E400C
:1048E000C2F80035FFF702FF3B68D7E7FC10002055
:1048F0001011002064250020000084500010845016
:10490000E98FFFFF014B1B68184700BF1011002003
:10491000014B9B68184700BF10110020014BDB685A
:10492000184700BF10110020BFF34F8F0549064BF9
:10493000CA6802F4E0621343CB60BFF34F8F00BF3D
:10494000FDE700BF00ED00E00400FA0530B44FF0D1
:10495000FE320025074B084C08494968C3F800247B
:10496000C3F80424C3F80824C3F80C24C4F8005581
:1049700030BC08470010845000008450F410002020
:1049800010B5044650B1636813F0685F05D0064A5D
:10499000934202D000236260236010BD034B0448A1
:1049A0005B689847EFE700BF2C5F5CA9F41000201C
:1049B000885E0100C8B143680D4A934213D013F0DA
:1049C000685F0ED0012350E8002F194640E8001C14
:1049D0009CF0000FF7D1012AF5D0BFF35F8F0020C4
:1049E000704704487047044870476FF4E0407047D0
:1049F0002C5F5CA9E98FFFFFEA8FFFFF034680B1C0
:104A0000426809498A420AD012F0685F05D0BFF3B4
:104A10005F8F002210461A607047044870470448B0
:104A200070476FF4E04070472C5F5CA9E98FFFFF8F
:104A3000EA8FFFFF10B5044620B10023034A23602C
:104A4000626010BD0248FFF781FFF6E73A00003AC6
:104A5000B05E01002DE9F047002878D00C4600290F
:104A600075D01D46002B72D007461AB101220023D3
:104A70002A6003602B68002B64D02946204600F092
:104A8000B7FD804600285FD12146286800F096FDDA
:104A90008046002858D12B68082B6CD0042B6DD091
:104AA000A3F10209B9FA89F94FEA59190121354EE2
:104AB000C6F8C411C6F84011C6F8C411636AC6F836
:104AC0003031D6F830219342F6D14FF0000A4FF042
:104AD000FF30C6F82CA1FFF7FBFD6FF01B0350461B
:104AE000C6F80031FFF702FEC6F80C91D6F8040AAA
:104AF00040F48060FFF7FAFD0A23C6F83831089BBE
:104B0000012B29D02369204AA2FB03231B09626AD7
:104B1000404602FB03F303EB43031A4ADB039B0902
:104B2000C2F8D8310123C2F82C313B682A6823F03F
:104B30007F4343EA02633B602A6843EA02233B6007
:104B4000BDE8F087DFF844804046BDE8F087DFF835
:104B500040804046BDE8F0874FF47F03D3F80C2C2B
:104B6000013206D0D3F80C3C074AA2FB03231B09F1
:104B7000CDE71623CBE74FF0030997E74FF0020983
:104B800094E700BF00108450ABAAAAAA310CF10030
:104B9000350CF10058B34B1EB3F5047F27D230B566
:104BA0004FF0000ECD00744671464B0901F01F0C0A
:104BB00050F82330BCF11F0F23FA0CF306D003F09A
:104BC000010319B901211C468E46EEE79C4201F112
:104BD000010106D01C464FF0010EA942E5D100208C
:104BE00030BD0EF1010E9645F7D1024830BD0148A7
:104BF000704700BF360CF100C0B32DE9F0434C1EE6
:104C0000B4F5047F1DD2E3B1DAB100252E46A846E3
:104C10002C46CF0003F1FF394FEA541C04F01F0E5D
:104C200050F82C10BEF11F0F21FA0EFC0CD00CF026
:104C3000010C4CB90126E04634463546ECE7964275
:104C400016D90C48BDE8F083AB420BD0C44508BF71
:104C50000136A945F3D001350134BC42DCD1002036
:104C6000BDE8F0830125E0462E46F5E70148704790
:104C70001D46F1E7370CF1002DE9F04F91B0834666
:104C8000DDE91B460D46002E6ED10F691C60002326
:104C90001A990B60002A00F02F819D4B6A6AD3F8A5
:104CA0003811D3F830319A4269D10A2967D19BF87B
:104CB0000330089304F10803079304230593954BED
:104CC000934CA3FB07239B0803EB4303A7EB43038E
:104CD000039306971A9B069E1E60002E00F0EA8042
:104CE00000F096FC00230993BBF1000F00F0D58083
:104CF00098464FF0010ADDF81C90002D00F0CD80A1
:104D0000089B002B3DD0284608A900F071FC002824
:104D100039D0814B984220D0089B082B00F0E480CA
:104D200000225B000893294608AB58460092FFF723
:104D300091FE7A4B984200F0D38070B9DBF80020E6
:104D4000130A03F47F03134323F07F43CBF80030AF
:104D5000059B013B0593BDD10020039000F058FC5A
:104D6000039811B0BDE8F08F4FF47F01D1F80C0C1F
:104D700001300CBF4FF40477D1F80C7C86E768480B
:104D8000EBE76648C5E72946089800F017FC0028BD
:104D9000BFD1089B082B00F0A980042B00F0A9804C
:104DA000A3F10203B3FA83F35B090493C4F8C4A12B
:104DB000C4F840A1C4F8C4A16B6AC4F83031D4F877
:104DC00030219342F6D100234FF0FF30C4F82C314C
:104DD000FFF77EFC002318466FF01B03C4F8003178
:104DE000FFF784FC049B4B4FC4F80C31D4F8040A41
:104DF00040F48060FFF77AFC0A23C4F838312B694D
:104E000009A8A7FB03236A6A1B0902FB03F303EB50
:104E10004303DB039B09C4F8D831C4F82CA1DBF8A9
:104E20000030089923F07F420B0243EA01631343E9
:104E3000CBF8003000F0B2FB099B03F01A030343E8
:104E40007FF46AAFA7FB0637D4F81431B8EB970F9D
:104E50000A93D4F818310B93D4F81C310C93D4F87E
:104E600020310D93D4F824310E93D4F828310F93C8
:104E700001D1039B9BB9484618220AA9183EFFF7A7
:104E8000B5FC09F1180908F101089EB100F0C0FB5A
:104E900000230993002D7FF433AF224839E74846B9
:104EA0001A46F61A0AA9994408F10108FFF79EFC70
:104EB000002EEBD1069F079E6A6939463046FFF700
:104EC00069FEAA6940B94FF4806339463046FFF75E
:104ED00093FE00283FF440AF00231A9A136018E7AE
:104EE0002B6A002B3FF439AF0F4836E703230493B6
:104EF0005CE70223049359E70122294658460096AD
:104F000008ABFFF7A7FD00283FF4D4AE25E700BFAC
:104F100000108450ABAAAAAA020CF100310CF100D7
:104F2000300CF100350CF100320CF10010B4DDE969
:104F3000013401940024DDF80CC0CDE902C410BC9A
:104F4000FFF79ABE30B51546012487B005AB009334
:104F50000022CDE9015404ABFFF78EFE07B030BD4F
:104F6000F0B587B0002966D01E46002B63D01446EA
:104F7000002A60D0314F0D4638684FF0FF31FFF7FF
:104F80004FFC00284DD10020FFF77AFC002844D1C7
:104F90002B4800F03FFAD8B101204FF0FF35FFF762
:104FA0006FFC002835D14FF408712648FEF70EFF3C
:104FB00004212548FEF70AFF21482821FEF706FFB5
:104FC0003868FFF735FC00282FD1284607B0F0BD20
:104FD0001C4A0346029205AA019204AA0390009279
:104FE000174902461848FFF7A1FF03460028D3D10E
:104FF00028461D46059B22469C4228BF1A46049916
:1050000032600831FFF7F2FB0120FFF739FC00287E
:10501000C9D00E48FFF79AFCC5E70D48FFF796FC8C
:10502000B6E70C48FFF792FCADE70B48FFF78EFCA4
:10503000284607B0F0BD4FF0FF35C6E7D41000207A
:105040007C250020A425002078250020305E01006A
:10505000105E0100F85D0100D45E010010B5044649
:1050600028B12046BDE81040F421FFF7C1BB044839
:10507000FFF76CFC2046BDE81040F421FFF7B8BBF9
:10508000EC5E010010B1F421FEF7A0BE704700BF36
:1050900008B521B1012908D06FF0360008BD012103
:1050A00000F058F80028F7D108BD022100F052F8AE
:1050B0000028F9D0F0E700BF30B505468818B0F5F4
:1050C000801F0B461446A1B001D8802A0CD9B3F535
:1050D000801F17D922461946284600F07DF804465D
:1050E00084B9204621B030BD6846FFF77FFB2246D9
:1050F0006946284600F070F8802104466846FFF7AC
:1051000077FBEDE76FF03604EBE700BF70B5E8B171
:105110000E46D9B1044600F031F80546B0B923680F
:10512000012B0BD0022B01D0284670BD1C2230462B
:1051300004F10801FFF75AFB284670BD20223046D3
:1051400004F10801FFF752FB284670BD6FF03605E9
:10515000EAE700BF78B138B50D46F0210446FFF705
:1051600047FB402320462560E36500F091FA0038B4
:1051700018BF012038BD0120704700BFF0B5056E93
:10518000A5B0044604AEE5B90023012701933046DB
:105190006760294602AA009300F046FA10B1012088
:1051A00025B0F0BD2A46204602A900F099FA002851
:1051B000F5D1204600F0AAFB0028F0D1206625B0EA
:1051C000F0BD802D2A46304628BF802204F16401BC
:1051D000FFF70CFB256ED7E7002800F0AE802DE925
:1051E000F04F1446A5B0002A3DD00F46002949D003
:1051F000B2F5803F0546006E20D34FF6FF7805F1EB
:10520000640AEB6D1A1AB2FBF3F103FB1122002AB8
:1052100065D18342B9464FF6FF7672D0B6FBF3FBF9
:1052200003FB0BFBBBF1000F30D1002E45D1A4F5E1
:105230007F44FF3CB4F5803F4744E2D2EA6D161A42
:10524000B6FBF2F302FB1366A64228BF2646002EE9
:1052500075D1824200F08D80B4FBF2F602FB06F6B7
:105260002EB9002C79D1002025B0BDE8F08F0023A5
:1052700031463846CDE9003302AA00F0D5F90028BE
:1052800000F09580012025B0BDE8F08F002359463D
:105290004846CDE9003302AA00F0C6F90028F1D152
:1052A0005A46284602A900F01BFA0028EAD1A6EBCC
:1052B0000B06286ED944002EB9D019304946324623
:1052C00005EB8000FFF792FAA4F57F44286EFF3CBF
:1052D0003044B4F5803F4744286692D2AEE7424559
:1052E00028BF4246164639465044FFF77FFA286EDB
:1052F000EB6D3044834207EB06092866A8EB0606EF
:105300008CD1802B28BF802351461A4604A8FFF772
:105310006DFA0023E96D02AACDE9003304A800F07C
:1053200083F90028AED12846EA6D02A900F0D8F929
:105330000028A7D1EB6D286670E70120704705F1C2
:105340006403394632461844FFF750FA286EEA6D76
:105350003044A41B374428667BE72B6E2246193362
:1053600005EB83003946FFF741FA2B6E23442B6689
:1053700079E7802A28BF802205F1640104A8FFF79D
:1053800035FA0023E96D04A8CDE9003302AA00F044
:105390004BF900287FF476AF2846EA6D02A900F0A9
:1053A0009FF900287FF46EAFEA6D286654E7324615
:1053B000284602A900F094F900287FF463AF37442F
:1053C000A41B4EE7F8B51C460546114816460F4685
:1053D000FFF744FE21460E48FFF75AFE044620B16F
:1053E0000B48FFF74FFE2046F8BD3A4629460848CD
:1053F000FFF762FE04460028F2D131460448FFF769
:1054000085FE04460248FFF73DFE2046F8BD00BF7A
:10541000C42700201C2370B582B001A90546019362
:1054200000F032F8044638B9019B1C2B07D0144C0D
:105430001C212846FFF7DCF9204602B070BDD5E9F3
:105440000112131E18BF0123003918BF01210126C4
:1054500028689B00EA6843EA4103002818BF43F02C
:105460000103EE612AB9C5E90834002BE4D1054CEB
:10547000DEE7204643F00803C5E9083402B070BDFA
:10548000370CF0000E0CF0000346002866D000290F
:1054900064D00A681C2A61D14FF47F023B49D2F8DC
:1054A000100C88425CD0D2F8101C013158D0D2F8D0
:1054B000101C4FF47F021960D2F8140C3449884252
:1054C00060D0D2F8141C01315CD0D2F8141C4FF417
:1054D0007F025960D2F8181C11F5947F4FD0D2F892
:1054E000181C01314BD0D2F8181C4FF47F02996080
:1054F000D2F81C0C274988423ED0D2F81C1C01313E
:105500003AD0D2F81C1C4FF47F02D960D2F8001CAC
:1055100070312FD0D2F8001C01312BD0D2F8001CF2
:105520004FF47F021961D2F8041CAF3120D0D2F8B9
:10553000041C01311CD0D2F8041C4FF47F025961C5
:10554000D2F8080C144988420DD0D2F8081C013159
:1055500009D0D2F8082C00209A61704701207047CA
:1055600040F6FC01A5E740F2373200209A6170470F
:105570005121E2E79021D3E742F60411C3E740F658
:10558000D861B2E742F2D001A1E700BFFCF8FFFF0B
:10559000D020FFFF0429FFFF37F3FFFF014608B5C6
:1055A0004FF48060FFF7AEF80022034BC3F8C82128
:1055B000C3F82C2108BD00BF001084500138072813
:1055C00005D8DFE800F0100E040A040404060748BA
:1055D0007047CB6800204B6270478B6800204B629D
:1055E00070474B68F6E70B68F4E700BF310CF10039
:1055F0000B6802E0082B0B6006D8026A13424FEAE0
:105600004303F7D00020704700487047310CF10089
:105610000022044B4FF48060C3F82C21C3F8C4214E
:10562000FFF756B800108450F0B5002483B0B0F1F5
:10563000005F8DF8074025D38C468444BCF1804F31
:1056400004461FD817461D4601220DF1070300F03E
:1056500097F90646B0B99DF80730099A3C603B714E
:1056600092B14DB10246089928460DF1070300F0AA
:1056700087F938B99DF807303046099A15601371DB
:1056800003B0F0BD4FF47506304603B0F0BD00BF67
:10569000D8B108B50368012B04D0022B0FD043B159
:1056A0000B4808BD20220B490830FFF79FF8002067
:1056B00008BD142208490830FFF798F8F7E72022C0
:1056C00006490830FFF792F8F1E74FF4730070478E
:1056D0000100F300FC5E01003C5F01001C5F010063
:1056E0002DE9F843002900F0F9800446002800F075
:1056F000F98003680F469046002B00F0C380013B01
:10570000012B00F2D7804FF0FF3178484FF00209AB
:10571000FFF786F8002840F0BF800020FFF7B0F8C0
:105720000646002840F0C280714AD2F81C39002B8E
:10573000FBD16F4DD5F8203C002BFBD14FF0FF3053
:10574000FEF7C6FFD5F8040A20F04000FEF7CEFFB2
:1057500001230722C5F81838C5F80029C5F8C43751
:10576000A36CC5F8CC37E36CC5F8D037C5F8C09743
:1057700023685BB1013B012B18D8636AC5F85C361E
:10578000236AC5F85836E369C5F85436A269584B00
:10579000C3F850266269C3F84C262269C3F848262C
:1057A000E268C3F84426A268C3F84026504AD2F8FB
:1057B0001039002BFBD1B8F1000F5FD06368402097
:1057C000012B08BFC2F884363A68494BC3F8282C2D
:1057D000C3F82C8CFEF790FF0646454AD2F81039E4
:1057E000002BFBD1424AD2F8203C002BFBD123688E
:1057F0005BB1013B012B18D8D2F85C366362D2F85A
:1058000058362362D2F85436E361394BD3F8502628
:10581000A261D3F84C266261D3F848262261D3F8FE
:105820004426E260D3F84036A36000230121304AC9
:10583000D2F8CC07A064D2F8D007E064C2F8C4174D
:10584000C2F88436C2F8C837D2F81039002BFBD121
:10585000C2F81838002E3BD1254BD3F8040A40F08B
:105860004000FEF743FF0120FFF70AF860BB1F4826
:10587000FEF7DEFF10BB3046BDE8F8830423C2F814
:10588000C837AAE74FF0FF3118484FF00109FEF77B
:10589000C7FF00283FF441AF1648FFF757F8002034
:1058A000FEF7EEFF064600283FF43EAF1248FFF732
:1058B0004DF839E7114E3046BDE8F8831048FFF740
:1058C00045F83046BDE8F8830E48FFF73FF8CEE7CD
:1058D000102104F10800FEF78BFFBDE70A4E3046A9
:1058E000BDE8F8834FF47306C5E700BFE41000205D
:1058F00000108450F85D0100105E01000100F3000B
:10590000505E0100305E01000300F300A0B30346C7
:1059100070B4D0E90240D3E9041226BA05BA0CBA31
:1059200010BAC3E90440D3E90612986A09BAC3E978
:10593000026512BA996100BAD3E9084125BA0CBAD6
:10594000C3E90725D3E90B12C3E9094009BAD86BAB
:1059500012BAD962D3E90D4125BAC3E90C250CBAB4
:1059600000BAD3E9101209BA12BAC3E90E40196499
:1059700000205A6470BC70474FF47300704700BF3A
:1059800000201870704700BF08B5074B044613B1DC
:105990000021AFF30080054B1868836A03B1984774
:1059A000204600F08DF800BF00000000505F0100AD
:1059B00070B50D4D00260D4C641BA410A64209D1F4
:1059C0000B4D00260B4C00F0FDF9641BA410A64201
:1059D00005D170BD55F8043B01369847EEE755F800
:1059E000043B01369847F2E7A0110020A0110020E7
:1059F000A0110020A4110020431810B501D21F2AC5
:105A000001D9002010BD013902F014030144102B0C
:105A100080EA01043CD009DC8BB1042BF1D11F2CAE
:105A200040E840F315D941E840F10EE0142BE8D1ED
:105A30001F2C40E8C0F30CD941E8C0F105E01F2C51
:105A400040E800F305D941E800F11C460B468C42C2
:105A5000D7D122F01402013A0A2AD2D801A151F872
:105A600022F000BFB35A0100AD5A01009F5A010055
:105A7000035A0100035A0100035A0100035A0100AE
:105A8000B95A0100B35A0100A75A01009F5A0100F8
:105A90001F2C40E880F3DCD941E880F1D5E713F40E
:105AA000001FAFD1ADE713F4801FFAE75B02A9D561
:105AB000A7E713F4002FF4E713F4802FF1E700BFFA
:105AC000FEE700BF002383F300887047FDF70ABBA1
:105AD000EFF30880EFF309812DE9F00F6B46724672
:105AE000FBF7CAF808B0FFF7F1FFFEE7FDF7FABAD7
:105AF000EFF30880EFF309812DE9F00F6B46724652
:105B0000FBF7BAF808B0FFF7F1FFFEE7FDF7EABAD6
:105B1000EFF30880EFF309812DE9F00F6B46724631
:105B2000FBF7AAF808B0FFF7F1FFFEE7FDF7DABAD6
:105B3000EFF30880EFF309812DE9F00F6B46724611
:105B4000FBF79AF808B0FFF7F1FFFEE7FDF7CABAD6
:105B5000EFF30880EFF309812DE9F00F6B467246F1
:105B6000FBF78AF808B0FFF7F1FFFEE7814270B457
:105B70000546144602D370BC00F02EB882182144AA
:105B80003CB141EA020313F003030FD1E0180328EC
:105B900012D86FF00300A3084343002019441A44AD
:105BA0002344984210D1284670BC704711F8013D3B
:105BB000013C02F8013DE3E7581850F8046C9818CE
:105BC00040F8046C043BE1E70C1A14F8016C141A59
:105BD00004F8016C0130E4E770B504463AB141EADB
:105BE000040313F003030CD1D518032D0FD822F0B2
:105BF00003031C441944002302F0030293420CD116
:105C000070BD11F8013B013A04F8013BE6E7CD1AFB
:105C10002E68E51A2E60043BE6E75D5CE55401332F
:105C2000ECE7F0B5044662B922F00303234402F026
:105C300003021A44934214D1F0BD04F8011B013A47
:105C4000F1E7A307F9D115460B0443EA01630B43BF
:105C500043EA01231619032DE6D9771B3B60043D67
:105C6000F9E703F8011BE5E708B5EFF30583C3F394
:105C700008030BB1FDF736FABDE80840FDF7BABAE4
:105C800010B50446EFF30583C3F308030BB1FDF72A
:105C900029FA2046BDE81040FDF7AFBA2DE9F041E2
:105CA00004460D4616461F46EFF30583C3F308036B
:105CB0000BB1FDF717FA3B46324629462046BDE8B0
:105CC000F041FCF7E5BC2DE9F04104460D461646CF
:105CD0001F46EFF30583C3F308030BB1FDF702FA88
:105CE0003B46324629462046BDE8F041FCF70ABD56
:105CF00008B5EFF30583C3F308030BB1FDF7F2F921
:105D0000BDE80840FDF749BA00207047704710B55C
:105D1000044608B1FDF784FF2046BDE81040FDF7BA
:105D20006FBF10B50446406A10B1A16AFFF7EFFFDC
:105D30000020C4E9090010BD38B50446FFF7F1FFA3
:105D4000236A2C22012B0CBF05466FF0960500211B
:105D50002046FFF766FF284638BD00207047704791
:105D60000020704713B5002001AB1446FEF70CF875
:105D700030B9019BA34218BF6FF0930002B010BD71
:105D80006FF09200FAE7002070472DE9E04F2746B8
:105D9000A046A146A246A346A446A2B02DEC000A06
:105DA00084F3008825462646A447EFF3148515F0B2
:105DB000080F18BFB0EE400A3DEC000A22B0BDE863
:105DC000E08F0000F8B500BFF8BC08BC9E467047E5
:105DD000F8B500BFF8BC08BC9E467047FF8FFFFFB8
:105DE000FF8FFFFFFE8FFFFFFE8FFFFFFD8FFFFF87
:105DF000FC8FFFFFFC8FFFFF4661696C20746F20F2
:105E000061637175697265206D757465780A00004B
:105E10004661696C20746F20696E63726561736599
:105E200020504D20636F756E7465720A000000008B
:105E30004661696C20746F20646563726561736587
:105E400020504D20636F756E7465720A000000006B
:105E50004661696C20746F2072656C6561736520A2
:105E60006D757465780A0000436F756C64206E6F01
:105E700074206C6F636B20706F776572207361762E
:105E800065206D75746578006D757465785F6672F0
:105E900065652063616C6C65642077697468204E69
:105EA000554C4C20706172616D6574657200000024
:105EB00043616E277420696E697469616C697A65E3
:105EC000206D757465782C20776173204E554C4C8D
:105ED0000D0A00004661696C20746F20756E6C6F4E
:105EE000636B206D757465780A0000000A6374782E
:105EF000206973204E554C4C0A00000067E6096A81
:105F000085AE67BB72F36E3C3AF54FA57F520E51DA
:105F10008C68059BABD9831F19CDE05BD89E05C16A
:105F200007D57C3617DD703039590EF7310BC0FFBD
:105F300011155868A78FF964A44FFABE012345676D
:105F400089ABCDEFFEDCBA9876543210F0E1D2C3C3
:105F50004011002054464D5F43525950544F005455
:105F6000464D5F504C4154464F524D5F534552563B
:105F70004943450000000000000000000000000050
:105F8000FFFFFFFFFFFFFFFFFFFFFFFFFFFFFFFF21
:105F9000FFFFFFFFFFFFFFFFFFFFFFFFFFFFFFFF11
:105FA000FFFFFFFFFFFFFFFFFFFFFFFFFFFFFFFF01
:105FB000FFFFFFFFFFFFFFFFFFFFFFFFFFFFFFFFF1
:107C00007FE97FE9FBF7ACBD7FE97FE9FBF7B7BD13
:107C10007FE97FE9FBF7DFBD7FE97FE9FBF7D2BDB5
:107C20007FE97FE9FBF7BABD00000000000000001B
:107C30000000000000000000000000000000000044
:107C40007AFFFFFF0090005000000000883501001F
:107C50000400000000000000000000000000000020
:107C6000000000000000000090ED00E000A00350C4
:107C70007FA60350009000506F9500501412002012
:107C8000A8110020440301000D5D0100095D010001
:107C9000235C0100DC1000200C11002004110020E6
:107CA00000110020FC1000201D49010011490100B5
:107CB0000549010000000000294901003811002099
:107CC00030110020281100200000000020110020A9
:107CD000354A010081490100B5490100FD49010013
:107CE000682500203A00003A6C2500203A00003A4E
:107CF000702500203A00003A742500203A00003A2E
:107D00000000000000000000000000000000000073
:107D10000000000000000000000000000000000063
:107D20000000000000000000000000000000000053
:107D30000000000000000000000000000000000043
:107D40000000000000000000000000000000000033
:107D50000000000000000000000000000000000023
:107D6000553801002D380100FFFFFFFFFFFFFFFF27
:107D7000FFFFFFFFFFFFFFFFFFFFFFFFFFFFFFFF13
:107D8000FFFFFFFFFFFFFFFFFFFFFFFFFFFFFFFF03
:107D9000FFFFFFFFFFFFFFFFFFFFFFFFFFFFFFFFF3
:107DA000FFFFFFFFFFFFFFFFFFFFFFFFFFFFFFFFE3
:108000007804012041BF0100697902002DBF010001
:108010002DBF01002DBF01002DBF01002DBF0100AC
:10802000000000000000000000000000F9C0010096
:108030002DBF010000000000B1C001002DBF0100F4
:108040007DC201007DC201007DC201007DC2010030
:108050007DC201007DC201007DC201007DC2010020
:108060007DC201007DC201007DC201007DC2010010
:108070007DC201007DC201007DC201007DC2010000
:108080007DC201007DC201007DC201007DC20100F0
:108090007DC201007DC201007DC201007DC20100E0
:1080A0007DC201007DC201007DC201007DC20100D0
:1080B0007DC201007DC201007DC201007DC20100C0
:1080C0007DC201007DC201007DC201007DC20100B0
:1080D0007DC201007DC201007DC201007DC20100A0
:1080E0007DC201007DC201007DC201007DC2010090
:1080F0007DC201007DC201007DC201007DC2010080
:108100007DC201007DC201007DC201007DC201006F
:108110007DC201007DC201007DC201007DC201005F
:108120007DC201007DC201007DC201007DC201004F
:108130007DC201007DC201007DC201007DC201003F
:108140007DC20100FFFFFFFF4FF0FF0C1CEAD05281
:108150001EBF1CEAD15392EA0C0F93EA0C0F6FD0AA
:108160001A4480EA010C400218BF5FEA41211ED088
:108170004FF0006343EA501043EA5111A0FB013174
:108180000CF00040B1F5000F3EBF490041EAD37149
:108190005B0040EA010062F17F02FD2A1DD8B3F1C5
:1081A000004F40EBC25008BF20F00100704790F034
:1081B000000F0CF0004C08BF49024CEA502040EA86
:1081C00051207F3AC2BFD2F1FF0340EAC25070474C
:1081D00040F400004FF00003013A5DDC12F1190F8A
:1081E000DCBF00F000407047C2F10002410021FAFC
:1081F00002F1C2F1200200FA02FC5FEA310040F114
:10820000000053EA4C0308BF20EADC70704792F08C
:10821000000F00F0004C02BF400010F4000F013AC4
:10822000F9D040EA0C0093F0000F01F0004C02BFBF
:10823000490011F4000F013BF9D041EA0C018FE72E
:108240000CEAD15392EA0C0F18BF93EA0C0F0AD034
:1082500030F0004C18BF31F0004CD8D180EA01005A
:1082600000F00040704790F0000F17BF90F0004FF3
:10827000084691F0000F91F0004F14D092EA0C0FD5
:1082800001D142020FD193EA0C0F03D14B0218BF68
:10829000084608D180EA010000F0004040F0FE40AE
:1082A00040F40000704740F0FE4040F4400070474A
:1082B00081F0004102E000BF83F0004330B54FEA97
:1082C00041044FEA430594EA050F08BF90EA020F04
:1082D0001FBF54EA000C55EA020C7FEA645C7FEA97
:1082E000655C00F0E2804FEA5454D4EB5555B8BFBA
:1082F0006D420CDD2C4480EA020281EA030382EA2B
:10830000000083EA010180EA020281EA0303362DBC
:1083100088BF30BD11F0004F4FEA01314FF4801C8F
:108320004CEA113102D0404261EB410113F0004FA1
:108330004FEA03334CEA133302D0524263EB430358
:1083400094EA050F00F0A780A4F10104D5F1200EF6
:108350000DDB02FA0EFC22FA05F2801841F1000151
:1083600003FA0EF2801843FA05F359410EE0A5F125
:1083700020050EF1200E012A03FA0EFC28BF4CF056
:10838000020C43FA05F3C01851EBE37101F000450C
:1083900007D54FF0000EDCF1000C7EEB00006EEB19
:1083A0000101B1F5801F1BD3B1F5001F0CD34908A3
:1083B0005FEA30004FEA3C0C04F101044FEA4452FA
:1083C00012F5800F80F09A80BCF1004F08BF5FEA81
:1083D000500C50F1000041EB045141EA050130BD61
:1083E0005FEA4C0C404141EB0101013C28BFB1F573
:1083F000801FE9D291F0000F04BF01460020B1FABE
:1084000081F308BF2033A3F10B03B3F120020CDA90
:108410000C3208DD02F1140CC2F10C0201FA0CF06E
:1084200021FA02F10CE002F11402D8BFC2F1200CD3
:1084300001FA02F120FA0CFCDCBF41EA0C01904089
:10844000E41AA2BF01EB0451294330BD6FEA0404D2
:108450001F3C1CDA0C340EDC04F11404C4F12002BD
:1084600020FA04F001FA02F340EA030021FA04F3CF
:1084700045EA030130BDC4F10C04C4F1200220FA26
:1084800002F001FA04F340EA0300294630BD21FA64
:1084900004F0294630BD94F0000F83F4801306BF2A
:1084A00081F480110134013D4EE77FEA645C18BF1E
:1084B0007FEA655C29D094EA050F08BF90EA020FB5
:1084C00005D054EA000C04BF1946104630BD91EAAD
:1084D000030F1EBF0021002030BD5FEA545C05D1B0
:1084E0004000494128BF41F0004130BD14F58004EF
:1084F0003CBF01F5801130BD01F0004545F0FE4163
:1085000041F470014FF0000030BD7FEA645C1ABF97
:10851000194610467FEA655C1CBF0B46024650EACE
:10852000013406BF52EA033591EA030F41F40021FA
:1085300030BD00BF90F0000F04BF0021704730B580
:108540004FF4806404F132044FF000054FF0000155
:1085500050E700BF90F0000F04BF0021704730B516
:108560004FF4806404F1320410F0004548BF4042EB
:108570004FF000013EE700BF42004FEAE2014FEA40
:1085800031014FEA02701FBF12F07F4393F07F4F1B
:1085900081F06051704732F07F4208BF704793F01E
:1085A0007F4F04BF41F40021704730B54FF4607431
:1085B00001F0004521F000411CE700BF50EA010234
:1085C00008BF704730B54FF000050AE050EA0102DD
:1085D00008BF704730B511F0004502D5404261EB4D
:1085E00041014FF4806404F132045FEA915C3FF48E
:1085F000D8AE4FF003025FEADC0C18BF03325FEA2B
:10860000DC0C18BF033202EBDC02C2F1200300FADB
:1086100003FC20FA02F001FA03FE40EA0E0021FA00
:1086200002F11444BDE600BF70B54FF0FF0C4CF4EE
:10863000E06C1CEA11541DBF1CEA135594EA0C0FA0
:1086400095EA0C0F00F0DEF82C4481EA030621EADB
:108650004C5123EA4C5350EA013518BF52EA033516
:1086600041F4801143F4801338D0A0FB02CE4FF0C8
:108670000005E1FB02E506F00042E0FB03E54FF0F8
:108680000006E1FB03569CF0000F18BF4EF0010EF0
:10869000A4F1FF04B6F5007F64F5407404D25FEAEC
:1086A0004E0E6D4146EB060642EAC62141EA55519F
:1086B0004FEAC52040EA5E504FEACE2EB4F1FD0CE1
:1086C00088BFBCF5E06F1ED8BEF1004F08BF5FEA5F
:1086D000500E50F1000041EB045170BD06F0004611
:1086E00046EA010140EA020081EA0301B4EB5C04BE
:1086F000C2BFD4EB0C0541EA045170BD41F48011B6
:108700004FF0000E013C00F3AB8014F1360FDEBFDA
:10871000002001F0004170BDC4F10004203C35DAB6
:108720000C341BDC04F11404C4F1200500FA05F339
:1087300020FA04F001FA05F240EA020001F00042DA
:1087400021F0004110EBD37021FA04F642EB060150
:108750005EEA430E08BF20EAD37070BDC4F10C047A
:10876000C4F1200500FA04F320FA05F001FA04F23E
:1087700040EA020001F0004110EBD37041F100012A
:108780005EEA430E08BF20EAD37070BDC4F1200535
:1087900000FA05F24EEA020E20FA04F301FA05F29D
:1087A00043EA020321FA04F001F0004121FA04F245
:1087B00020EA020000EBD3705EEA430E08BF20EA15
:1087C000D37070BD94F0000F0FD101F0004640004F
:1087D00041EB010111F4801F08BF013CF7D041EAD1
:1087E000060195F0000F18BF704703F000465200D5
:1087F00043EB030313F4801F08BF013DF7D043EAA6
:108800000603704794EA0C0F0CEA135518BF95EA5B
:108810000C0F0CD050EA410618BF52EA4306D1D1E2
:1088200081EA030101F000414FF0000070BD50EA01
:10883000410606BF1046194652EA430619D094EA8B
:108840000C0F02D150EA013613D195EA0C0F05D175
:1088500052EA03361CBF104619460AD181EA0301C9
:1088600001F0004141F0FE4141F470014FF0000081
:1088700070BD41F0FE4141F4780170BD70B54FF01C
:10888000FF0C4CF4E06C1CEA11541DBF1CEA13559C
:1088900094EA0C0F95EA0C0F00F0A7F8A4EB05047E
:1088A00081EA030E52EA03354FEA013100F0888075
:1088B0004FEA03334FF0805545EA131343EA12633E
:1088C0004FEA022245EA111545EA10654FEA0026F3
:1088D0000EF000419D4208BF964244F1FD0404F5AC
:1088E000407402D25B084FEA3202B61A65EB030508
:1088F0005B084FEA32024FF480104FF4002CB6EBC5
:10890000020E75EB030E22BFB61A754640EA0C0044
:108910005B084FEA3202B6EB020E75EB030E22BF84
:10892000B61A754640EA5C005B084FEA3202B6EBC5
:10893000020E75EB030E22BFB61A754640EA9C0084
:108940005B084FEA3202B6EB020E75EB030E22BF54
:10895000B61A754640EADC0055EA060E18D04FEA12
:10896000051545EA16754FEA06164FEAC30343EAB2
:1089700052734FEAC2025FEA1C1CC0D111F4801F7F
:108980000BD141EA00014FF000004FF0004CB6E778
:1089900011F4801F04BF01430020B4F1FD0C88BF17
:1089A000BCF5E06F3FF6AFAEB5EB030C04BFB6EB22
:1089B000020C5FEA500C50F1000041EB045170BD15
:1089C0000EF0004E4EEA113114EB5C04C2BFD4EB42
:1089D0000C0541EA045170BD41F480114FF0000EC6
:1089E000013C90E645EA060E8DE60CEA135594EA42
:1089F0000C0F08BF95EA0C0F3FF43BAF94EA0C0F45
:108A00000AD150EA01347FF434AF95EA0C0F7FF4B9
:108A100025AF104619462CE795EA0C0F06D152EA0D
:108A200003353FF4FDAE1046194622E750EA4106F1
:108A300018BF52EA43067FF4C5AE50EA41047FF402
:108A40000DAF52EA43057FF4EBAE12E74FEA410265
:108A5000B2F1E04324BFB3F5001CDCF1FE5C0DD99C
:108A600001F0004C4FEAC0024CEA5070B2F1004FE6
:108A700040EB830008BF20F00100704711F0804FE9
:108A800021D113F13872BCBF01F00040704741F4AE
:108A900080114FEA5252C2F11802C2F1200C10FAB2
:108AA0000CF320FA02F018BF40F001004FEAC12396
:108AB0004FEAD32303FA0CFC40EA0C0023FA02F33A
:108AC0004FEA4303CCE77FEA625307D150EA013310
:108AD0001EBF4FF0FE4040F44000704701F00040E0
:108AE00040F0FE4040F40000704700BF80F00040BE
:108AF00002E000BF81F0004142001FBF5FEA410376
:108B000092EA030F7FEA226C7FEA236C6AD04FEA75
:108B10001262D2EB1363C1BFD218414048404140BA
:108B2000B8BF5B42192B88BF704710F0004F40F46C
:108B3000000020F07F4018BF404211F0004F41F488
:108B4000000121F07F4118BF494292EA030F3FD054
:108B5000A2F1010241FA03FC10EB0C00C3F1200367
:108B600001FA03F100F0004302D5494260EB4000F6
:108B7000B0F5000F13D3B0F1807F06D340084FEA61
:108B8000310102F10102FE2A51D2B1F1004F40EB56
:108B9000C25008BF20F0010040EA030070474900BE
:108BA00040EB0000013A28BFB0F5000FEDD2B0FA5B
:108BB00080FCACF1080CB2EB0C0200FA0CF0AABF7E
:108BC00000EBC25052421843BCBFD040184370471C
:108BD00092F0000F81F4000106BF80F40000013222
:108BE000013BB5E74FEA41037FEA226C18BF7FEAF9
:108BF000236C21D092EA030F04D092F0000F08BF3B
:108C00000846704790EA010F1CBF0020704712F021
:108C10007F4F04D1400028BF40F00040704712F160
:108C200000723CBF00F50000704700F0004343F0C5
:108C3000FE4040F4000070477FEA226216BF0846FB
:108C40007FEA23630146420206BF5FEA412390EABE
:108C5000010F40F4800070474FF0000304E000BFB4
:108C600010F0004348BF40425FEA000C08BF704765
:108C700043F0964301464FF000001CE050EA010229
:108C800008BF70474FF000030AE000BF50EA01023E
:108C900008BF704711F0004302D5404261EB41012B
:108CA0005FEA010C02BF84460146002043F0B64350
:108CB00008BFA3F18053A3F50003BCFA8CF2083A75
:108CC000A3EBC25310DB01FA02FC634400FA02FC7E
:108CD000C2F12002BCF1004F20FA02F243EB020085
:108CE00008BF20F00100704702F1200201FA02FCE7
:108CF000C2F1200250EA4C0021FA02F243EB0200DA
:108D000008BF20EADC7070477BB972B90029BEBF8A
:108D100000204FF0004106E008BF00281CBF6FF0A4
:108D200000414FF0FF3000F057B8ADF1080C6DE98D
:108D300004CE002909DB002B1ADB00F04FF8DDF828
:108D400004E0DDE9022304B07047404261EB4101D9
:108D5000002B1BDB00F042F8DDF804E0DDE9022324
:108D600004B0404261EB4101524263EB4303704760
:108D7000524263EB430300F031F8DDF804E0DDE933
:108D8000022304B0404261EB41017047524263EB61
:108D9000430300F023F8DDF804E0DDE9022304B02A
:108DA000524263EB4303704753B94AB9002908BFE5
:108DB00000281CBF4FF0FF314FF0FF3000F00CB81F
:108DC000ADF1080C6DE904CE00F008F8DDF804E020
:108DD000DDE9022304B07047704700BF2DE9F0477A
:108DE00086468C460846089E154674461946002B52
:108DF00040F0C1808542B2FA82F245D94AB1C2F14F
:108E0000200300FA02FC954094402EFA03F343EA53
:108E10000C0C4FEA154EA8B2230CBCFBFEF80EFB5F
:108E200018CC08FB00F943EA0C43994528D9EB1804
:108E300008F1FF3704D2994502D9A8F102072B4463
:108E4000A3EB0903A4B2B3FBFEFC0EFB1C330CFB2B
:108E500000F044EA0344A04214D92C190CF1FF336A
:108E600004D2A04202D9ACF102032C44241A43EAF2
:108E700007401EB1D440002334607360BDE8F08722
:108E80004746DDE76346F1E792BB431B01214FEA0A
:108E9000154EAFB2200CB3FBFEFC0EFB1C330CFBDB
:108EA00007F840EA0343984561D9EB180CF1FF300D
:108EB00004D2984502D9ACF102002B44A3EB08037D
:108EC000A4B2B3FBFEFC0EFB1C330CFB07F744EA19
:108ED0000344A7424DD92C190CF1FF3304D2A74209
:108EE00002D9ACF102032C44E41B43EA0040C0E782
:108EF000C2F120039540944020FA03F12EFA03F3C7
:108F00004FEA154E9040AFB20343B1FBFEFC0EFB9F
:108F10001C10190C0CFB07F841EA0041884522D9C6
:108F200069180CF1FF3004D2884502D9ACF1020077
:108F30002944A1EB08019BB2B1FBFEFC0EFB1C1106
:108F40000CFB07F743EA01439F420ED9EB180CF1E3
:108F5000FF3104D29F4202D9ACF102012B44DB1B4A
:108F600041EA004193E76046E3E76146F7E7604680
:108F7000A4E76346B8E7834206D916B9002108463C
:108F80007CE7C6E900E0F9E7B3FA83F78FB98342DB
:108F900001D3724508D8BEEB020460EB0303012045
:108FA0009C461EB9002169E73846FAE7C6E9004C3D
:108FB000F8E7C7F1200CBB400EFA07F522FA0CF4D3
:108FC0002EFA0CF1BA401C4320FA0CF3B8404FEAD9
:108FD000144901431FFA84FEB3FBF9F809FB18306A
:108FE0000B0C08FB0EFA43EA00439A4540D9E318FC
:108FF00008F1FF3004D29A4502D9A8F102002344B7
:10900000A3EB0A0389B2B3FBF9F809FB183308FB99
:109010000EFE41EA03418E452CD9611808F1FF3359
:1090200004D28E4502D9A8F10203214443EA00404C
:10903000A1EB0E01A0FB02984145CE46434602D368
:1090400006D14D4504D20138B9EB020E68EB04039A
:10905000002EA7D0B5EB0E0261EB030101FA0CFC68
:1090600022FA07F3F9404CEA0303C6E9003199E715
:109070004046C5E74346D9E710F8012B11F8013BFC
:10908000012A28BF9A42F7D0D01A7047034613F836
:10909000012B002AFBD1181A01387047000000008C
:1090A0002DE9F0419846002386B0CDE9043304232E
:1090B0000D46174606460193002800F0B5800029AA
:1090C00000F0B280062104A810F060F8044648B110
:1090D00003460121584A594810F0B8F9204606B015
:1090E000BDE8F081014604AA304610F02AF8044693
:1090F00048B10346524A0121504810F0A7F904A88C
:1091000010F06EF8EAE76A46012104A810F01AF997
:10911000044610B103464B4AEDE7009BB3B1042B64
:109120001AD0052B0CBF0923FF232B70032101ABA1
:1091300002AA04A810F032F9064678B10346424A62
:1091400001213E4810F082F93446D8E70023002080
:109150002B706860A860D2E70723E6E7019B002B2D
:10916000F4D018336B4403F8100C02A9384612F0FF
:109170003EF90222314602A80CF096FE2B78C0B2CE
:10918000092B06D10F2824D96FF0150423462F4A46
:10919000B1E70F28F8D8072B22D12D4B2D4F33F8EC
:1091A0001000D8B1FFF7D6F921A3D3E90023FFF7C8
:1091B0003BFAFFF74BFC042168600DEB010302AAA8
:1091C00004A8019110F0EAF8064660B10346224A6D
:1091D000B6E7224B224F33F81000E2E72148EAE7D6
:1091E0006FF07F04D2E7019B02A918336B4403F8A8
:1091F000100C404612F0FBF80222314602A80CF097
:1092000053FEC3B20F2B07D90121174A0B4810F0A8
:109210001DF96FF0150472E7581CC0B2FFF720FD6E
:109220003946FEF791FF95E76FF0150456E700BF4A
:109230007B14AE47E17A24404FDB0200F0BB020012
:1092400078DB0200A1DB0200C3DB0200EFDB0200DF
:1092500018C302000AD7A33F13DC0200F8C20200C1
:109260000AD723400AD7A3403EDC0200F8B502F13A
:10927000080323F0070300AFADEB030D0546684676
:10928000144612F090F800236E460DF804308AB0B0
:109290006A460849D661C2E90515074911620749BE
:1092A00042F8101F4FF42351054802F0D5F8BD468F
:1092B000F8BD00BF3EC3020000020103040000022B
:1092C00008BC02002DE9F04389B00B7806460C4635
:1092D00002AF092B00F2D680DFE813F00A0040004D
:1092E0004400C000D400D400D400C700D400CE0095
:1092F000CD6935B12B46644A012164480DF021FB4C
:1093000028E00321624A61480EF067FA614B07F1D9
:109310000C0493E80700604B84E807007C606C460F
:109320008AB0BB6002AA5D4B53615D4B936105231C
:10933000D3614FF4007313845A4B42F8103F4FF43B
:10934000135152482B4602F087F83046A546391D86
:109350000FF048FA1C37BD46BDE8F083CB69524A8E
:109360000321CAE74A69CB690321009247484F4A63
:109370000EF046FAD4F81480B8F1800F12D9DFF855
:10938000309149463046A8F180020FF0D8FA051E08
:1093900027D028DBA8EB0508B8F1800FF1D86FF0D3
:1093A000790901E04FF000094246304640490FF08C
:1093B000C9FA0546B8B9237B012B06D1238B304669
:1093C000BB8107F10C010FF0BFF9B9F1000F16D006
:1093D00063698022012100922C48364A0EF010FA6F
:1093E000B8E76FF00405237B012B06D1238B3046B1
:1093F000BB8107F10C010FF0A7F9002D17DB6269A3
:109400002B492D48FFF732FF05222C49284811F03F
:10941000F6FF10B90FF06CFE9CE70622284924489D
:1094200011F0EDFF002895D10FF065FE92E715F1E0
:109430007A0FCDD02B460121224A14480DF081FA33
:109440000321214A11480EF0C8F930460FF0A2F965
:10945000034600283FF47EAF1C4A4DE7CB690BB1B1
:109460001B4A49E78B881B4A7AE7CB690BB11A4A3A
:1094700042E78B88194A73E7CB69002B3FF46AAF48
:10948000174A39E7174A6BE743C3020008BC0200DA
:109490005BC3020050BC02000100D20471C3020091
:1094A0008BC302000400000191C30200AEC302009E
:1094B00052DC0020CCC302001BC4020026C4020000
:1094C0002CC4020033C4020053C4020070C4020062
:1094D00089C402009FC40200B4C40200CAC40200CE
:1094E000DFC40200F7C402002DE9F0434FF0050885
:1094F00089B0DFF8749000AF064614461D46C7E9F0
:1095000005233974C7F80890C7F80C80042178182F
:1095100003F000F97B682A46BB83BB7F214623F01A
:10952000030312486C46BB77FFF7A0FE8AB06A4679
:109530000F4BC2F81C80C2E905394FF40073138445
:109540000C4B42F8103F00234FF413510A4801F02E
:1095500083FF07F10801A54630460FF0B1F8243724
:10956000BD46BDE8F08300BF15C502001BC5020063
:1095700028C502000400000108BC02002DE9F04FDC
:1095800001269DB002AF07F1140804460FF03FF822
:1095900054220021404611F013FF3B464246002171
:1095A000C7E9076645480EF048FA054688B1034604
:1095B0003146434A43480DF0C4F9434A31464148D5
:1095C0000EF00BF96FF0090528466C37BD46BDE873
:1095D000F08F4FF0080A3E68DFF8F09039482EB35C
:1095E000B369082B4AD1F36939495B6801204B60A4
:1095F00045F6073308804B803E1D10233246043168
:1096000003F08CFAE94688B002AB324AC3E905267A
:109610004FF400729A831A462F4B42F8103F0023F2
:109620004FF4E651274801F017FFCD4638680EF099
:1096300006FA274B17216363284B4046A364284A48
:1096400009F0F2F8034668B30121264A1D480DF0DF
:1096500078F92548E062FFF719FD042284F85E20BE
:10966000224A0023E26480222149C4E90E33C4E97E
:1096700015122063226584F82430A5E7EB468AB0F2
:1096800002AAC2E90593182313620523C2F81CA09D
:1096900042F8103F00234FF4215101F0DDFEDD467A
:1096A00036689BE787F823000F231421114ACDF871
:1096B00000800D480CF00AFACBE700BF3DC5020060
:1096C0004BC5020008BC020062C502009FC5020033
:1096D00020DC002089C5020003000001C5920100C2
:1096E000C2C50200CAC502003EDC002052DD0020D7
:1096F000D2DC0020EBC502002123012110B5074A6E
:109700000748FFF7F1FE034630B1BDE810400321E2
:10971000044A05480DF025B910BD00BFF4C502008C
:1097200018D3002016C6020008BC020098B50446F3
:109730000321224A224800AF0DF011F923781BB112
:10974000032B20D0BD4698BD237A012B19D0052BC1
:10975000F8D11C4B6C4688B06A461B49C2E9051318
:109760004FF400739383194B42F8103F00234FF4DA
:10977000E651134801F070FEA54615480BF082F83B
:10978000E0E7144BE6E7217A134A144B6C4688B0A5
:10979000012908BF13466A461149C2E905134FF46F
:1097A00000739383094B42F8103F00234FF4E651B6
:1097B000034801F051FEA546C4E700BF6DC6020094
:1097C00008BC02004AC6020079C60200030000017C
:1097D00020C9002031C602005EC6020068C6020031
:1097E00099C602002DE9F047002582B0624C0321A2
:1097F000624A634802AF0DF0B2F82E46A146DFF888
:109800008481DFF87CA194F8543053B1B4F852301D
:10981000B4F8562003210092504642460DF0F0FF66
:10982000013501360C2E04F10C04ECD12B4603213A
:10983000554A53480DF095F80122E8214E480AF0A8
:10984000B3F9804640B103460121504A4C480DF01F
:1098500088F8BD46BDE8F08799F85030DB07F8D5A9
:109860000FF046FCD9E9000100220023FEF726FD97
:109870006D4688B002AC0426A246454BC4E90601F9
:1098800063614AF8106F4FF40351434652463C4817
:1098900001F0E2FDD9E90201AD4600220023FEF706
:1098A0000DFD88B03B4BC4E90601636126614FF4AE
:1098B000035143465246324801F0CEFDAD460021E9
:1098C000D9F81000FFF718F988B0334B6361FEF741
:1098D00053FE2661C4E906014FF403514346524644
:1098E000274801F0B9FDAD468AB099F8384099F89B
:1098F000390099F83A10B9F83C3002AA53620623AD
:10990000DFF898C0C2E90701C2E905C442F8103F78
:10991000234C43464FF44351194801F09DFD94F800
:109920000080AD46B8F1000F93D111F030FB88B044
:109930000DF108094FF47A721A4BC9F81430A0FBE4
:10994000020302FB0131C00B4FF47A72002340EA9C
:109950004140C90BFFF7D8F94A46C9E9060142F868
:10996000106F4FF403514346054801F075FD012384
:10997000AD4623706DE700BFD8C90020A6C602001F
:1099800008BC0200B3C60200C3C60200E4C602005F
:1099900007C702001DC7020033C702004BC7020001
:1099A000D2DD00206FC70200072805D0092808D0A3
:1099B000012808D1FFF716BF034A032103480CF022
:1099C000CEBF034AF9E770478CC7020008BC02000B
:1099D0009EC70200F8B500AF6C4688B06A46724B6D
:1099E0005361724B93614FF400739383704B42F851
:1099F000103F00234FF4E6516E4801F02DFDA546BF
:109A000005F0E8F820B101216B4A6A480CF0A7FF85
:109A100003216A4A67480CF0A2FF04F0F3F90346F9
:109A200060B1674A012163480CF09BFF0121654A40
:109A300060480CF094FF0020BD46F8BD0321624A47
:109A40005C480CF08CFF61480FF0E4FC034608B161
:109A50005F4AE7E74FF0FF324FF0FF335D480AF00F
:109A600035FF544803215C4A0CF079FF5B480AF04B
:109A70002BFAC8B15A4A01214E480CF070FF5948E0
:109A800005F0D8F820B10121574A4A480CF067FF89
:109A90005648FFF773FD0346002838D0544A012189
:109AA00044480CF05EFFC6E70321524A41480CF0DF
:109AB00056FF0AF099F9044608B14F4ADBE70FF068
:109AC00017FB00214FF480300BF0E6FB20460FF02F
:109AD00012FBD4E701340AD03C230321474A35481E
:109AE0000CF03FFF4FF4F01000210BF0D5FB0321E9
:109AF000434A30480CF033FF3C480EF09FFD0346CC
:109B000040B1404A01212B480CF02BFFE2E704460C
:109B10003D4DECE7294635480CF015FF0346F8B9F2
:109B2000324E30460EF0D3FE0246012128460EF09A
:109B30007DF8002816DA0DF07EFF344A0368012113
:109B40001C480CF00EFF0321314A1A480CF007FFA5
:109B500026480EF01FFE03460028BBD02D4AD1E751
:109B60002D4A9CE730460EF08DFE034620B110F1E1
:109B70000B0F01D0294AE2E7EB88D90706D530461A
:109B80000EF0BCFE034608B1254AD8E7B5F9063009
:109B90001A0705D5234A012106480CF0E0FED2E75A
:109BA0009B06BED5204AF6E7B9C70200D5C702001A
:109BB0000300000108BC0200DFC7020004C8020065
:109BC0001FC80200F1C8020051C802002D97010011
:109BD0006BC8020020C9002094C80200A9990100A6
:109BE000ADC80200676902000FC9020018D3002047
:109BF00038C90200CEC80200DCC802005DC90200FC
:109C00007BC90200A3C9020010D30020D3C90200FF
:109C100027CA020041CA0200BDC90200E7C902000A
:109C2000FEC9020016CA02001ECA02002DE9F04F4A
:109C300091B0009302F004030293C2F3C203013314
:109C4000840705460E46DDF868900392059340F0C0
:109C5000BB81041D30B1072909D86FF01B0011B07A
:109C6000BDE8F08F01F00706341DC6F10806009B21
:109C70004FF000084FF0040A591E4FF0FF334746DB
:109C80000193C3465346CDF810800DB1009A22606F
:109C90000598002800F3E8809848009A824203D390
:109CA00097488242C0F0E080039AA4EB050E920729
:109CB0004FEA9E0000F103810F2F00F2B180002DCA
:109CC00000F0058107F140020DEB020C019A0CF83F
:109CD000200C0CF8102C049801300490E7E07A284E
:109CE0005DD84B280ED8472859D829282DD82528A3
:109CF00052D054D820287AD02338D0F1000B4BEB27
:109D0000000B74E04C382E2849D8DFE800F070488A
:109D1000484848484848484848484B4848484848C0
:109D200048484859484B4B595959704B6D487048F1
:109D3000184B184848827F4B48484B487F0000200A
:109D40004FF0000B4FF0040A38E001222A38C0B26D
:109D500002FA00F010EA0E0F49D110F0625C2FD128
:109D600010EA020B43D06046013C5444B4FBFAF4C1
:109D70000AFB04F4002D61D0A3EB050CA444B44508
:109D80003FF66BAF002868D1042B47D159F8043B4C
:109D90002360042304342AE0019A013A01924FF02F
:109DA000000B24E011F8010C6C2834D1002011F8CC
:109DB000023C83466C2BC5D14FF0080A5346D3E7CB
:109DC00009F1070929F00709073424F00704F9E825
:109DD00002AB35B106982044B0423FF63EAFC4E92D
:109DE00000AB4FF0000B08344FF0080A534611F84F
:109DF000010F002878D0BBF1000F7FF470AF252849
:109E0000F5D14FF0010B019B013301934FF0040A90
:109E1000ECE7584694E700208346A5E7082B02D0DC
:109E20006FF015001BE709F1070929F00709F9E8A8
:109E30000223C4E9002308230834D8E768B9042BB7
:109E400002D109F10409A4E7082BE9D109F10709B6
:109E500029F0070909F10809EDE7059A013A059289
:109E600059F8042B009210E7039A900720D54FF081
:109E7000010CA4EB050E4FEA9E00BEF5007FCFD289
:109E80000F2FCDD8F5B107F140020DEB020E019A6C
:109E9000C0B20EF8200C0EF8102CBCF1000F3FF4ED
:109EA0001AAF60F07F000EF8200C08F101080137AE
:109EB000C5F108024FF6DA7E0434069297E74FF0B8
:109EC000000CDAE7BCF1000F01D00136EFE7029891
:109ED00002360028EBD10098CDE90631FFF7D6F81D
:109EE000DDE906310644E2E7631BB3F5806F97D2E4
:109EF00045B9A6F10804E018B1E600BFACB802000D
:109F00004CEA0200029A9B0828602B709DF81030E2
:109F1000C2B1EB7085F80280B8F1000F05D00022C5
:109F200008A8C5F1010C97420ED14FF0000AC5F107
:109F300001030DF1200901930DF1300B574512D1AA
:109F4000601B8CE66B70E5E710F8013B190608D53D
:109F500004EB0C0EB64503F07F033FF67EAE04F82B
:109F6000013B0132DFE7B8F1000F03D099F900207F
:109F7000002A17DB029BD3B11AF80B2004F8012B3F
:109F80000022019B98182044B0423FF666AE99F833
:109F90000000009904F8010B2046039211F003FA27
:109FA000039A14440AF1010A09F10109C6E799F874
:109FB000002055F822300093029B009845F822308B
:109FC000FFF764F8421CDCE76FF00D0047E600BFC6
:109FD0002DE9F04F97B000AFD7F880B03B62CBF3DC
:109FE000C0030446894690F802A0FA62BB6141B9F9
:109FF000457800780AEB800020444D4517D8A0EB47
:10A000000409E378FB61BAF1000F02D01BF0010FE5
:10A0100016D1FB6953BBFB6A1BB1494620463A6A1D
:10A0200098474D4628465C37BD46BDE8F08F461C34
:10A030003046FFF72BF80130304409F10109DCE725
:10A04000626823787A62FA6A9900796104EB830185
:10A05000002A40F001810E464FF000084D4601EB0A
:10A060000A094E454CD101EB0A0610E01BF0020F25
:10A07000D1D023789A007A61626804EB83017A6216
:10A08000FA6A002A77D14D46904601EB0A061BF08A
:10A09000050F0CBF02230123FB62FB6906EB430A99
:10A0A0000BF00203BB625645BCD016F8021B16F833
:10A0B000013C54F82390AF4B994502D3AE4B9945E0
:10A0C00036D3BB69002B40D0786A0CF031FF0028F2
:10A0D0003BD0E9468AB06A46A84B53617B6AC2E925
:10A0E00006314FF400731384A54B42F8103F002350
:10A0F0004FF41251A34801F0AFF9023DCD46D2E72B
:10A1000016F8013BF96254F82300FEF7BFFFD7F8B9
:10A110008430F96A01304BB1D7F8883098453EBF9A
:10A12000D7F8843023F8180008F10108054498E7AF
:10A13000BB6923B1786A0CF0FBFE0028C9D11BF083
:10A14000010F05D1FB6AED1AADE7BB6A002BAAD05F
:10A150004846FEF79BFFD7F8843053B1D7F88830D4
:10A1600098453FBFD7F88420431C22F8183008F1E7
:10A170000108054497E7BAF1000F73D01BF00406FD
:10A1800073D0D046002607F1480052463B61B962C1
:10A1900011F009F9B96A3B6901EB0A02BA62FA697E
:10A1A000F9695200FA60BA6A02EB41023A610BF0B7
:10A1B0000202BA603A69B96A8A4258D162781BF0E1
:10A1C000020F18BF00217A6208BF4FEA5801B21887
:10A1D0001BF0010FD2B240F09F801BF0040F14BFA0
:10A1E00040460020BB616270A070E17020463A6A70
:10A1F0007969FB6A9847051EFFF614AFBB694146B3
:10A2000023707B6A3A6A6370FB6984F802A0E3708A
:10A2100007F14800FB6A9847B0F10008C0F2B4802B
:10A220007B69A9EB0A01C91AFB683A6AC91AD7E91E
:10A230000A0398470028C0F2A9804FF0000BA844F9
:10A2400008EB000507F1380AB34567D300213A6AE5
:10A250000846FB6A9847E5E656464FF0000807F1C6
:10A26000380092E75646D04696E7B04694E7BA6A79
:10A2700012F8021B12F8015CBA6254F825003D4A3C
:10A28000904202D33C4A90421ED3BA6932B1786AF6
:10A290007B600CF04DFE7B6800288BD1BA6802BB56
:10A2A00008F1280207F1300C08F10100944407F18D
:10A2B000580208F1020852FA80F00CF8101C5FFAFC
:10A2C00088F800F8105C75E7BA693AB1786A7B6083
:10A2D0000CF02EFE7B6800287FF46CAF1BF0010FA2
:10A2E00009D006F1280207F13000711C161806F893
:10A2F000205CCEB25EE71BF0040F3FF45BAF08F1C9
:10A30000280207F1300008F1010102EB000808F80B
:10A31000105C5FFA81F84DE7002063E71BF80A3014
:10A3200054F8239087F83730D7F88430FBB133F8EE
:10A330001B8001213A6AFB6A07F137009847002821
:10A3400024DB0544B8F1000F06D14846FEF79EFE17
:10A3500000F101081FFA88F8414648463A6AFB6A4C
:10A360009847002812DB05440BF1010B6CE7D7F886
:10A370008480DEE7ACB802004CEA02006FCA02003B
:10A3800004000001C0BB020045464BE6054649E615
:10A39000014B1860704700BF80C5002030B5002514
:10A3A00087B0CDE903010446009503A9054805954A
:10A3B00000F010F9DDE904309842B8BF255407B029
:10A3C00030BD00BF7F6F0200032808B506D90DF02D
:10A3D00032FB092303604FF0FF3008BD2822044BF5
:10A3E00002FB0033D3E8AF3F002BF0D00020F4E7AE
:10A3F00088D3002070B504460E461546FFF7E4FFEB
:10A4000000280DDB28236343064AD11849683160D0
:10A4100015B10C3313442B6028235C43105970BDD5
:10A420000020FCE780D3002070B500254FF0FF33FB
:10A430004FF0FF3217480AF03FF9174BD3E8AF2F20
:10A440007AB10135042D03F12803F7D10DF0F3FAA9
:10A4500017234FF0FF3503600E480AF0A5F9284690
:10A4600070BD28246C43D3E8EF0F0130C3E8E10F3F
:10A470000029F8D1094E331932515A6004F10C0009
:10A48000304410F01BFB04F12000304410F017FCA6
:10A49000E2E700BF78C8002088D3002080D30020E6
:10A4A00010B40446104628225443084B1A19195177
:10A4B000506040B1C26832B10C34234440F20512FE
:10A4C00010BC0CF093BD10BC704700BF80D30020BF
:10A4D0002823434330B50D4908330B44D3E8AF2F4D
:10A4E00092B1541ED3E8EF5F954204D1C3E8EC4F1C
:10A4F000BCF1000FF6D1F1D1012A05D12823584330
:10A5000000230A180B50536030BD00BF80D30020D9
:10A51000F0B5024601680A270020074E0B461C785A
:10A520000131355D6D0701D41360F0BD07FB0043B9
:10A53000A3F13000F2E700BFD0E802002DE9F84FA8
:10A5400015469A46D378224A6F2B12F803B08046FC
:10A550000F460BF0030B29D024D8582B0CBF102624
:10A560000A26DDF828903246002340463946FEF799
:10A570001BFC092AD4B21ED83034B045E4B277F1BE
:10A58000000709F8014D01D3D14511D82B789B065E
:10A5900005D5082E15D1AB7843F00803AB704846BB
:10A5A000BDE8F88F03F0F703702BD7E70826D8E74C
:10A5B00080460F46D7E7BBF1010F0CBF3734573445
:10A5C000DBE7102EEBD1AB7843F01003E6E700BFDA
:10A5D000D0E802002DE9F04F8A4616461C460025B9
:10A5E00097B00390307808B928464AE3731C2528B1
:10A5F000049307D05146039B98470028C0F241833B
:10A600000135F0E11822002110A810F0D9FE73786E
:10A61000252B00F0A380002398469E469C461846B2
:10A62000711C0F4611F8012B2B2A00F0C68000F296
:10A63000BD80202A00F0C480232A00F0C4802BB102
:10A640009DF8483043F040038DF84830B8F1000FD2
:10A6500005D09DF8483043F020038DF84830BEF116
:10A66000000F05D09DF8483043F010038DF84830B6
:10A67000BCF1000F05D09DF8483043F008038DF879
:10A68000483028B19DF8483043F004038DF8483035
:10A690009DF8483003F04401442903D16FF3861339
:10A6A0008DF848309DF848302A2A43F080030997F6
:10A6B0008DF8483040F08C809DF8493043F001031C
:10A6C0008DF849307B1C1A782E2A0CBF01210021FD
:10A6D0009DF8492061F341028DF849200CD15A1CA4
:10A6E00009925A782A2A40F083809DF84920023343
:10A6F00042F004028DF849201A786C2A00F0A480F8
:10A7000000F28680682A00F08C806A2A00F0A5801A
:10A710004C2A00F0AA801A4612F8013B782B0492CA
:10A720008DF84B309DF8492000F217816D2B00F217
:10A73000A980692B00F21181572B00F2BE80412BBA
:10A7400003D0453B022B00F2088104229DF84A30D9
:10A7500062F302038DF84A300123CAE0B21C04926E
:10A760008DF84B309DF84930D90740F1FD8054F801
:10A77000048BB8F1000F07DA9DF84820C8F10008F3
:10A7800042F004028DF848205A0740F1F68054F850
:10A7900004BBBBF1000F80F2F5809DF849306FF3E8
:10A7A00041038DF849304FF0FF3BEBE02D2A0DD0EF
:10A7B000302A7FF444AF012333E74FF0010C30E738
:10A7C0004FF0010E2DE74FF001082AE7012028E79E
:10A7D00009A8FFF79DFE099BBB423FF474AF9DF8AB
:10A7E00048201390C00F60F341028DF848206AE7BB
:10A7F00009A8FFF78DFE9DF848301490C3F340027E
:10A8000042EAD07262F341038DF84830099B73E746
:10A81000742A26D07A2A7FF47EAF06219DF849203B
:10A820000CE05A78682A9DF8492006D1012161F38D
:10A83000C6028DF8492002336DE7022161F3C6029A
:10A840008DF84920013366E75A786C2A9DF8492033
:10A8500001D10421EBE70321F0E705219DF8492010
:10A86000ECE707219DF84920E8E7BDF8482022F4ED
:10A87000F04222F0020242F4804242F00202ADF8BD
:10A880004820DFE76E3BD9B201238B4040F2824182
:10A890000B4238D113F0240F52D1DF075DD50321CD
:10A8A0009DF84A3061F302038DF84A3002F07803D4
:10A8B000A3F14000434243411BE00120A3F15801B2
:10A8C000C9B200FA01F111F4624F7FF43EAF40F6D5
:10A8D000010739421DD111F4043F3ED09DF84A30A2
:10A8E00060F3020302F07802402A8DF84A3034D037
:10A8F00000239DF84820C2F340010B4363F341025B
:10A900008DF848202EE702219DF84A3061F30203BA
:10A91000E8E702209DF84A1002F0780260F3020195
:10A92000402A8DF84A1002BF9DF8481041F00101FD
:10A930008DF84810632BDBD1131E18BF0123D8E715
:10A9400003219DF84A3012F0780F61F302038DF86D
:10A950004A3014BF01230023CBE79DF8483043F071
:10A9600001038DF84830C3E79DF94820002AACBFA9
:10A970004FF0FF38DDF84C8006E79F077FF513AFF7
:10A98000DDF850B00023CDE913339DF84A309DF82F
:10A99000491003F00703012BC1F3C30133D1CB1ED0
:10A9A000042B04D8DFE803F0214646212100236868
:10A9B00001294FEAE372CDE910321CD19DF94030F4
:10A9C000DA17CDE9103204349DF8483013F003074C
:10A9D00050D032465146049B03980CF016FB0028D9
:10A9E000C0F24F810544049EFCE554F8043BDA179D
:10A9F000CDE91032E8E70229E5D11AB243F3C033BA
:10AA0000CDE91023DFE7022B24D1CB1E042B04D881
:10AA1000DFE803F018101018180001294FF00002A9
:10AA200054F8043B14D00229CDE91032CCD19BB2AA
:10AA30001093C9E7073424F00704F4E80223CDE9B2
:10AA40001023C1E754F8043B109300231193BBE794
:10AA5000DBB2CDE7042B08D1073424F00704D4E996
:10AA600000230834CDE91023AEE7032BACD154F812
:10AA7000043BDDE79DF84B007828B4D862281DD848
:10AA800025283FF4B7AD5828ADD1DDE910010DF10F
:10AA90003E03009312AA0AABFFF750FDBBF1000F73
:10AAA000814680F29880B9F1000F9CD00DF13E06EE
:10AAB000A6EB0903002F50D001334EE06338152870
:10AAC00091D801A252F820F049AB0100ADAB0100D2
:10AAD000E7A90100E7A90100E7A90100E7A9010032
:10AAE000ADAB0100E7A90100E7A90100E7A901005A
:10AAF000E7A9010037AC0100D1AB0100F9AB0100BF
:10AB0000E7A90100E7A9010021AB0100E7A90100C5
:10AB1000D1AB0100E7A90100E7A90100D1AB010019
:10AB2000BBF1000FDDF840900ADB5946484610F0B3
:10AB30008BFCB9F1000F3FF456AF09EB000676E04D
:10AB40004846FEF7A3FAF8E7109B00278DF8283057
:10AB500001230DF129060DF128099DF84A1011F085
:10AB60001002069200F081800233139A134405927A
:10AB70004A0644BF14995B18B8F1000F40F38E8069
:10AB8000A8EB03089DF848305807C3F3800B00F189
:10AB90008580590678D53FB151463846039B984782
:10ABA00000286EDB5F46013530236EE01E075ABF7A
:10ABB000C3F300135F012B27DDE91023002BBFF641
:10ABC00064AF524263EB43032D27CDE910235CE7CA
:10ABD00000275AE700279DF848100DF13E03A3EB2C
:10ABE00009036FF386119B458DF848107FF65BAF24
:10ABF000ABEB0303139356E7109880B30DF13E06B9
:10AC00000AAB0021009612AAFFF798FCBDF84A3063
:10AC1000BBF1000F03F0EF0343F4F04343F01003E4
:10AC20008146ADF84A30D5DA00283FF4DCAE002783
:10AC3000A6EB090391E7109B07293FF6D4AEDFE8A6
:10AC400001F00C04060C08080C0C1D70CBE61D80EE
:10AC5000C9E6EA17C3E90052C5E61D60C3E6314EF6
:10AC600007460523A6F1050977E7080748BF013322
:10AC70007BE7184607935146039B98470028079B9C
:10AC800004DA17B0BDE8F08F2023C34659460029E7
:10AC90000BF1FF3BEDDC4544D8466D1A37B1514608
:10ACA0003846039B98470028EBDB01359DF84A3076
:10ACB000DA0601D41B0706D551463020039B98477E
:10ACC0000028DEDB0135069B3BB151469DF84B0069
:10ACD000039B98470028D4DB0135059F2F4406E0ED
:10ACE00051463020039B98470028CADB01357B1B67
:10ACF000002BF5DC33464A46514603980CF085F9A3
:10AD00000028BEDB0544A844A8EB0503002B7FF711
:10AD10006AAE51462020039B98470028B1DB0135DD
:10AD2000F2E700BF28CB02002DE9F047058B04466F
:10AD30002807904611D4022905F0070540F0CC8081
:10AD400020460CF0CDFB78B10138218B042811D8B6
:10AD5000DFE800F0C2106D85950001290CBF45F0B9
:10AD6000100545F02005258388F31188BFF36F8F08
:10AD7000BDE8F08701F0070AAA4500F0A58000278A
:10AD8000B9463E46A368002B00F0BC8041F00801A4
:10AD9000218388F31188BFF36F8FA168002900F029
:10ADA000BA800D68002900F0B6803346524620462E
:10ADB000D1F80480C047002D76D02B6829461D4667
:10ADC000F0E701F007035A1F012A1BD8002221F0E7
:10ADD0000701062B276889B2C4E9002209D13B4646
:10ADE00003E0628B013262831B68002BF9D141F0D2
:10ADF0000201204621830CF073FB00287AD041F039
:10AE0000200176E0042B0AD121F0070189B2204607
:10AE100021830CF065FB10B141F020012183218BCF
:10AE200001F0070AAA454FD00027B946AAE72369CF
:10AE300021F0070141F00601062DD3F8009021838F
:10AE40002DD1B9F1000F3FD041F00801218388F3E3
:10AE50001188BFF36F8F20463949C84729E021F098
:10AE60000701236941F0040189B2042DD3F804904D
:10AE70002183E6D000274FF0040A3E4682E721F006
:10AE80000701236941F0050189B2052DD3F8089027
:10AE90002183D6D000274FF0050A3E4672E70027EF
:10AEA0004FF0060A3E466DE72B4687E7B9F1000FE3
:10AEB000D1D1EFF31188202383F31288BFF36F8F72
:10AEC000238B23F008032383258BEA062ED525F058
:10AED0001003238305F007056669218B002EBFF65A
:10AEE00070AF00232768C4E9003321F0070141F067
:10AEF00001012183218B4FF0000901F0070AAA45C7
:10AF00007FF440AF002F9CD041F00801218388F3EB
:10AF10001188BFF36F8F002FC8D03D683946334684
:10AF2000524620460CF008FB2F46F4E7AB067FF5AF
:10AF30001BAF25F02003238305F0070500E700BFC2
:10AF4000657502002DE9F047044607464FF00109F8
:10AF5000DFF8508014B93846BDE8F08794FAA4F5BC
:10AF6000B5FA85F509FA05F32E0108EB05156FEA28
:10AF7000030A24EA03042B7B002BEBD058F806309D
:10AF80001B694BB94644736804222846196807EACE
:10AF90000A0700F04DFADDE7284698470028D9D186
:10AFA000F0E700BF40BC020030B5002289B00F4975
:10AFB0000F4810F033F8002200230024CDE90623C7
:10AFC0000E230C4DCDE903344FF440722846CDE9F1
:10AFD0000144094B0949009409F0AEFE084928468E
:10AFE0000FF077FE204609B030BD00BF05B001006C
:10AFF00050CF0020C0CA0020DDB2010038E300209D
:10B0000029CB0200014809F03DBC00BF08C900205F
:10B010002DE9F04780461F480F460CF05CFB0646C2
:10B02000002830D000252846BDE8F087237B6BB18F
:10B030002368DB680BB12046984723681B69D3B9A6
:10B04000636804222046196800F0F2F901361034D2
:10B050004C45EBD3B8F1000FE5D0002DE2D02846E7
:10B06000FFF770FF0546002FF7D000214FF4A470C2
:10B070000AF012F9F1E7204698470028E0D00AFAD2
:10B0800006F31D43E2E705464FF0010A024CDFF8E4
:10B090000C90DDE730D4002040BC020050BC020020
:10B0A000014B53F820007047BCBC020008B50346B2
:10B0B00008462BB1044A136000F05EFC002008BD76
:10B0C0006FF01500FBE700BF84C5002010B5044CED
:10B0D000237813B9034809F0D5FB0123237010BD71
:10B0E000D3DD002008C9002010B5044606480CF046
:10B0F000F2FA3CB1054BD3E8EF1F0139C3E8E21F78
:10B10000002AF8D110BD00BF28D400202CD4002084
:10B1100000200146034BD3E8EF0FC3E8E21F002AEB
:10B12000F9D1704728D4002070B5FFF7F1FF05462C
:10B13000074C084EB44200D370BD63685B792BB1F5
:10B1400023685B6813B12946204698471034F1E71D
:10B1500040BC020050BC020010B5044C044920461B
:10B160000CF066F8034B1C6010BD00BFE4C7002064
:10B17000A8BC020020D4002008B50023074A4FF4E1
:10B1800000411370064A07481360074A1360FFF72F
:10B190008DFFBDE80840FFF7DFBF00BFD4DD002012
:10B1A00028D40020D37602002CD4002001460022AF
:10B1B000002301480CF05DB8E4C7002001480CF002
:10B1C000F3B800BFE4C70020024B014618680CF03A
:10B1D0003FB900BF20D4002001480CF074B900BF73
:10B1E000E4C7002070B5264B1878002847D0FFF739
:10B1F000E5FF054670B1234BD3E8EF1F0139C3E8E3
:10B20000E21F002AF8D1204C204EB4422DD328460C
:10B21000FFF7DAFF1E4B1F4C1B68002B19DD0FF0E8
:10B22000B6FE4FF47A72A0FB020302FB0131C30B9E
:10B2300043EA4143D4E900209B1A40F2E9324FEA45
:10B24000D13161EB0001934271F1000101D3FFF7AD
:10B250006BFFD4E9003213F57A7342F10002C4E9BE
:10B260000032BDE87040FFF7B7BF63685B7923B178
:10B270002368294620461B6898471034C5E770BDEF
:10B28000D3DD00202CD4002040BC020050BC0200C2
:10B2900028D4002048CF002070B50D4D297861B921
:10B2A0000120FFF7B5FE0B4C0B4EB44206D3FFF75F
:10B2B00099FF0028FBD101232B7070BD63685B7977
:10B2C0001BB1236820469B6898471034EDE700BF08
:10B2D000D4DD002040BC020050BC020000212DE95A
:10B2E000F0470846FFF794FE044648B340F267680B
:10B2F0004FF0000909F0EEFF1A4B186030B11A4BFD
:10B300001B68092B02DD194809F0BCFA0025184F0B
:10B31000DFF858A044B12046FFF714FE044618B9E0
:10B320004FF0FF384FF0FF39FFF75CFF064628B9B2
:10B33000B5B942464B46504609F0C8FA3546E9E7EA
:10B340004FF0FF384FF0FF39D4E72B689B691BB1F2
:10B3500000222846114698471035BD42F5D3E8E74C
:10B36000044DFAE724D400202CD4002008C9002082
:10B3700050BC020040BC020013B518480CF0ABF9F9
:10B38000174B1B7873B1EFF31184202383F31288DA
:10B39000BFF36F8FFFF726FF84F31188BFF36F8F22
:10B3A00002B010BD0F4B1B68002BF9D050B9002222
:10B3B00000230D48CDE900234FF4004200230AF09A
:10B3C000F1F9EDE70928EBD107480FF033FE074804
:10B3D00002B0BDE8104009F055BA00BF2CD40020DF
:10B3E000D4DD002024D4002050CF002008C9002044
:10B3F00010B5064B04461B6898472146A0600448D8
:10B400000BF0B3FFBDE81040FFF7B6BF84C50020C6
:10B41000E4C70020044A054B9B1AB1EBD30F34BF9D
:10B4200052F8310000207047B8BB020040BC020057
:10B43000084B10B4C31A44681B11013323714368CD
:10B440009A7101224368196043685A7110BCFFF772
:10B450003DBE00BF40BC02002DE9F04F8FB0C1F3EC
:10B460004A2804AF0D469146B8607B600C0DB8F1D8
:10B47000000F63D000264FF0040B4FF00A0A07F1CB
:10B480001403C7F80C80C7E907667E620193CDF804
:10B4900008B0CDF800A007F11C0332464846F96811
:10B4A000FEF796FDB0F5006F03461CD36C468AB0DC
:10B4B000D9F8041004AB26481A46C3E9050140F246
:10B4C000FF71D9614FF400711984224B42F8103F8B
:10B4D0004FF4125133462048FFF7BEFFA5462C37E4
:10B4E000BD46BDE8F08FC0F30A0804F11700184408
:10B4F00020F0070080083B60FFF758FE68F35325F3
:10B50000044690B13B6800F11001C7E9083607F125
:10B510001403F961CDE900A3CDF808B048460F4AFD
:10B52000F96807F11C03FEF753FD68F353252A461B
:10B5300020467B68B9680CF000F9D0E704F11700E9
:10B5400020F007008008FFF731FE0446EDE700BF5A
:10B550003ECB020004000001D8BB02000F770200BE
:10B560002DE9F04F87B00446DDE9105ADDE9126994
:10B570000F4693469846A6B3102133465246002004
:10B58000CDF80090CDF81490FEF750FB014605F180
:10B5900017000844144B04F007040BF0070BE400F9
:10B5A00020F0070003EA412344EA8B1480081C437F
:10B5B0000391FFF7FBFD44EA0554054640B13EB157
:10B5C000334652460399CDF800901030FEF72EFB1B
:10B5D000434622463946284607B0BDE8F04F0CF0F6
:10B5E000ACB83146D3E700BF00FE0F00406820B181
:10B5F000034BC01A40F3CF0070474FF0FF30704745
:10B60000B8BB02000EB403B503AB53F8042B0146DC
:10B61000044801930CF00EF902B05DF804EB03B09E
:10B62000704700BF5D780200CA0605D48B064CBF88
:10B6300002490349FFF7E6BF704700BF64E4020018
:10B6400063E402002DE9F04F89B09A46149B9DF8FF
:10B650004CB00693159B04460593169B0D469046E9
:10B66000179E0493BBF1000F00F09D8006F48073D9
:10B6700007930CF04AF806F00209024600283ED073
:10B6800020469249FFF7BEFF0746B9F1000F08D0E8
:10B6900016F0440F35D12A4620468D49FFF7B2FFF8
:10B6A000074406F0010353B18A4B204653F82B2080
:10B6B000894B8A49002A08BF1A46FFF7A3FF06F400
:10B6C0008073002B49D006F00803002B63D1B8F13A
:10B6D000000F66D0424620468149FFF793FF05469A
:10B6E000069B3D44002B6DD1049B002B73D1F307C7
:10B6F00000F1E58031462046FFF796FFD9E0074686
:10B70000C3E7784B18680028CAD0774B4FF47A7992
:10B710001B684FF46161B5FBF3F5B5FBF0F300FB7B
:10B72000135509FB05F5B3FBF1F2B5FBF0FE4FF045
:10B730003C0C01FB123100FB1E55B1FBFCF309FB75
:10B7400005F5B5FBF0F50CFB131120460091CDE992
:10B7500001E56649FFF756FFA2E706F00803EBB1E3
:10B76000634B204653F82B206249FFF74BFF0546F9
:10B77000B8F1000F05D0424620465949FFF742FF75
:10B780000544BAF1000FABD0524620465A49FFF7A4
:10B7900039FF0544A4E74FF0000AE1E706F0080589
:10B7A000E6E745469CE7BAF1010F069B06D1002B60
:10B7B00065D1049B002B7CD000250CE0002BF8D039
:10B7C0004E485DE04E48069B22464E490BF07FFBFB
:10B7D000049B002B69D0DFF83081DFF83091049FA3
:10B7E0003146102F204628BF10274FF0000AFFF7E0
:10B7F0001BFF554546DC059B494620461A78FFF756
:10B8000001FF4FF0010A1AF0070F03D1414620460D
:10B81000FFF7F8FE57453CD9059B4946204613F8EB
:10B820000A20FFF7EFFE0AF1010ABAF1100FEAD180
:10B830004FF0000A20463649FFF7E4FE5246059BCA
:10B8400020469A5C334B995C11F0970F08BF2E226B
:10B850003149FFF7D7FE0AF1010ABAF1100F1DD0E6
:10B860001AF0070F03D141462046FFF7CBFE57459C
:10B870005246E4D841462046FFF7C4FEEBE7204895
:10B880005D46A0E741462046FFF7BCFE0AF1010AEB
:10B89000AFE720462149FFF7B5FEC4E7059B3B44CF
:10B8A0000593049BDB1B049399D1BBF1000F7FF43C
:10B8B0001EAF204609B0BDE8F04F0BF0C2BF2046D6
:10B8C000054A0649FFF79EFE14E700BF82CB02003F
:10B8D00086CB0200CCBC02007DCB020003D6020066
:10B8E000ABCB020038D4002034D400208FCB020030
:10B8F000E0BC0200AFCB0200B5CB02008B780200A7
:10B900005D78020035780200C2CB0200BACB02009B
:10B91000C4CB0200D0E802005ED90200C0CB020016
:10B9200042F20F7373B58B4228BF0B46056804467D
:10B93000052168460D4A0BF042FB0646636828461F
:10B940000B225B680A490BF067FF63683246694661
:10B9500028465B680BF060FF63681B2228465B6823
:10B9600004490BF059FF02B070BD00BF2EC60200A3
:10B97000E2CB0200C6CB020000210123064A90421E
:10B9800006D8064A01B901231360054B18607047B9
:10B99000012140085B00F2E740420F0034D4002050
:10B9A00038D40020F8B50D460446064F4618B44278
:10B9B00001D12846F8BD14F8011BBB6801485B683B
:10B9C0009847F4E78CB90200014B036000207047F0
:10B9D00028BD020008B504480BF0E4FABDE80840B1
:10B9E00002480BF0DFBA00BF28CC02005DCC020099
:10B9F0002DE9F04706460C4600AF002936D0D1E9C4
:10BA00000012E9468AB06D46A3684FF0050AA846C1
:10BA10001F48C5E90723C5E9050148F810AF002311
:10BA200042464FF421511B48FFF716FDD4E903129B
:10BA3000CD466369AD461848C5E90723C5E9050148
:10BA4000C5F810A0002342464FF421511148FFF7DA
:10BA500003FDCD46E3690121104A0E480BF0C6FEF6
:10BA6000A36901210E4A0B480BF0C0FE012E07D13D
:10BA7000EFF305830B4A31460648103B0BF0B6FE48
:10BA80002146304608F06AFCBD46BDE8F08700BF9D
:10BA90008BCC020028BC0200BACC0200E9CC020028
:10BAA000F8CC020026CD020030BFFFF7FDBF00BF7B
:10BAB000074A936893F90E10002907DB52699342F5
:10BAC0001FBF044A536843F080535360704700BF60
:10BAD000DCDB002000ED00E070B52A4C06460D4688
:10BAE00029482A490BF047FFA36ADB0647D52648B9
:10BAF00027490BF040FF1120A36A1C0704D52248F8
:10BB000024490BF038FF12201E4CA36A990712D566
:10BB100021491D480BF02FFF636BA26A120609D55D
:10BB200001211E4A18480BF061FE1EB1A36A23F0E2
:10BB30008003A3621320134CA36ADE0704D51248C6
:10BB400017490BF018FF1420A36A9C0604D50E4871
:10BB500014490BF010FF15200A4B9A6AD10658BF02
:10BB60009A6A9A6A920642BF5A6A22F400525A624C
:10BB70009A6A42F0FF029A6200232B7070BD102077
:10BB8000BAE700BF00ED00E028BC020039CD02009A
:10BB90004FCD020082CD020095CD0200ADCD020056
:10BBA000C3CD0200E2CD020010B5244C2449254843
:10BBB0000BF0E1FEA36A99013ED5224822490BF021
:10BBC000DAFE1E20A36ADA0104D51E481F490BF0D5
:10BBD000D2FE1F20194CA36ADB0204D519481C4968
:10BBE0000BF0C9FE0220A36A1C0304D515481949AD
:10BBF0000BF0C1FE2120114CA36A590304D5114852
:10BC000015490BF0B8FE2220A36A9A0304D50D480B
:10BC100012490BF0B0FE2320084CA36ADB0304D5C5
:10BC200008480F490BF0A7FE2420A36A6FEA0343DC
:10BC30006FEA1343A36210BD1D20C3E700ED00E0CF
:10BC400011CE020028BC020029CE02003CCE020028
:10BC500056CE020080CE02009ECE0200C3CE02006D
:10BC6000DDCE020070B5294C06460D46284829490C
:10BC70000BF081FEA36AD9043CD5254826490BF078
:10BC80007AFE1720A36A1A0504D5214823490BF030
:10BC900072FE18201D4CA36A9B0512D51C48204932
:10BCA0000BF069FEA36BA26A100409D501211D4A9D
:10BCB00017480BF09BFD1EB1A36A23F40043A36257
:10BCC0001920124CA36A590504D5114816490BF0E6
:10BCD00052FE1A20A36ADA050ED50D4813490BF05F
:10BCE0004AFE1B20094A936A43F47F439362002370
:10BCF0002B7070BD1620C5E7A36A9B04F2D50448DB
:10BD00000B490BF038FE1C20ECE700BF00ED00E013
:10BD100028BC020008CF02001ECF020082CD020024
:10BD20002FCF020048CF02005DCF020078CF020083
:10BD3000E2CD02002DE9F0478AB0694B0446D3F802
:10BD400004A089461646002500AFCAF3080885F30B
:10BD50001188BFF36F8F02F07F43B3F17F4F1ED185
:10BD6000D3071CD4500603D4110708D4012508E0DA
:10BD70005C495D480BF0FFFD16F0040600D04C4610
:10BD800000250023FB71A8F10303092B00F2868034
:10BD9000DFE803F0077C7F798484848484822C46E6
:10BDA000EFE7524950480BF0E6FD00234C4EFB7183
:10BDB000F36A9A0705D54E494B480BF0DCFD00238A
:10BDC00029E0F36A002B01DA4A49F5E7F36A5B00E0
:10BDD000F5D5494944480BF0CEFD7369A26943F497
:10BDE00080737361BFF34F8FBFF36F8F736932F846
:10BDF000022C23F480737361BFF34F8FBFF36F8FF7
:10BE00004DF602739A4228D1236801213B4A3648F5
:10BE10000BF0ECFC2368FA79DAB907F1080604F1B3
:10BE2000200C324620686168083403C26445164617
:10BE3000F7D17A6A002D4ED0C2F3080121B96FEA1A
:10BE400052226FEA42227A62184607F10801FFF790
:10BE5000CFFD2837BD46BDE8F087B36ADBB22BB112
:10BE60000120F91DFFF738FE0346D4E7B36A13F447
:10BE70007F4F04D00120F91DFFF7F4FEF4E7B36A09
:10BE8000B3F5803F9BD3FFF78FFEEDE70020F91D50
:10BE9000E8E70020F91DEFE719498DE7194A6E46DA
:10BEA0001AF4F87F8AB0184B18BF13466A46174930
:10BEB000C2E90513A8F11003D3614FF40073138492
:10BEC000134B42F8103F00234FF411510648FFF77F
:10BED000C3FAB54673E722F4FF7222F00102B2E71B
:10BEE00000ED00E0BECF020028BC0200E1CF02005E
:10BEF000F8CF020019D0020027D0020046D002007D
:10BF000062D00200A5CF020090CF020086D00200CE
:10BF100004000001044B5A6942F010025A615A6948
:10BF200042F480625A61704700ED00E0EFF3088050
:10BF3000EFF3098101B57246FFF7FCFE01BD00BFBA
:10BF4000002080F31488BFF36F8F002080F30A88ED
